:100000000C9445080C9476080C9476080C947608A9
:100010000C9476080C9476080C9476080C94760868
:100020000C9476080C9476080C9476080C94760858
:100030000C9476080C9427730C9476080C9476082C
:100040000C9476080C9476080C9476080C94760838
:100050000C9476080C9476080C9476080C94DC6E5C
:100060000C9476080C94E06C0C9441610C94760826
:100070000C9476080C9476080C9476080C94760808
:100080000C9476080C9476080C9476080C947608F8
:100090000C9476080C9476080C9476080C944B74A7
:1000A0000C9476080C9476080C9476080C947608D8
:1000B0000C9476080C9476080C9476080C947608C8
:1000C0000C9476080C9476080C9476080C941761BE
:1000D0000C94ED600C9476080C94C3600C949960B9
:1000E0000C947608BB35A3370B370437D436C436A7
:1000F000A337A136A337A337A337A337A337C92420
:100100003225A425B82522282A28E428022AB82B3B
:10011000BC2CF32C082D0E2DA337502D542D482E1A
:1001200002307A31B4321433ED336D3474347C35AB
:10013000964242435F43734387439B43B843CC4358
:10014000E043FD431144254439441745566B596B30
:10015000486B4C6B526B906B5D6B616B676B6B6B41
:100160006F6B756B796B7D6B906B836B876B8B6B38
:10017000084AD73B3BCE016E84BCBFFDC12F3D6C0E
:1001800074319ABD56833DDA3D00C77F11BED9E474
:10019000BB4C3E916BAAAABE000000803F076342A1
:1001A00036B79BD8A71A39685618AEBAAB558C1D0E
:1001B0003CB7CC5763BD6DEDFD753EF6177231BF90
:1001C000000000803F08000000BE922449123EABB0
:1001D000AAAA2ABECDCCCC4C3E00000080BEABAA61
:1001E000AAAA3E00000000BF000000803F000000FF
:1001F0000000084178D3BB4387D1133D190E3CC39F
:10020000BD4282AD2B3E68EC8276BED98FE1A93E1D
:100210004C80EFFFBE01C4FF7F3F000000000000E4
:100220004E414E494E495459494E46CDCCCC3D0ADB
:10023000D7233C17B7D13877CC2B329595E6241FBE
:10024000B14F0A000020410000C84200401C462077
:10025000BCBE4CCA1B0E5AAEC59D7400407A10F34A
:100260005A00A0724E18090010A5D4E80000E876E4
:1002700048170000E40B54020000CA9A3B0000003B
:10028000E1F505000080969800000040420F000054
:1002900000A08601000000102700000000E8030015
:1002A0000000006400000000000A000000000001DF
:1002B00000000000002C76D888DC674F0823DFC1DF
:1002C000DFAE59E1B1B796E5E3E453C63AE651999A
:1002D0007696E8E6C28426EB898C9B62ED407C6FC3
:1002E000FCEFBC9C9F40F2BAA56FA5F490055A2A7A
:1002F000F75C936B6CF9676DC11BFCE0E40D47FE86
:10030000F520E6B500D0ED902E030094357705007A
:1003100080841E080000204E0A000000C80C333301
:1003200033330F986E12831141EF8D2114893BE610
:100330005516CFFEE6DB18D1844B381BF77C1D9099
:100340001DA4BBE424203284725E228100C9F12402
:10035000ECA1E53D2723696E707574204453546306
:10036000616C6962726174653A0020766F6C7461C9
:1003700067653D002354757262696469747920551C
:1003800070706572204C696D69743A200020766F38
:100390006C746167653D0023566F6C7461676520FE
:1003A00073656E736F723A002343757272656E7473
:1003B0002073656E736F723A00234E6F206E656511
:1003C0006420746F2063616C69627261746520637C
:1003D000757272656E742073656E736F722100237F
:1003E0004143533731322063757272656E742073E6
:1003F000656E736F72206F666673657420563D007C
:10040000234F322063616C6962726174696F6E3A66
:100410002000576946692049503A00234D53204532
:100420006E61626C656400234D53204469736162A0
:100430006C6564002343757272656E742073656E1B
:10044000736F723A0023506172616D6574657273E7
:10045000004E6F20445320546865726D6F6D657453
:10046000657221004F3220436F6E6300434F32208C
:10047000436F6E630053656E736F72206572726FA7
:10048000722100234E6F2073656E736F72210043DB
:100490004F3220436F6E63004D6561737572696EF4
:1004A0006700234E6F2073656E736F7220666F72E4
:1004B00020504D21004E6F2073656E736F722100C6
:1004C000504D313A322E353A3130004D65617375F9
:1004D00072696E672E2E0054757262696469747950
:1004E00000234E6F2073656E736F7220666F7220EB
:1004F00074656D7020262068756D69646974792152
:10050000004E6F2053656E736F72210020666F720C
:100510002074656D7020262068756D696469747932
:1005200021002353656E736F72204572726F7220C3
:100530000053656E736F72204572726F72210023D3
:1005400057726F6E672073656E736F7220666F727D
:100550002074656D7020262068756D6964697479F2
:10056000210057726F6E672053656E736F722100A2
:1005700054656D702048756D6964697479004C69C3
:1005800067687420496E74656E7369747900466C8F
:10059000616D652049520070482076616C75650078
:1005A00023496E76616C6964206B65792100204D6A
:1005B000756C746973656E736F7273004D756C74CE
:1005C0006973656E736F72730044697361626C6501
:1005D00000456E61626C6500237265706C696573BD
:1005E0003D00232D2D2D2D2D2D2D2D2D2D2D2D2D62
:1005F0002D2D2D2D2D2D2D2D2D2D2D2D2D2D2D2D2B
:100600002D2D2D2D2D2D2D00235265736F6C75749E
:10061000696F6E3A20202000234D696E2056616C70
:1006200075653A2020202000234D61782056616CAA
:1006300075653A202020200023556E69717565206C
:1006400049443A20202020002344726976657220B4
:100650005665723A202020002353656E736F723AFC
:100660002020202020202000232D2D2D2D204D6105
:10067000676E657469632053656E736F72202D2DEC
:100680002D2D2D2D2D2D2D2D2D2D2D2D2D2D2D2D9A
:100690002D2D002020202020202020202020202060
:1006A000202020002020202020202020202020206A
:1006B000202020200020202020202020202020205A
:1006C000202020202000202020202020202020204A
:1006D000202020202020002020202020202020203A
:1006E000202020202020002020202020202020202A
:1006F0002020202020200044433A436C6561722072
:100700004C43440044423A5265736574204C6F6711
:100710006765720044303A566F6C746167650044D7
:10072000393A43757272656E7400566F6C74616706
:10073000652B43757272656E740044383A456C657A
:1007400063747269630044373A4D6F74696F6E0069
:1007500044363A44532054656D700044353A55563A
:1007600020496E74656E736974790044343A4F326F
:1007700020636F6E632E0044333A434F3220636F21
:100780006E632E0044323A504D28313A322E353ABB
:100790003130290044323A504D28313A322E353A20
:1007A0003130292A0044313A54757262696469749F
:1007B000790044303A566F6C7461676500393A6F5E
:1007C0007220334420616363656C2E00393A496EB0
:1007D000636C2E20616E672E00383A704820766177
:1007E0006C756500373A49522054656D7000373A90
:1007F00049522054656D702A00363A4D61676E6526
:10080000746963206669656C6400353A47617320DA
:100810004C6576656C00343A495220466C616D65D2
:1008200000333A4C6967687420496E742E00323A7E
:10083000616E642048656967687400323A54656D7A
:100840007020507265737375726500313A54656D2E
:10085000702048756D696469747900303A536F751A
:100860006E64204C6576656C00303A536F756E642B
:10087000204C6576656C2A0054696D65206C61704A
:1008800073653A00576946692049503A00676574B4
:1008900053656C665465737442697428293A200064
:1008A0006973496E74657272757074456E61626CBD
:1008B00065642831293A2000676574496E74657251
:1008C000727570744D617070696E672831293A20B5
:1008D00000676574496E74657272757074536F75D4
:1008E0007263652831293A2000676574496E746522
:1008F0007272757074536F7572636528293A20009F
:100900006765745261746528293A20332E31343179
:1009100035393F00616363656C2E69734C6F7750A6
:100920006F77657228293A2000616363656C2E69D0
:100930007341736C65657028293A200061636365B3
:100940006C2E6973546170536F757263654F6E5A84
:1009500028293A2000616363656C2E6973546170C5
:10096000536F757263654F6E5928293A2000616391
:1009700063656C2E6973546170536F757263654F54
:100980006E5828293A2000616363656C2E697341B3
:1009900063746976697479536F757263654F6E5AC3
:1009A00028293A2000616363656C2E697341637482
:1009B0006976697479536F757263654F6E5928292A
:1009C0003A200069734163746976697479536F756D
:1009D0007263654F6E5828293A200069735461701C
:1009E000446574656374696F6E4F6E5A28293B20A5
:1009F00066616C73653F200069735461704465746F
:100A0000656374696F6E4F6E5A28293B2074727546
:100A1000653F20006973546170446574656374694F
:100A20006F6E4F6E5928293B2066616C73653F20BD
:100A3000006973546170446574656374696F6E4FC7
:100A40006E5928293B20747275653F2000697354E4
:100A50006170446574656374696F6E4F6E582829C0
:100A60003B2066616C73653F20006973546170447C
:100A70006574656374696F6E4F6E5828293B2074E6
:100A80007275653F20006765745375707072657389
:100A90007342697428293B2066616C73653F2000AE
:100AA0006765745375707072657373426974282931
:100AB0003B20747275653F200069734163746976E9
:100AC000697479416328293A20006973496E61632A
:100AD0007469766974795A456E61626C6564282917
:100AE0003A20006973496E61637469766974795953
:100AF000456E61626C656428293A20006973496E0D
:100B0000616374697669747958456E61626C656475
:100B100028293A2000697341637469766974795AA7
:100B2000456E61626C656428293A200069734163EF
:100B300074697669747959456E61626C65642829B7
:100B40003A20006973416374697669747958456E17
:100B500061626C656428293A200067657446726595
:100B60006546616C6C4475726174696F6E28293AD0
:100B700020006765744672656546616C6C546872E6
:100B80006573686F6C6428293A200067657454693E
:100B90006D65496E616374697669747928293A20B4
:100BA00000676574496E6163746976697479546825
:100BB000726573686F6C64282920006765744163EF
:100BC0007469766974795468726573686F6C6428A7
:100BD000292000676574446F75626C6554617057B5
:100BE000696E646F7728292000676574446F7562A9
:100BF0006C655461704C6174656E637928293A2084
:100C0000006765745461704475726174696F6E2811
:100C1000293A2000676574417869734F6666736589
:100C2000742826782C2026792C20267A293A200030
:100C30006765745461705468726573686F6C64287A
:100C4000293A200058595A2047733A200058595AD7
:100C500020434F554E54533A20007365742067610A
:100C6000696E735B5D3A006761696E735F6F72698D
:100C7000675B5D3A002353657474696E6773206F18
:100C80006620616C6C2073656E736F72733A0043FB
:100C9000616C6962726174696F6E20507265737302
:100CA0007572653D00536561206C6576656C2050FA
:100CB0002863616C63293D00234572726F723A703C
:100CC0007265737375726520424D503038352C2033
:100CD000636865636B20776972696E6721004952AA
:100CE0002054656D702073656E736F7220666F752A
:100CF0006E6400504D322E352073656E736F722016
:100D00006C696B656C7920666F756E6400536F75E6
:100D10006E64204C6576656C2073656E736F72200F
:100D2000666F756E6400576946692049503A0053F2
:100D3000656E736F7220736C6F7420616E642074C3
:100D40007970653A0057656C636F6D6520746F202C
:100D5000456455484B003E4D6F74696F6E20627953
:100D600020756C747261736F6E632073656E736F40
:100D7000723A0A0046696E64696E6720576946696F
:100D800020495000697465726174696F6E3D00732B
:100D9000656E736F72233D0043757272656E7420C9
:100DA0007374617475733A206379636C653D006E8A
:100DB0006379636C653D006E73656E736F72733D2E
:100DC000006D61786E73656E736F72733D00656E52
:100DD00061626C65643D00234D756C746973656E6A
:100DE000736F7273206D6561737572656D656E7476
:100DF0002073657474696E67733A000000210024E3
:100E00000027002A002D00300033000101000004FB
:100E10000107010A0100002200250028002B002EF6
:100E2000003100340002010000050108010B01003F
:100E30000020002300260029002C002F0032000093
:100E40000100000301060109010505050507050864
:100E5000080808020202020A0A080804040404013D
:100E6000010101010101010303030303030303045F
:100E70000707070C0C0C0C0C0C0C0C0202020206EF
:100E8000060606060606060B0B0B0B0B0B0B0B01DF
:100E9000021020200808102040102040800201028B
:100EA0000108040201010204081020408080402053
:100EB000100804020180040201804020100804028E
:100EC000010804020101020408102040800102040C
:100ED000081020408000000A0B02090C0D0E0807C4
:100EE00003040100000000000000000000000000FA
:100EF00000000000000000000000000000000000F2
:100F000000121110000000000000000000000000AE
:100F10000000000000000000000000005EBCE26174
:100F20003FDD83C29C7E20A3FD1F41009D23BE4662
:100F3000DB65F88C11AF32CA57E9744F66662061E1
:100F400069722D636F6E6421004974277320746F7A
:100F50006F20636F6F6C210054656D702069732082
:100F600066696E6521004973206169722D636F6E39
:100F700064206F6E3F004974277320717569746532
:100F800020686F7421004974277320766572792078
:100F9000686F742120004F6666206169722D636F4F
:100FA0006E6421004974277320746F6F20636F6F24
:100FB0006C210054656D702069732066696E65212F
:100FC000004973206169722D636F6E64206F6E3FFC
:100FD000004974277320717569746520686F7421E6
:100FE0000049742773207665727920686F74210038
:100FF00054656D702048756D696469747900736516
:10100000703D006976616C3D006E697465723D00EB
:10101000230023456E64206F66204D756C746973E0
:10102000656E736F72204379636C6523004E6F2089
:1010300073656E736F72210049522054656D70653F
:10104000726174757265004D6561737572696E6762
:101050002E2E004572726F72206E756D6265722061
:10106000666F722074686520617272617920746F96
:10107000206176726167696E67212F6E00416E672D
:101080006C65732F0000B89C139F11241FBECFEF17
:10109000D1E2DEBFCDBF00E00CBF1DE0A0E0B2E0BA
:1010A000ECEBF7E501E00BBF02C007900D92AE3DFF
:1010B000B107D9F725E1AEEDBDE001C01D92AD301D
:1010C000B207E1F718E0C4E4D8E000E006C02197D9
:1010D0000109802FFE010E9410A9C334D10780E0CE
:1010E0000807A9F70E94FC9B0C94CDAB0C94000060
:1010F0002F923F924F925F926F927F928F929F9228
:10110000AF92BF92CF92DF92EF92FF920F931F9315
:10111000CF93DF93CDB7DEB7C654D1090FB6F8949D
:10112000DEBF0FBECDBF0091E70D002321F010926E
:10113000E70D0C9428248091CB139091CC13019748
:1011400009F050C060E070E087EC93E10E941D5D03
:10115000082E000C990B0E9464AB892B09F442C045
:1011600065E77BE0CE0183960E943A5FBE016D5D2C
:101170007F4F87EC93E10E942E5D811127C06BE8C1
:101180007AE0CE0145960E943A5FBE016B5E7F4FCA
:1011900087EC93E10E942E5D811114C06DE27DE029
:1011A000CE0101960E943A5FBE016F5F7F4F87ECD0
:1011B00093E10E942E5D01E0811100E0CE010196D5
:1011C0000E94505ECE0145960E94505ECE018396ED
:1011D0000E94505E002331F067EC73E18BEB93E1EA
:1011E0000E94025E8091CB139091CC13049708F07B
:1011F00042C062EA78E0CE0101960E943A5FBE01E9
:101200006F5F7F4F87EC93E10E942E5D082FCE0128
:1012100001960E94505E002371F161E070E087EC5E
:1012200093E10E941D5D80330CF4845E6AE270E0FD
:10123000681B710987FD73954AE0CE0101960E94F3
:10124000DF5EBE016F5F7F4F87EC93E10E94175E08
:10125000CE0101960E94505E67EC73E18BEB93E147
:101260000E94025E87EC93E10E94495CCB010E94E0
:1012700042240C94282463ED75E0CE0145960E942B
:101280003A5FBE016B5E7F4F87EC93E10E942E5D5B
:10129000811116C067ED75E0CE0101960E943A5F9C
:1012A000BE016F5F7F4F87EC93E10E942E5D01E0EE
:1012B000811101C000E0CE0101960E94505E01C084
:1012C00001E0CE0145960E94505E002309F48BC3D5
:1012D00065E474E0CE0101960E942A5FCE0101967A
:1012E0000E944A7FCE0101960E94505E6BED75E030
:1012F000CE0101960E943A5F6FEA74E1CE01019639
:101300000E94605DBC01CE0145960E94325FCE0115
:1013100045960E944A7FCE0145960E94505ECE01BE
:1013200001960E94505E6091B9047091BA04809158
:10133000BB049091BC040E9438A420E030E048EC4B
:1013400052E40E9488A6AB01BC0122E0CE01459682
:101350000E94845E61EF75E0CE0101960E943A5FC3
:10136000BE016B5E7F4FCE0101960E94605D6BE80F
:1013700077E00E94495DBC01CE0183960E94325FF6
:10138000CE0183960E944A7FCE0183960E94505ED2
:10139000CE0101960E94505ECE0145960E94505E9D
:1013A0004091B5045091B6046091B7047091B804AF
:1013B00024E0CE0145960E94845E66E076E0CE0190
:1013C00001960E943A5FBE016B5E7F4FCE0101968F
:1013D0000E94605DBC01CE0183960E94325FCE0107
:1013E00083960E944A7FCE0183960E94505ECE0172
:1013F00001960E94505ECE0145960E94505E40913B
:10140000A9045091AA046091AB047091AC0422E04D
:10141000CE018F960E94845E4091A1045091A20457
:101420006091A3047091A40423E0CE0189960E94E8
:10143000845E4091AD045091AE046091AF04709110
:10144000B00422E0CE0183960E94845E4091A50400
:101450005091A6046091A7047091A80423E0CE01E6
:1014600045960E94845E63E276E0CE0101960E947A
:101470003A5FBE016B5E7F4FCE0101960E94605DB8
:1014800068E376E00E94495DBE016D5D7F4F0E947A
:10149000605D6BE376E00E94495DBE01675D7F4F52
:1014A0000E94605D68E376E00E94495DBE01615D77
:1014B0007F4F0E94605D61E476E00E94495DBC015F
:1014C000CE01C5960E94325FCE01C5960E944A7F2A
:1014D000CE01C5960E94505ECE0101960E94505EDC
:1014E000CE0145960E94505ECE0183960E94505ECA
:1014F000CE0189960E94505ECE018F960E94505E6A
:1015000064E374E0CE0101960E942A5F00914912C3
:10151000E02E002E000CFF08E114F104A1F520914B
:101520004A1230914B1240914C1250914D1260E092
:1015300070E080EA90E40E9488A6AB01BC0122E042
:10154000CE0183960E94555E66E476E0CE01459614
:101550000E943A5FBE016D5D7F4FCE0145960E94AD
:10156000605D6AE776E00E94495DBC01CE010196AC
:101570000E94C15DCE0145960E94505ECE018396C9
:101580000E94505E0AC021E0E216F10431F461E5E8
:1015900076E0CE0101960E94B35DC70102970297E3
:1015A00038F54AE00402B00111244AE0CE018396E6
:1015B0000E94DF5E6FE576E0CE0145960E943A5FBD
:1015C000BE016D5D7F4FCE0145960E94605D65E76F
:1015D0007BE00E94495DBC01CE0101960E94C15D85
:1015E000CE0145960E94505ECE0183960E94505EC9
:1015F00054E0E516F10419F46BE676E006C065E008
:10160000E616F10434F06DE776E0CE0101960E9413
:10161000B35DBE016F5F7F4FCE0145960E94325F82
:10162000CE0145960E944A7FCE0145960E94505EAB
:1016300065E876E0CE0101960E94ED5D809146124C
:1016400060914712709148124AE0833014F00C9474
:10165000D623CE0183960E94DF5E66E676E0CE0159
:1016600045960E943A5FBE016D5D7F4FCE01459663
:101670000E94605D6DE479E00E94495DBC01CE018D
:1016800001960E94C15DCE0145960E94505ECE013A
:1016900083960E94505EBE016F5F7F4FCE014596DC
:1016A0000E94325FCE0145960E944A7FCE01459648
:1016B0000E94505E40912D0550912E0560912F059E
:1016C0007091300522E0CE0183960E94845E65E928
:1016D00076E0CE0145960E943A5FBE016D5D7F4F78
:1016E000CE0145960E94605D6BEA76E00E94495DFE
:1016F000BC01CE0189960E94325FCE0189960E947C
:101700004A7FCE0189960E94505ECE0145960E9486
:10171000505ECE0183960E94505E40912905509103
:101720002A0560912B0570912C0522E0CE0183964D
:101730000E94845E62EB76E0CE0145960E943A5F9D
:10174000BE016D5D7F4FCE0145960E94605D65ECE8
:1017500076E00E94495DBC01CE0189960E94325F0D
:10176000CE0189960E944A7FCE0189960E94505EE2
:10177000CE0145960E94505ECE0183960E94505E37
:1017800001E9C02E04E0D02EEE24E394F12C09E10F
:1017900080918F04909190048E159F050CF450C099
:1017A000F601A190B1906F014AE0B501CE01899692
:1017B0000E94DF5E4AE0B701CE0183960E94DF5EA1
:1017C00068EC76E0CE0145960E943A5FBE016D5D01
:1017D0007F4FCE0145960E94605D62EA7BE00E94E9
:1017E000495DBE01675D7F4F0E94605D60ED76E000
:1017F0000E94495D0A9DB0010B9D700D1124635E2E
:101800007D4F0E94495DBC01CE018F960E94325FE0
:10181000CE018F960E944A7FCE018F960E94505E25
:10182000CE0145960E94505ECE0183960E94505E86
:10183000CE0189960E94505EFFEFEF1AFF0AA8CFF3
:101840008091901290919112892B71F466ED76E05F
:10185000CE0145960E943A5FCE0145960E944A7F8E
:10186000CE0145960E94505E809190129091911207
:10187000019771F465EE76E0CE0145960E943A5FDD
:10188000CE0145960E944A7FCE0145960E94505E49
:101890008091901290919112029771F46FEE76E020
:1018A000CE0145960E943A5FCE0145960E944A7F3E
:1018B000CE0145960E94505E6091270570912805E3
:1018C0004AE0CE0183960E94DF5E61E077E0CE01C0
:1018D00045960E943A5FBE016D5D7F4FCE014596F1
:1018E0000E94605DBC01CE0189960E94325FCE01EC
:1018F00089960E944A7FCE0189960E94505ECE0151
:1019000045960E94505ECE0183960E94505E4091A3
:10191000190250911A0260911B0270911C0222E080
:10192000CE0183960E94845E6EE177E0CE014596FB
:101930000E943A5FBE016D5D7F4FCE0145960E94C9
:10194000605D66EE7CE00E94495DBC01CE01899637
:101950000E94325FCE0189960E944A7FCE0189960D
:101960000E94505ECE0145960E94505ECE01839645
:101970000E94505E4091150250911602609117022C
:101980007091180222E0CE0183960E94845E6EE27E
:1019900077E0CE0145960E943A5FBE016D5D7F4FB4
:1019A000CE0145960E94605D66EE7CE00E94495D36
:1019B000BC01CE0189960E94325FCE0189960E94B9
:1019C0004A7FCE0189960E94505ECE0145960E94C4
:1019D000505ECE0183960E94505E10921402CE019A
:1019E00001960E94505E8091CB139091CC1383306E
:1019F000910508F035C18130910541F460E070E057
:101A000087EC93E10E941D5D182F58C0029709F0E2
:101A100055C062EA78E0CE0101960E943A5FBE01AD
:101A20006F5F7F4F87EC93E10E942E5D082FCE0100
:101A300001960E94505E002309F440C061E070E00E
:101A400087EC93E10E941D5D682FCE0101960E94F4
:101A50000A5FBE016F5F7F4F8BEB93E10E94175EC1
:101A6000CE0101960E94505E60E070E087EC93E149
:101A70000E941D5D182F8091250E8823F9F06EE3DA
:101A800077E0CE0101960E943A5F67EC73E1CE01E8
:101A900001960E94605D68E87DE00E94495DBC019E
:101AA0008EE990E10E94995FCE0101960E94505EFE
:101AB0006BEB73E18EE990E10E948860812F012E2B
:101AC000000C990B0E9464AB892BB1F00E94EB676C
:101AD0000E94283F68E87DE0CE0101960E943A5FAF
:101AE0004AE050E060E070E0CE0101960E940B40B9
:101AF000CE0101960E94505E123409F443C0CCF42A
:101B0000103309F45FC07CF4133209F452C01A3266
:101B100009F078C067E577E087EC93E10E94ED5D1E
:101B20008FEF9FEF6CC0113309F45BC01134F9F0F3
:101B300069C01136E1F02CF4133479F1143439F022
:101B400061C0133651F1F4F0143609F05BC0809196
:101B5000BF139091C013892B09F47EC08BEB93E1E6
:101B60000E94495C97FD02C00C94E92375C06BE4A8
:101B700077E087EC93E10E94ED5D8091210E9091DA
:101B8000220E3DC06EE477E087EC93E10E94ED5DAC
:101B90001092DE0D8CEF9FEF32C061E577E087ECAD
:101BA00093E10E94ED5D81E08093DE0D8DEF9FEF6C
:101BB00026C064E577E087EC93E10E94ED5D8EEF4F
:101BC0009FEF1DC062EE7CE08BEB93E10E94ED5D28
:101BD00062EE7CE087EC93E10E94ED5D80E090E0B6
:101BE0000EC068E577E08BEB93E10E94ED5D68E560
:101BF00077E087EC93E10E94ED5D81E090E00E9448
:101C000042242AC0612FCE0101960E940A5FBE01C4
:101C10006F5F7F4F8BEB93E10E94175ECE010196C1
:101C20000E94505E60E070E08BEB93E10E941D5DCE
:101C3000082E000C990B0E9464AB892B39F08BEBBA
:101C400093E10E94495CCB010E94422464E670E06B
:101C500080E090E00E94986E0E94D06E0C94C523A4
:101C600021E030E040E050E067EC73E1CE01019606
:101C70000E944E5FBE016F5F7F4F89EA93E10E9431
:101C8000175ECE0101960E94505E67E877E0CE01B4
:101C900045960E943A5FBE016B5E7F4F87EC93E1F1
:101CA0000E942E5D811116C060E97DE0CE01019693
:101CB0000E943A5FBE016F5F7F4F87EC93E10E9405
:101CC0002E5D11E0811101C010E0CE0101960E944D
:101CD000505E01C011E0CE0145960E94505E112376
:101CE00009F4BEC08091CB139091CC13409710F0B3
:101CF0000C94282442E050E067EC73E1CE01019699
:101D00000E94394BBE016F5F7F4F89EA93E10E94C9
:101D1000175ECE0101960E94505E69EA73E1CE0122
:101D200001960E94325FCE0101960E946B45CE0162
:101D300001960E94505E89EA93E10E943E5C20E099
:101D400030E048EC52E40E9497A40E9421A7AB0126
:101D5000BC014093B9045093BA046093BB047093E0
:101D6000BC042AE0CE0101960E94B35ECE0101962A
:101D70000E946B45CE0101960E94505E6091B904AD
:101D80007091BA048091BB049091BC048B019C01BA
:101D900000591F452140310901341C4921053105F5
:101DA00088F06AE577E0CE0101960E943A5F69EA21
:101DB00073E1CE0101960E94605D6DE677E00E94BE
:101DC000495DBFC119821A821B821C821D821E823C
:101DD0001F8218860E9438A420E030E048EC52E4CC
:101DE0000E9488A68E010F5F1F4F22E047E00E94ED
:101DF0003F9FBC018FEA93E10E94ED5D6DE777E0C4
:101E0000CE0145960E943A5F6FEA73E1CE01459696
:101E10000E94605D6AE877E00E94495DBC018FEA3C
:101E200093E10E94025ECE0145960E94505E1092A0
:101E30000615109205158091B9049091BA04A091ED
:101E4000BB04B091BC0480931A1290931B12A09310
:101E50001C12B0931D1280E090E00E943F797AC17D
:101E60006FE877E0CE0145960E943A5FBE016B5E57
:101E70007F4F87EC93E10E942E5D811116C065E9CA
:101E800077E0CE0101960E943A5FBE016F5F7F4FFF
:101E900087EC93E10E942E5D11E0811101C010E0FA
:101EA000CE0101960E94505E01C011E0CE01459620
:101EB0000E94505E112309F46EC026E030E045E038
:101EC00050E067EC73E1CE0101960E944E5FBE01C7
:101ED0006F5F7F4F89EA93E10E94175ECE01019602
:101EE0000E94505E89EA93E10E94495C6B017C018B
:101EF00069EA76E0CE0101960E943A5FBE016F5F0B
:101F00007F4F87EC93E10E94B35CAC014F5F5F4F62
:101F100067EC73E1CE0145960E94394BBE016B5EC2
:101F20007F4F89EA93E10E94175ECE0145960E9499
:101F3000505ECE0101960E94505E89EA93E10E94B4
:101F4000495CDB01EFE8F4E041E050E020918F04D0
:101F500030919004241735075CF0228133812A17D1
:101F60003B0711F4138212824F5F5F4F3296EECF20
:101F70009601220F331FF901E157FB4F71836083F4
:101F800082E090E00E94386967EC73E18EE990E1AD
:101F90000E94886049C06BE977E0CE0145960E94B7
:101FA0003A5FBE016B5E7F4F87EC93E10E942E5D2E
:101FB000811116C061EA77E0CE0101960E943A5F76
:101FC000BE016F5F7F4F87EC93E10E942E5D11E0B1
:101FD000811101C010E0CE0101960E94505E01C047
:101FE00011E0CE0145960E94505E112339F1EFE8D1
:101FF000F4E081E090E020918F0430919004281764
:10200000390774F0863091051CF49383828305C0F0
:102010009C012E5F3F4F3383228301963296EBCF94
:1020200082E090E00E943869109206151092051522
:1020300080E090E00E943F790C94B12367EA77E05A
:10204000CE0145960E943A5FBE016B5E7F4F87ECE2
:1020500093E10E942E5D811116C06EEA77E0CE01F9
:1020600001960E943A5FBE016F5F7F4F87EC93E15C
:102070000E942E5D11E0811101C010E0CE01019699
:102080000E94505E01C011E0CE0145960E94505E54
:102090001123F9F08091C60E9091C70E892BA1F4FF
:1020A00081E090E09093C70E8093C60E8EED93E092
:1020B00090930615809305150E94697968EC70E08D
:1020C00080E090E00E94986EE0E0F0E019950C94BA
:1020D000B32365EB77E0CE0145960E943A5FBE01DF
:1020E0006B5E7F4F87EC93E10E942E5D811116C0DD
:1020F0006DEB77E0CE0101960E943A5FBE016F5F03
:102100007F4F87EC93E10E942E5D11E0811101C0A9
:1021100010E0CE0101960E94505E01C011E0CE0198
:1021200045960E94505E1123F1F065EC77E0CE01F8
:1021300001960E943A5F69EA74E1CE0101960E941D
:10214000605DBC018FEA93E10E94025ECE010196C0
:102150000E94505E61EC7CE0CE0101960E943A5FE5
:102160006FEA73E19BC76FEC77E0CE0145960E9462
:102170003A5FBE016B5E7F4F87EC93E10E942E5D5C
:10218000811116C066ED77E0CE0101960E943A5F9C
:10219000BE016F5F7F4F87EC93E10E942E5D11E0DF
:1021A000811101C010E0CE0101960E94505E01C075
:1021B00011E0CE0145960E94505E112399F06DED1D
:1021C00077E0CE0101960E943A5F6FEA74E1CE019A
:1021D00001960E94605DBC018FEA93E10E94025E5D
:1021E0000C94191E6CEE77E0CE0145960E943A5F82
:1021F000BE016B5E7F4F87EC93E10E942E5D8111E3
:1022000016C063EF77E0CE0101960E943A5FBE01EF
:102210006F5F7F4F87EC93E10E942E5D11E081118B
:1022200001C010E0CE0101960E94505E01C011E095
:10223000CE0145960E94505E112309F48FC069EAD1
:1022400076E0CE0101960E943A5FBE016F5F7F4F3C
:1022500087EC93E10E94B35CAC014F5F5F4F67EC8A
:1022600073E1CE0145960E94394BBE016B5E7F4FF4
:1022700089EA93E10E94175ECE0145960E94505E66
:10228000CE0101960E94505E89EA93E10E94495C6A
:102290008B0167E274E08FEA93E10E94C75D809151
:1022A000A912882331F06BE174E08FEA93E10E9478
:1022B000C75D0115110511F40C94A323CE010196FD
:1022C0000E941462CE0101960E944A7FCE010196BF
:1022D0000E94505E0230110514F40C94B12365E79E
:1022E0007CE0CE0145960E942A5FBE016B5E7F4F67
:1022F000CE0101960E94325FCE0101960E944A7F74
:10230000CE0101960E94505EE12CF12C8091AB121F
:10231000082E000C990BE816F9068CF4B701CE01D3
:1023200001960E944D86CE0101960E944A7FCE0101
:1023300001960E94505EFFEFEF1AFF0AE7CFCE0131
:1023400045960E94505E0230110511F40C94B123A1
:102350008CE291E00E94B9790C94B1236AEF77E0A6
:10236000CE0145960E943A5FBE016B5E7F4F87ECBF
:1023700093E10E942E5D811116C061E078E0CE01EC
:1023800001960E943A5FBE016F5F7F4F87EC93E139
:102390000E942E5D11E0811101C010E0CE01019676
:1023A0000E94505E01C011E0CE0145960E94505E31
:1023B000112309F495C367EC73E1CE018F5B9F4F46
:1023C0000E94325F69EA76E0CE0101960E943A5F90
:1023D000BE016F5F7F4FCE018F5B9F4F0E94B35C4A
:1023E000AC014F5F5F4FBE016F5B7F4FCE01CB965D
:1023F0000E94394BCE0101960E94505EBE016F5B78
:102400007F4FCE0101960E94325FCE0101960E945D
:102410006B45CE0101960E94505E6EEF77E0CE01D3
:1024200001960E943A5FBE016F5F7F4FCE01CB964F
:102430000E94035D8C01CE0101960E94505E6FEBFD
:102440007CE0CE01C5960E943A5F6FEB7CE0CE0146
:102450008F960E943A5F1016110694F5A8014F5FFF
:102460005F4F21968EAD9FAD21974817590790F485
:10247000BE01655C7F4FCE0101960E94394BBE01C3
:102480006F5F7F4FCE01C5960E94175ECE01019609
:102490000E94505E980140E050E0BE01655C7F4FB5
:1024A000CE0101960E944E5FBE016F5F7F4FCE014D
:1024B0008F960E94175ECE0101960E94505E0DC05D
:1024C0006FEB7CE0CE01C5960E94ED5DBE01655CC0
:1024D0007F4FCE018F960E94025E8BA99CA9892B0B
:1024E00009F4EEC2CE018F960E94495C8B01015027
:1024F00011090831110514F007E110E017FF02C0BF
:102500000FEF1FEF4AE0B801CE0145960E94DF5E53
:1025100060E078E0CE0183960E943A5FBE016B5E78
:102520007F4FCE0183960E94605DBC01CE01019673
:102530000E94325FCE0101960E946B45CE0101964A
:102540000E94505ECE0183960E94505ECE01459659
:102550000E94505EBE016B5C7F4FCE01CB960E9405
:10256000025E6EEF77E0CE0101960E943A5FBE01F7
:102570006F5F7F4FCE01CB960E94035D7C01CE0141
:1025800001960E94505E6FEB7CE0CE01C5960E94E2
:10259000ED5D6FEB7CE0CE018F960E94ED5D1E1429
:1025A0001F040CF050C0A7014F5F5F4F21968EAD06
:1025B0009FAD21974817590790F4BE01655C7F4F86
:1025C000CE0101960E94394BBE016F5F7F4FCE0155
:1025D000C5960E94175ECE0101960E94505E97013B
:1025E00040E050E0BE01655C7F4FCE0101960E9445
:1025F0004E5FBE016F5F7F4FCE018F960E94175EC8
:10260000CE0101960E94505EAE014F5F5F4F3A01CE
:10261000E12CF12CA8014F5F5F4F8AE0849F90016D
:10262000859F300D1124B90167557D4E6B01809F48
:102630009001819F300D1124C90189549D4E5C0188
:10264000BAE23B2EC3C06FEB7CE0CE01C5960E9480
:10265000ED5DBE01655C7F4FCE018F960E94025EEC
:10266000D3CFE114F10409F0BEC00F3F9FEF19076B
:1026700009F4B9C0CE018F960E94545CC114D104F4
:1026800039F044E050E0B601CE018F960E94638B92
:10269000B601CE0183960E943A5F65E078E0CE01F4
:1026A00089960E943A5FBE016D5D7F4FCE0189968B
:1026B0000E94605DBC01CE0145960E94325FCE0152
:1026C00045960E946B45CE0145960E94505ECE0114
:1026D00089960E94505ECE0183960E94505E8BA91F
:1026E0009CA9029708F478C061E070E0CE018F9653
:1026F0000E941D5D082E000C990B803391050CF48F
:102700004C96E32DE81B8E2FF5018083FFEFEF1A27
:10271000FF0ABE016B5C7F4FCE01CB960E94025E2A
:102720006EEF77E0CE0145960E943A5FBE016B5E88
:102730007F4FCE01CB960E94035D2C01CE014596C2
:102740000E94505E6FEB7CE0CE01C5960E94ED5D6D
:102750006FEB7CE0CE018F960E94ED5D14141504A2
:102760000CF049C0A2014F5F5F4F21968EAD9FAD27
:1027700021974817590790F4BE01655C7F4FCE0141
:1027800045960E94394BBE016B5E7F4FCE01C596C8
:102790000E94175ECE0145960E94505E920140E075
:1027A00050E0BE01655C7F4FCE0145960E944E5FB2
:1027B000BE016B5E7F4FCE018F960E94175ECE01E9
:1027C00045960E94505E22E0620E711C8BA99CA966
:1027D000892B09F046CF1DC0CE018F960E94495C1F
:1027E000F501608393CFCE018F960E94495CF3017F
:1027F000718360838BCF6FEB7CE0CE01C5960E9426
:10280000ED5DBE01655C7F4FCE018F960E94025E3A
:10281000DACF0F3F4FEF140709F07EC06EEF77E07D
:10282000CE0145960E943A5FBE016B5E7F4FCE019E
:10283000C5960E94035D8C01CE0145960E94505EB4
:1028400017FF3EC109811A811016110634F40931AF
:1028500011052CF008E110E002C001E010E0009347
:10286000AB124AE0B801CE0183960E94DF5E63E1BD
:1028700078E0CE0189960E943A5FBE016D5D7F4F80
:10288000CE0189960E94605DBC01CE0145960E94F2
:10289000325FCE0145960E946B45CE0145960E945F
:1028A000505ECE0189960E94505ECE0183960E94B2
:1028B000505EE114F10459F18B819C8197FF02C0B5
:1028C00080E090E09093AD128093AC1251E0E51659
:1028D000F104E9F08D819E81181619062CF48017F9
:1028E000910724F48C0102C001E010E00150009334
:1028F000B01262E0E616F10451F08F819885181647
:10290000190614F081E090E081508093B1128CE2BE
:1029100091E00E948F79D4C08091AA12082E000CF9
:10292000990B081719070CF084C04AE0B701CE01D3
:1029300083960E94DF5E6DE178E0CE0189960E9469
:102940003A5FBE016D5D7F4FCE0189960E94605D4A
:10295000BC01CE0145960E94325FCE0145960E9491
:102960006B45CE0145960E94505ECE0189960E942D
:10297000505ECE0183960E94505E8AE0809FF001F7
:10298000819FF00D1124E755FD4E81E0878783E09C
:1029900090E0918B808B938B828BE114F10409F48E
:1029A0008FC08B819C818038910514F08FE790E077
:1029B00080387FEF970714F480E89FEF878781E0E6
:1029C000E816F10409F47CC08AE0809FF001819F41
:1029D000F00D1124E755FD4E8D819E8197FF02C0B9
:1029E00080E090E0918B808B92E0E916F10409F48D
:1029F00067C08AE0809FF001819FF00D1124E755A8
:102A0000FD4E8F81988597FF02C080E090E0938B08
:102A1000828B8091AB12082E000C990B08171907B6
:102A20001CF00F5F0093AB128CE291E00E94B97929
:102A300047C0BE016B5C7F4FCE0189960E94325F1A
:102A40006091AA12062E000C770B4AE0CE01459643
:102A50000E94DF5E65E278E0CE0183960E943A5FD5
:102A6000BE01675D7F4FCE0183960E94605D66E385
:102A700078E00E94495DBE016B5E7F4F0E94605D01
:102A8000BC01CE0189960E94025ECE0183960E940F
:102A9000505ECE0145960E94505EBE01675D7F4F3D
:102AA000CE0145960E94325FCE0145960E944A7F34
:102AB000CE0145960E94505ECE0189960E94505EDE
:102AC000CE018F960E94505ECE01C5960E94505E48
:102AD000CE01CB960E94505ECE018F5B9F4FDEC52C
:102AE0006AE378E0CE0145960E943A5FBE016B5ED4
:102AF0007F4F87EC93E10E942E5D811116C06FE33A
:102B000078E0CE0101960E943A5FBE016F5F7F4F71
:102B100087EC93E10E942E5D11E0811101C010E06D
:102B2000CE0101960E94505E01C011E0CE01459693
:102B30000E94505E112309F444C069EA76E0CE0198
:102B400001960E943A5FBE016F5F7F4F87EC93E171
:102B50000E94B35CAC014F5F5F4F67EC73E1CE0145
:102B600045960E94394BBE016B5E7F4F89EA93E127
:102B70000E94175ECE0145960E94505ECE010196DE
:102B80000E94505E89EA93E10E94495C61157105DB
:102B900021F481E08093130210C06130710519F4B3
:102BA000109213020AC06230710511F00C94B12327
:102BB00081E080931302109212020E94FB670C9432
:102BC000B12364E478E0CE0145960E943A5FBE01ED
:102BD0006B5E7F4F87EC93E10E942E5D811116C0E2
:102BE00068E478E0CE0101960E943A5FBE016F5F13
:102BF0007F4F87EC93E10E942E5D11E0811101C0AF
:102C000010E0CE0101960E94505E01C011E0CE019D
:102C100045960E94505E112309F422C143E050E022
:102C200067EC73E1CE0101960E94394BBE016F5FE4
:102C30007F4F89EA93E10E94175ECE0101960E94C0
:102C4000505E69EA73E18EE990E10E94886010921B
:102C500006151092051569EA73E185EB94E10E946F
:102C6000025E69EA73E18FEA94E10E94025E86E304
:102C700092E1009739F048E050E0BC0185EB94E127
:102C80000E94638B84E992E1009739F04CE050E0B8
:102C9000BC018FEA94E10E94638B809105159091AD
:102CA00006150E943F796CE478E0CE0101960E94FF
:102CB0003A5F6FEA74E1CE0101960E94605DBC014B
:102CC000CE0183960E94325FCE0101960E94505E33
:102CD0008091901290919112892B39F4BE016D5D13
:102CE0007F4F84E69FE00E94995F809190129091BF
:102CF0009112029709F09BC06FEA74E1CE018996A8
:102D00000E94325F64E578E0CE0101960E943A5F4E
:102D1000CE0101960E94739CCE0101960E94505EE6
:102D200064EF71E080E090E00E94986E67E578E0E3
:102D3000CE0101960E943A5FCE0101960E94739CDB
:102D4000CE0101960E94505E64EF71E080E090E059
:102D50000E94986E60E678E0CE0101960E943A5F8C
:102D6000CE0101960E94739CCE0101960E94505E96
:102D700064EF71E080E090E00E94986E69E678E090
:102D8000CE0101960E943A5FCE0101960E94739C8B
:102D9000CE0101960E94505E64EF71E080E090E009
:102DA0000E94986E67E778E0CE0101960E943A5F34
:102DB000CE0101960E94739CCE0101960E94505E46
:102DC00064EF71E080E090E00E94986E6CE478E03F
:102DD000CE0101960E943A5FBE01675D7F4FCE0132
:102DE00001960E94605DBC01CE0145960E94325F53
:102DF000CE0101960E94505ECE0145960E94545C21
:102E0000BE016B5E7F4FCE0101960E94325FCE0104
:102E100001960E94739CCE0101960E94505ECE01E5
:102E200045960E94505ECE0189960E94505E68EBE6
:102E30007BE080E090E00E94986E66E372E1CE0154
:102E400001960E943A5FCE0101960E946B45CE0129
:102E500001960E94505E10921402CE0183961EC409
:102E600065E878E0CE0145960E943A5FBE016B5E50
:102E70007F4F87EC93E10E942E5D811116C06AE8B6
:102E800078E0CE0101960E943A5FBE016F5F7F4FEE
:102E900087EC93E10E942E5D11E0811101C010E0EA
:102EA000CE0101960E94505E01C011E0CE01459610
:102EB0000E94505E112309F462C044E050E067ECC8
:102EC00073E1CE0101960E94394BBE016F5F7F4FC7
:102ED00089EA93E10E94175ECE0101960E94505E3E
:102EE0006FE878E0CE0145960E943A5F69EA73E1A7
:102EF000CE0145960E94605DBC01CE0101960E9404
:102F0000325FCE0145960E94505E80919012909162
:102F10009112892B39F4BE016F5F7F4F84E69FE0E9
:102F20000E94995F8091901290919112029779F48A
:102F3000BE016F5F7F4FCE0145960E94325FCE018A
:102F400045960E94739CCE0145960E94505E68EBA8
:102F50007BE080E090E00E94986EBE016F5F7F4F43
:102F6000CE0145960E94325FCE0145960E946B4588
:102F7000CE0145960E94505E109214028DC366E900
:102F800078E0CE0145960E943A5FBE016B5E7F4FAE
:102F900087EC93E10E942E5D811116C06AE978E00A
:102FA000CE0101960E943A5FBE016F5F7F4F87ECB2
:102FB00093E10E942E5D11E0811101C010E0CE016D
:102FC00001960E94505E01C011E0CE0145960E941C
:102FD000505E112309F475C067EC73E189EA93E14F
:102FE0000E94025E81E08093140267EC73E1CE01DF
:102FF00001960E94325FCE0101960E946B45CE0180
:1030000001960E94505E80919012909191120297C9
:1030100009F169EA73E184E69FE00E94995F68EB39
:103020007BE080E090E00E94986ECE0101960E94C5
:10303000B799BE016F5F7F4F87EC93E10E94175EE7
:10304000CE0101960E94505E60ED77E080E090E056
:103050000E94986E8091901290919112029771F453
:1030600069EA73E1CE0101960E94325FCE010196BA
:103070000E94739CCE0101960E94505E8091CB13FA
:103080009091CC13892B11F40C94B12361EC7CE06A
:10309000CE0101960E943A5F67EC73E1CE01019682
:1030A0000E94605DBC01CE0145960E94325FCE0158
:1030B00045960E944A7FCE0145960E94505E0C9430
:1030C000AD236EE978E0CE0145960E943A5FBE01DD
:1030D0006B5E7F4F87EC93E10E942E5D811116C0DD
:1030E00064EA78E0CE0101960E943A5FBE016F5F0C
:1030F0007F4F87EC93E10E942E5D11E0811101C0AA
:1031000010E0CE0101960E94505E01C011E0CE0198
:1031100045960E94505E112309F45DC08091901283
:1031200090919112019711F00C94B123CE01019668
:103130000E942B638D819E81009711F40C94AD2326
:10314000E981FA812081222311F40C94AD230797A1
:1031500010F40C94AD2362E174E0CE0145960E9418
:103160002A5F48EC50E06FEF7FEFCE0145960E945A
:103170000B40CE0145960E94505EBE016F5F7F4FAF
:10318000CE0145960E94325F40ED57E06FEF7FEF32
:10319000CE0145960E948C3FCE0145960E94505E1E
:1031A0006AEA78E0CE0145960E943A5FBE016F5F01
:1031B0007F4FCE0145960E94605DBC01CE01839693
:1031C0000E94325FCE0183960E944A7FCE01839691
:1031D0000E94505E70CF68EB78E0CE0145960E9469
:1031E0003A5FBE016B5E7F4F87EC93E10E942E5DDC
:1031F000811116C06DEB78E0CE0101960E943A5F16
:10320000BE016F5F7F4F87EC93E10E942E5D11E05E
:10321000811101C010E0CE0101960E94505E01C0F4
:1032200011E0CE0145960E94505E1123F1F025E099
:1032300030E044E050E067EC73E1CE0101960E947B
:103240004E5FBE016F5F7F4F89EA93E10E94175E78
:10325000CE0101960E94505E89EA93E10E94495C8A
:10326000709391126093901251C062EC78E0CE019D
:1032700045960E943A5FBE016B5E7F4F87EC93E1FB
:103280000E942E5D811117C067EC78E0CE01019697
:103290000E943A5FBE016F5F7F4F87EC93E10E940F
:1032A0002E5DFF24F394811101C0F12CCE01019613
:1032B0000E94505E02C0FF24F3948E010B5E1F4FEC
:1032C000C8010E94505EFF2089F126E030E044E012
:1032D00050E067EC73E1CE0101960E944E5FBE01A3
:1032E0006F5F7F4F89EA93E10E94175ECE010196DE
:1032F0000E94505E89EA93E10E94495C70939312A8
:1033000060939212709328056093270567EC73E130
:10331000CE0101960E94325FCE0101960E946B455C
:10332000CE0101960E94505E0C9414106CEC78E073
:10333000C8010E943A5FB80187EC93E10E942E5DBC
:10334000811117C063ED78E0CE0101960E943A5FCB
:10335000BE016F5F7F4F87EC93E10E942E5DFF24DB
:10336000F394811101C0F12CCE0101960E94505EB0
:1033700002C0FF24F394C8010E94505EFF2069F14F
:1033800027E030E046E050E067EC73E1CE010196C3
:103390000E944E5FBE016F5F7F4F89EA93E10E94FA
:1033A000175ECE0101960E94505E89EA93E10E9469
:1033B000495C672B19F41092250E03C081E08093BD
:1033C000250E67EC73E1CE0101960E94325FCE01BB
:1033D00001960E946B450C94AD236AED78E0CE0116
:1033E00083960E943A5FBE016D5D7F4F87EC93E14B
:1033F0000E942E5D81112FC06DED78E0C8010E9402
:103400003A5FB80187EC93E10E942E5D811117C0ED
:1034100060EE78E0CE0101960E943A5FBE016F5FD8
:103420007F4F87EC93E10E942E5DFF24F39481117E
:1034300001C0F12CCE0101960E94505E02C0FF2413
:10344000F394C8010E94505ECE0183960E94505EA4
:10345000F11005C027C1CE0183960E94505E8AE01C
:10346000A82EB12CC12CD12C760166246A9493E04D
:10347000792E6EE170E080E090E00E94986E80917D
:1034800010020E944E6EB3010E94FDA8072E000C90
:10349000880B990B0E9438A420E030E040EA50E409
:1034A0000E9497A49B01AC01C701B6010E94C2A56E
:1034B0006B017C01E1E0AE1AB108D9F620E030E002
:1034C00040E251E40E9488A62B013C0163EE78E0C3
:1034D000C8010E943A5FB80187EC93E10E942E5D1B
:1034E00081110C94202467EE78E0CE0101960E94B1
:1034F0003A5FBE016F5F7F4F87EC93E10E942E5DC4
:10350000FF24F394811101C0F12CCE0101960E9499
:10351000505EC8010E94505EFF2009F43FC020E0C9
:1035200030E040E650E4C301B2010E9497A49B0141
:10353000AC0160E070E080E890E40E94C1A5AB01BE
:10354000BC0140930C0250930D0260930E027093E5
:103550000F0222E0CE0101960E94845EBE016F5FE1
:103560007F4F8FEA93E10E94175ECE0101960E9481
:10357000505E6BEE78E0CE0101960E943A5F6FEAF2
:1035800073E1CE0101960E94605DBC018FEA93E178
:103590000E94025ECE0101960E94505E6AEF78E0C2
:1035A000C8010E943A5FB80187EC93E10E942E5D4A
:1035B00081110C9424246FEF78E0CE0101960E94D3
:1035C0003A5FBE016F5F7F4F87EC93E10E942E5DF3
:1035D000FF24F394811101C0F12CCE0101960E94C9
:1035E000505EC8010E94505EFF2009F43FC020E0F9
:1035F00030E040E650E4C301B2010E9497A49B0171
:10360000AC0160E070E080E291E40E94C1A5AB01F2
:10361000BC01409308025093090260930A02709320
:103620000B0222E0CE0101960E94845EBE016F5F14
:103630007F4F8FEA93E10E94175ECE0101960E94B0
:10364000505E64E079E0CE0101960E943A5F6FEA35
:1036500073E1CE0101960E94605DBC018FEA93E1A7
:103660000E94025ECE0101960E94505E61EC7CE0F9
:10367000CE0101960E943A5F6FEA73E1CE01019696
:103680000E94605DBC01C8010E94325FC8010E94B7
:103690004A7FC8010E94505ECE0101960E94505E92
:1036A0000C94B32364E179E0CE0101960E943A5F65
:1036B000BE016F5F7F4F87EC93E10E942E5DF82E75
:1036C000CE0101960E94505EFF2009F46BC08091EC
:1036D000CB139091CC13079710F40C94B32346E0CE
:1036E00050E067EC73E1CE0101960E94394BBE01B8
:1036F0006F5F7F4F89EA93E10E94175ECE010196CA
:103700000E94505E89EA93E10E943E5CAB01BC01DD
:103710004093190250931A0260931B0270931C028B
:1037200021E0C8010E94845E6EE177E0CE0101963F
:103730000E943A5FB801CE0101960E94605D66EE7C
:103740007CE00E94495DBC018FEA93E10E94025E29
:10375000CE0101960E94505EC8010E94505E6FEA41
:1037600073E1CE0101960E94325FCE0101960E9464
:103770004A7FCE0101960E94505E0E94D06E28EED4
:1037800033E040E050E00E9490A5CA01B9010E94D8
:1037900036A46093DF0D7093E00D8093E10D90935C
:1037A000E20DE1C76BE179E0CE0101960E943A5F3C
:1037B000BE016F5F7F4F87EC93E10E942E5DF82E74
:1037C000CE0101960E94505EFF20D1F18091CB1373
:1037D0009091CC13079708F4C6C746E050E067EC19
:1037E00073E1CE0101960E94394BBE016F5F7F4F9E
:1037F00089EA93E10E94175ECE0101960E94505E15
:1038000089EA93E10E943E5CAB01BC014093150242
:1038100050931602609317027093180221E0C801BA
:103820000E94845E6EE277E0CE0101960E943A5FCC
:10383000B801CE0101960E94605D66EE7CE07CC11D
:1038400062E279E0C8010E943A5FB80187EC93E137
:103850000E942E5D811117C068E279E0CE010196C9
:103860000E943A5FBE016F5F7F4F87EC93E10E9439
:103870002E5DFF24F394811101C0F12CCE0101963D
:103880000E94505E02C0FF24F394C8010E94505E63
:10389000FF2009F4BAC08091CB139091CC13079705
:1038A000F8F046E050E067EC73E1CE0101960E942B
:1038B000394BBE016F5F7F4F89EA93E10E94175E2B
:1038C000CE0101960E94505E89EA93E10E943E5C1F
:1038D00060932D0570932E0580932F0590933005EE
:1038E000809106029091070299270E94736ABC0199
:1038F000990F880B990B0E9438A42DE038E643E518
:103900005BE30E9497A46B017C012091F504309148
:10391000F6044091F7045091F8040E9432A418165E
:103920004CF06091DD047091DE048091DF04909191
:10393000E0041BC02091090530910A0540910B0558
:1039400050910C05C701B6010E9477A787FF05C0FB
:10395000C701B6010E946E7808C06091F1047091B1
:10396000F2048091F3049091F40420E030E048ECFC
:1039700052E40E9497A46B017C0120E030E0A90191
:103980000E9432A4181634F0C12CD12CA8EAEA2ED9
:10399000A1E4FA2EC0922D05D0922E05E0922F05BB
:1039A000F0923005C0924E12D0924F12E092501217
:1039B000F09251128091250E882381F060E074E02E
:1039C0008EE990E10E94A75F60912D0570912E0510
:1039D00080912F05909130050E94B18810920615B4
:1039E0001092051580E090E00E943F7940912D05EE
:1039F00050912E0560912F057091300522E0C8018D
:103A00000E94845E6EE279E089C668E379E0C801CD
:103A10000E943A5FB80187EC93E10E942E5D81110C
:103A200017C06CE379E0CE0101960E943A5FBE01B7
:103A30006F5F7F4F87EC93E10E942E5DFF24F3942C
:103A4000811101C0F12CCE0101960E94505E02C08E
:103A5000FF24F394C8010E94505EFF2009F46FC058
:103A60007090040260E0872D0E940F6EF9E1AF2E86
:103A7000B12CC12CD12C7601872D0E944E6EBC0139
:103A8000990F880B990B0E9438A49B01AC01C701C8
:103A9000B6010E94C2A56B017C016AE070E080E083
:103AA00090E00E94986EF1E0AF1AB10829F720E08B
:103AB00030E040EA50E4C701B6010E9497A420E03C
:103AC00030EC4FE754E40E9488A620E030E048EC58
:103AD00051E40E9488A66093290570932A0580937B
:103AE0002B0590932C05609364127093651280935C
:103AF000661290936712109206151092051580E0D9
:103B000090E00E943F794091290550912A056091EB
:103B10002B0570912C0522E0C8010E94845E62EBA7
:103B200076E0CE0101960E943A5FB801CE0101967F
:103B30000E94605D65EC76E00E94495DF8C560E436
:103B400079E0C8010E943A5FB80187EC93E10E94D6
:103B50002E5D811117C066E479E0CE0101960E94C6
:103B60003A5FBE016F5F7F4F87EC93E10E942E5D4D
:103B7000FF24F394811101C0F12CCE0101960E9423
:103B8000505E02C0FF24F394C8010E94505EFF20E3
:103B900009F459C080914912082E000C990B019725
:103BA000039708F049C089E390E00E94736ABC0162
:103BB000990F880B990B0E9438A42AE137E64CE94B
:103BC00050E40E9497A460934A1270934B12809322
:103BD0004C1290934D12109206151092051580E02C
:103BE00090E00E943F796FED73E08FEA93E10E94CD
:103BF000C75D40914A1250914B1260914C127091E6
:103C00004D1222E0CE0101960E94845EBE016F5FDC
:103C10007F4FC8010E94325F6CE479E0C8010E94C6
:103C2000495DBC018FEA93E10E94C15DC8010E9419
:103C3000505ECE01019685C569EB73E08FEA93E192
:103C40000E94C75D80C56FE479E0C8010E943A5FB9
:103C5000B80187EC93E10E942E5D811117C063E5E6
:103C600079E0CE0101960E943A5FBE016F5F7F4FFF
:103C700087EC93E10E942E5DFF24F394811101C033
:103C8000F12CCE0101960E94505E02C0FF24F394F5
:103C9000C8010E94505EFF2009F440C126E030E0D8
:103CA00044E050E067EC73E1CE0101960E944E5F64
:103CB000BE016F5F7F4F89EA93E10E94175ECE01DC
:103CC00001960E94505E89EA93E10E94495C4B0193
:103CD0005C011B0169EA76E0CE0101960E943A5F21
:103CE000BE016F5F7F4F87EC93E10E94B35CAC0134
:103CF0004F5F5F4F67EC73E1C8010E94394BB80119
:103D000089EA93E10E94175EC8010E94505ECE01CD
:103D100001960E94505EF090020289EA93E10E94AF
:103D20003E5C2B013C01640121E0C21AD108809164
:103D3000250E8823B9F065E573E08EE990E10E94D5
:103D4000A75F4AE050E0B4018EE990E10E946F6005
:103D500068E87DE08EE990E10E949860C301B201BD
:103D60000E94B1886F2DC8010E94B67218870F8318
:103D70001D821E82198289E08A8381E08B838C8375
:103D80001C8A1B8ACE0101960E941272CE010196F6
:103D90000E94266FCE0101960E94878AEE80F12C48
:103DA0004BE0E416F1041CF0EAE0EE2EF12C5BE5AA
:103DB0008516910408F44CC076E2A72E7EE0B72E5B
:103DC0003501212C312C2101C12CD12CCE14DF0442
:103DD000B9F06C2DCE0101960E9462709B01AC017E
:103DE000F30161937193819391933F01C201B101FA
:103DF0000E94C2A51B012C01FFEFCF1ADF0AE6CFFC
:103E0000B7010F2C000C880B990B0E9438A49B0162
:103E1000AC01C201B1010E9488A62B013C01C12C5A
:103E2000D12CCE14DF0409F457C0F5012081318173
:103E300042815381C301B2010E94C1A5F501619382
:103E40007193819391935F01FFEFCF1ADF0AE9CF5E
:103E5000121413040CF5E214F30424F4670121E0B6
:103E6000C21AD1086C2DCE0101960E9462709B018E
:103E7000AC01C601880F991F880F991FBC016A5DAC
:103E8000714F6B01C301B2010E94C1A5F6016083AD
:103E900071838283938320C02328F1F436E2A32E1A
:103EA0003EE0B32EC12CD12CCE14DF04A9F06C2D32
:103EB000CE0101960E9462709B01AC01C301B20168
:103EC0000E94C1A5F50161937193819391935F0164
:103ED000FFEFCF1ADF0AE8CFE6E2FEE0A8E6B2E1A4
:103EE00041915191619171914D935D936D937D934A
:103EF0002EE0EE34F207A1F7109206151092051588
:103F000080E090E00E943F7944E050E067EC73E18C
:103F1000C8010E94394B67E579E000C468E779E0A1
:103F2000C8010E943A5FB80187EC93E10E942E5DC0
:103F3000811117C06FE779E0CE0101960E943A5FC8
:103F4000BE016F5F7F4F87EC93E10E942E5DFF24DF
:103F5000F394811101C0F12CCE0101960E94505EB4
:103F600002C0FF24F394C8010E94505EFF2009F4B0
:103F70001AC127E030E046E050E067EC73E1CE0183
:103F800001960E944E5FBE016F5F7F4F89EA93E109
:103F90000E94175ECE0101960E94505E89EA93E16D
:103FA0000E94495C7B016093491287EC93E10E9477
:103FB000545C68E87DE0CE0101960E943A5FBE0144
:103FC0006F5F7F4F87EC93E10E94B35CAC014F5F62
:103FD0005F4F67EC73E1C8010E94394BC8010E9432
:103FE0003E5C60934A1270934B1280934C129093F4
:103FF0004D12C8010E94505ECE0101960E94505E93
:1040000068EA73E08FEA93E10E94C75D44E0E4163A
:10401000F1049CF452E0E516F1040CF059C0E114EF
:10402000F104B9F0EA94EF2809F094C061E576E074
:104030008FEA93E10E94B35D70C074E0E716F1046B
:1040400009F088C066E776E08FEA93E10E94B35DED
:10405000A1C020E030E0A90160914A1270914B129A
:1040600080914C1290914D120E9432A4181664F067
:1040700080E090E0A0E8BFE380934A1290934B1257
:10408000A0934C12B0934D1220914A1230914B12D2
:1040900040914C1250914D1260E070E080EA90E443
:1040A0000E9488A6AB01BC0122E0C8010E94555EB7
:1040B00066E476E0CE0101960E943A5FB801CE0137
:1040C00001960E94605D6AE776E00E94495D56C0F5
:1040D0008AE08E9DB0018F9D700D11244AE0C801C9
:1040E0000E94DF5E6FE576E0CE0101960E943A5FA6
:1040F000B801CE0101960E94605D65E77BE00E94F9
:10410000495DBC018FEA93E10E94C15DCE01019639
:104110000E94505EC8010E94505E20E030E048E4FA
:1041200053E460914A1270914B1280914C1290911D
:104130004D120E9432A418166CF180E090E4ACE1BC
:10414000B5E480934A1290934B12A0934C12B09313
:104150004D1220C060914912062E000C770B4AE0E8
:10416000C8010E94DF5E66E879E0CE0101960E94F8
:104170003A5FB801CE0101960E94605DBC018FEAF2
:1041800093E10E94C15DCE0101960E94505EC8017C
:104190000E94505E109206151092051580E090E086
:1041A0000E943F79D0C26FE879E0C8010E943A5F6F
:1041B000B80187EC93E10E942E5D811117C066E97A
:1041C00079E0CE0101960E943A5FBE016F5F7F4F9A
:1041D00087EC93E10E942E5DFF24F394811101C0CE
:1041E000F12CCE0101960E94505E02C0FF24F39490
:1041F000C8010E94505EFF2009F4C5C027E030E0EE
:1042000046E050E067EC73E1CE0101960E944E5FFC
:10421000BE016F5F7F4F89EA93E10E94175ECE0176
:1042200001960E94505E89EA93E10E94495C609386
:10423000461287EC93E10E94545C89EA93E10E9464
:10424000495C611571058105910519F485E090E0DF
:1042500007C0613071058105910539F489E190E06D
:10426000909348128093471223C068E87DE0CE0106
:1042700001960E943A5FBE016F5F7F4F87EC93E12A
:104280000E94B35CAC014F5F5F4F67EC73E1C80104
:104290000E94394BC8010E94495C70934812609398
:1042A0004712C8010E94505ECE0101960E94505EE6
:1042B000109206151092051580E090E00E943F795B
:1042C00067E973E08FEA93E10E94C75D809146122F
:1042D00083301CF560914712709148124AE0C80182
:1042E0000E94DF5E6DE979E0CE0101960E943A5F9F
:1042F000B801CE0101960E94605D6DE479E00E94F4
:10430000495DBC018FEA93E10E94C15DCE01019637
:104310000E94505EC8010E94505E80914612833018
:104320000CF411C260914712709148124AE0CE011C
:1043300083960E94DF5E60914612062E000C770B7A
:104340004AE0C8010E94DF5E66E879E0CE0101968E
:104350000E943A5FB801CE0101960E94605DBE01E5
:104360006D5D7F4F0E94605DBC018FEA93E10E940A
:10437000C15DCE0101960E94505EC8010E94505E50
:10438000CE018396DEC168EA79E0C8010E943A5FF7
:10439000B80187EC93E10E942E5D811117C06CEA91
:1043A00079E0CE0101960E943A5FBE016F5F7F4FB8
:1043B00087EC93E10E942E5DFF24F394811101C0EC
:1043C000F12CCE0101960E94505E02C0FF24F394AE
:1043D000C8010E94505EFF2009F449C0809100028C
:1043E000909101020E94FA926093A1047093A2043A
:1043F0008093A3049093A4046093321270933312B9
:104400008093341290933512C12C20E5D22E23ECE8
:10441000E22E27E4F22EC092A904D092AA04E092E0
:10442000AB04F092AC04C0922A12D0922B12E0920C
:104430002C12F0922D122091250E21110E94B1888C
:10444000109206151092051580E090E00E943F79C9
:104450004091A1045091A2046091A3047091A4041E
:1044600022E0C8010E94845E60EB79E057C16BEBEB
:1044700079E0C8010E943A5FB80187EC93E10E949D
:104480002E5D811117C06FEB79E0CE0101960E947D
:104490003A5FBE016F5F7F4F87EC93E10E942E5D14
:1044A000FF24F394811101C0F12CCE0101960E94EA
:1044B000505E02C0FF24F394C8010E94505EFF20AA
:1044C00009F477C08091CB139091CC130497F8F046
:1044D00044E050E067EC73E1CE0101960E94394B55
:1044E000BE016F5F7F4F89EA93E10E94175ECE01A4
:1044F00001960E94505E89EA93E10E943E5C6093BF
:10450000AD047093AE048093AF049093B0046091B7
:10451000AD047091AE048091AF049091B0046093AB
:1045200026127093271280932812909329122091BB
:10453000250E222319F042E00E944A768091000263
:10454000909101020E94FA926093A5047093A604D0
:104550008093A7049093A80460932E1270932F1257
:1045600080933012909331128091250E882381F030
:104570006DE873E08EE990E10E94A75F6091A50469
:104580007091A6048091A7049091A8040E94B1881C
:10459000109206151092051580E090E00E943F7978
:1045A0004091A5045091A6046091A7047091A804BD
:1045B000AFC06BEC79E0C8010E943A5FB80187ECAC
:1045C00093E10E942E5D811117C06FEC79E0CE015E
:1045D00001960E943A5FBE016F5F7F4F87EC93E1C7
:1045E0000E942E5DFF24F394811101C0F12CCE01B5
:1045F00001960E94505E02C0FF24F394C8010E94FD
:10460000505EFF2009F4AFC08091CB139091CC1382
:104610000497F8F044E050E067EC73E1CE010196B6
:104620000E94394BBE016F5F7F4F89EA93E10E9480
:10463000175ECE0101960E94505E89EA93E10E94C6
:104640003E5C6093A9047093AA048093AB0490939A
:10465000AC048091A9049091AA04A091AB04B091FC
:10466000AC0480932A1290932B12A0932C12B09337
:104670002D128091250E882389F064E773E08EE97E
:1046800090E10E94A75F6091A9047091AA048091B3
:10469000AB049091AC0442E00E944A768091000203
:1046A000909101020E94FA926093A1047093A20477
:1046B0008093A3049093A4046093321270933312F6
:1046C00080933412909335128091250E882381F0C7
:1046D0006AE673E08EE990E10E94A75F6091A10411
:1046E0007091A2048091A3049091A4040E94B188C7
:1046F000109206151092051580E090E00E943F7917
:104700004091A1045091A2046091A3047091A4046B
:1047100022E0C8010E94845E63EC79E0CE0101963C
:104720000E943A5FB801CE0101960E94605DBC0113
:104730008FEA93E10E94025ECE0101960E94505ED4
:10474000C8010E94505E6FEA73E1CE0101960E949B
:10475000325FCE0101960E944A7FCE0101960E94EF
:10476000505E1092140280911402882371F067EC5D
:1047700073E1CE0101960E94325FCE0101960E9444
:104780006B45CE0101960E94505E0E94D06E6093F0
:10479000E30D7093E40D8093E50D9093E60D6FEBC0
:1047A0007CE087EC93E10E94ED5D52C0CE018396E0
:1047B0000E94DF5E66E879E0CE0145960E943A5F8E
:1047C000BE016D5D7F4FCE0145960E94605D0C94E9
:1047D0003E0B61E070E08BEB93E10E941D5D182FB2
:1047E0008091250E882361F064E477E08EE990E102
:1047F0000E9498606BEB73E18EE990E10E94886003
:1048000010330CF4145E6AE270E0611B710917FD4D
:1048100073954AE0CE0101960E94DF5EBE016F5F94
:104820007F4F8BEB93E10E94175ECE0101960E94B1
:10483000505E8BEB93E10E94495CCB010C94FF0D21
:10484000FF24F3940C94891AFF24F3940C94F11A26
:10485000CA5BDF4F0FB6F894DEBF0FBECDBFDF914E
:10486000CF911F910F91FF90EF90DF90CF90BF906D
:10487000AF909F908F907F906F905F904F903F9000
:104880002F9008952F923F924F925F926F927F9256
:104890008F929F92AF92BF92CF92DF92EF92FF9250
:1048A0000F931F93CF93DF93CDB7DEB7C555D109D3
:1048B0000FB6F894DEBF0FBECDBF8C01C090210EA5
:1048C000D090220E8091250E882349F068ED75E086
:1048D0008EE990E10E94A75FC8010E943C887801A0
:1048E00025E0E20EF11C85E0E816F10408F1809164
:1048F000210E9091220E8017910711F10E94283FFE
:104900000E94EB671093220E0093210E4AE0B8013B
:10491000CE0101960E94DF5EBE016F5F7F4F8BEB81
:1049200093E10E94175ECE0101960E94505E08C07E
:104930000E3F9FEF190721F40E94FB670C94553836
:104940006FEB7CE08FEA93E10E94ED5DA5E0EA1653
:10495000F10490F068E87DE0CE0101960E943A5F94
:104960004AE050E06FEF7FEFCE0101960E940B40CE
:10497000CE0101960E94505EF8017C96E632F10568
:1049800010F00C94A3378827EE58FF4F8F4F0C94EC
:1049900010A90E94283F89E390E00E94617F20E0F7
:1049A00030E04AE754E40E9497A4AB01BC0121E047
:1049B000CE0101960E94845E63ED79E0CE0180967F
:1049C0000E943A5FBE016F5F7F4FCE0180960E94CA
:1049D000605D66ED79E00E94495DBC018FEA93E17C
:1049E0000E94025ECE0180960E94505ECE0101962A
:1049F0000E94505E6AED79E089EA93E10E94ED5DE4
:104A000069EA73E1CE0101960E94325F4AE050E00C
:104A100068E070E0CE0101960E94C540CE0101968B
:104A20000E94505E6FEA73E1CE0101960E94325FF0
:104A30004AE050E06FEF7FEFCE0101960E948C3F7D
:104A4000CE0101960E94505E69EA73E18FEA93E11C
:104A50000E94C15D8091DE0D882311F40C94D4373F
:104A60000C94992FE090CE04F090CF040E94283F40
:104A700089E390E00E94617F0E9421A728EE33E045
:104A8000269FF001279FF00D369FF00D11244AE07C
:104A9000BF01CE0101960E94DF5E63ED79E0CE0199
:104AA00080960E943A5FBE016F5F7F4FCE01809675
:104AB0000E94605D66ED79E00E94495DBC018FEA6D
:104AC00093E10E94025ECE0180960E94505ECE016C
:104AD00001960E94505E8091B3139091B413099790
:104AE00010F022E001C023E0C70164962FAF649765
:104AF0000E94F17FAB01BC0164962FAD6497CE019B
:104B000001960E94845E61E77DE0CE0180960E945E
:104B10003A5FBE016F5F7F4FCE0180960E94605D5D
:104B200065EC76E00E94495DBC018FEA93E10E944A
:104B3000C15DCE0180960E94505ECE0101960E941A
:104B4000505E62EE79E058CF8091DE0D882321F02F
:104B50000E947C640C94D437609115027091160207
:104B600080911702909118020E94D7650C94D43757
:104B7000D09002026FEB7CE0CE01805C9F4F0E94E0
:104B80003A5F7E01B0E2EB0EF11C6D2DC7010E9471
:104B9000B672F886EF821D821E82198289E08A83AE
:104BA00081E08B838C831C8A1B8ACE0101960E9434
:104BB0001272CE0101960E94266FCE0101960E94CC
:104BC000878AEE80F12CE3E0EE16F10409F473C15C
:104BD0006BEE79E0CE01805C9F4F0E94ED5D6FEB44
:104BE0007CE08FEA93E10E94ED5DBE01605C7F4F47
:104BF000CE018E960E94325F4AE050E060E070E0A5
:104C0000CE018E960E94C540CE018E960E94505EC7
:104C100061E080E00E941F766FE07AE0CE01805C68
:104C20009F4F0E94ED5D66E2862E6EE0962EAA24CE
:104C3000A394B12CC12CD12CCE14DF040CF0F1C004
:104C40006C2DCE0101960E946270D4012D913D9190
:104C50004D915D914D010E94C2A52B013C0120E0C8
:104C600030E04CEF52EC0E9432A487FF21C04AE0B2
:104C7000B501CE018E960E94DF5E65E578E0CE013B
:104C8000C4960E943A5FBE01625D7F4FCE01C4961A
:104C90000E94605D65EF79E00E94495DBC018FEA8A
:104CA00093E10E94C15DCE01C4960E94505E45C052
:104CB00022E0B301A201CE018E960E94845E4AE0FA
:104CC000B501CE01C4960E94DF5E65E578E0CE01B5
:104CD000CA960E943A5FBE016C5C7F4FCE01CA96B5
:104CE0000E94605D69EA76E00E94495DBE01625DF6
:104CF0007F4F0E94605DBC0183EA93E10E94025EE7
:104D0000CE01CA960E94505ECE01C4960E94505EAB
:104D1000CE018E960E94505E63EA73E1CE018E96BC
:104D20000E94325F68E87DE0CE018E960E94495D68
:104D3000BC018FEA93E10E94C15DCE018E960E9474
:104D4000505EB1E0EB16F10461F4C114D10409F036
:104D500061C06FEA73E1CE01805C9F4F0E94025EEA
:104D600059C0E2E0EE16F10419F522E0B301A20108
:104D7000CE01C4960E94845EBE016C5C7F4FCE0162
:104D80008E960E94325F68E87DE0CE018E960E948A
:104D9000495DBC01CE01805C9F4F0E94C15DCE0188
:104DA0008E960E94505ECE01C4960E94505E32C024
:104DB000F3E0EF16F10471F163EA73E1CE018E9630
:104DC0000E94325F44E150E06FEF7FEFCE018E969C
:104DD0000E948C3FCE018E960E94505E6DE27DE077
:104DE000CE018E960E943A5FCE018E960E944C3F75
:104DF000CE018E960E94505E80911302882351F05E
:104E000080911202882331F060ED77E080E090E03D
:104E10000E94986E2FEFC21AD20A8FEFA81AB80A12
:104E20000BCFCE01805C9F4F0E94545C8FEA93E1D0
:104E30000E94545CE114F104A9F461E574E08FEA86
:104E400093E10E94C75D61E07AE0CE018E960E94F8
:104E50003A5F4AE050E06FEF7FEFCE018E960E94FE
:104E60008C3FE7C094E0E916F10414F00C94F53798
:104E7000BE01605C7F4FCE018E960E94325F4AE099
:104E800050E06FEF7FEFCE018E960E948C3FCE01F7
:104E90008E960E94505E6DE27DE0CE018E960E945D
:104EA0003A5FCE018E960E944C3FCE018E960E94B4
:104EB000505E0C94F5376CE07AE0CE01805C9F4F39
:104EC0000E94ED5DBE01605C7F4FCE018E960E9418
:104ED000325F4AE050E060E070E0CE018E960E94C2
:104EE000C540CE018E960E94505E6FEB7CE08FEA4B
:104EF00093E10E94ED5D6FEA73E1CE01805C9F4F0C
:104F00000E94025EE12CF12C6E2DCE0101960E94D2
:104F100062704B015C0122E0AB01BC01CE01E114E7
:104F2000F10469F48E960E94845EBE01625D7F4F3B
:104F30008BEB94E10E94995FCE018E961CC0C496C3
:104F40000E94845EBE016C5C7F4FCE018E960E94F3
:104F5000325F68E87DE0CE018E960E94495DBC011B
:104F6000CE01805C9F4F0E94C15DCE018E960E9453
:104F7000505ECE01C4960E94505E22E0B501A401AD
:104F8000CE01C4960E94845EBE016C5C7F4FCE0150
:104F90008E960E94325F68E87DE0CE018E960E9478
:104FA000495DBC018FEA93E10E94C15DCE018E96FE
:104FB0000E94505ECE01C4960E94505EAFEFEA1A86
:104FC000FA0AB3E0EB16F10409F09ECFCE01805C43
:104FD0009F4F0E94545CBE01605C7F4FCE018E9655
:104FE0000E94325F4AE050E06FEF7FEFCE018E9675
:104FF0000E948C3FCE018E960E94505E0E946A3FB6
:105000008FEA93E10E94545C62E17AE0CE018E96D1
:105010000E943A5F6FEA73E1CE018E960E94605D56
:105020006CE17AE00E94495DBC018FEA93E10E9445
:10503000025ECE018E960E94505ECE01805C9F4F34
:105040000C94D23780910402909105020E94459001
:105050000C94D437809106029091070299270E9400
:10506000736ABC01990F880B990B0E9438A42DE03C
:1050700038E643E55BE30E9497A46B017C01209135
:10508000F5043091F6044091F7045091F8040E9421
:1050900032A418164CF06091DD047091DE0480910A
:1050A000DF049091E0041BC02091090530910A05AE
:1050B00040910B0550910C05C701B6010E9477A7DE
:1050C00087FF05C0C701B6010E946E7808C06091D5
:1050D000F1047091F2048091F3049091F40420E0C3
:1050E00030E048EC52E40E9497A420E030E048EA27
:1050F00051E40E9497A420912D0530912E054091F6
:105100002F05509130050E9488A66B017C0164E652
:1051100074E089EA93E10E94C75D69EA73E1CE0118
:1051200001960E94325F42E350E060E070E0CE0101
:1051300001960E94C540CE0101960E94505E22E079
:10514000B701A601CE0101960E94845E65E37AE074
:10515000CE0180960E943A5FBE016F5F7F4FCE0105
:1051600080960E94605D6FE27AE00E94495DBC011A
:105170008FEA93E10E94025ECE0180960E94505E0B
:10518000CE0101960E94505E6FEA73E1CE01019656
:105190000E94325F42E350E06FEF7FEFCE01019655
:1051A0000E948C3FCE0101960E94505E8091DE0DE0
:1051B000882311F40C94D43760E273E080E090E02F
:1051C0000E94986E0C94D4370E94283F68E974E0DE
:1051D0008FEA93E10E94C75D6FEA73E1CE01019609
:1051E0000E94325F4AE050E060E070E0CE0101963C
:1051F0000E94C540CE0101960E94505E6FE874E0A7
:1052000089EA93E10E94C75D69EA73E1CE010196E4
:105210000E94325F44E150E06FEF7FEFCE010196D4
:105220000E948C3FCE0101960E94505E8091230E19
:105230009091240E8430910549F40E94115B8111F4
:105240001AC01092240E1092230E15C0892B99F4C7
:105250000E94115B882339F084E090E09093240E43
:105260008093230E08C00E94115B8111F5CF0E942C
:10527000115B8111F1CF8091230E9091240E049740
:1052800041F163E874E08FEA93E10E94C75D6FEA41
:1052900073E1CE0101960E94325F4AE050E060E087
:1052A00070E0CE0101960E94C540CE0101960E9499
:1052B000505E6FEA73E1CE0101960E94325F68E8AA
:1052C0007DE0CE0101960E94495D69EA73E10C948C
:1052D000E4338AE090E00E9427686B017C0120E0C3
:1052E00030E0A9010E9432A4181634F08AE090E060
:1052F0000E9427686B017C015BE0A52EB12C20E0A9
:1053000030E041EE53E4C701B6010E9432A4181602
:1053100084F420E030E0A901C701B6010E9432A464
:105320001816C4F065E774E08FEA93E10E94C75D48
:1053300042C0E1E0AE1AB10861F368EC70E080E0D1
:1053400090E00E94986E83E090E00E9427686B01D5
:105350007C01D5CF20E030E048EC52E4C701B60133
:105360000E9432A487FF02C021E001C020E0B70103
:10537000A601CE0101960E94845E64E37AE0CE012C
:1053800080960E943A5FBE016F5F7F4FCE0180968C
:105390000E94605D69E37AE00E94495DBC018FEA8A
:1053A00093E10E94025ECE0180960E94505ECE0183
:1053B00001960E94505E6FEA73E1CE0101960E9451
:1053C000325F42E350E06FEF7FEFCE0101960E9423
:1053D0008C3FCE0101960E94505E6CE674E089EA33
:1053E00093E10E94C75D69EA73E1CE0101960E94D4
:1053F000325F42E350E060E070E0CE0101960E942F
:10540000C540D0CE0E94D06E2B013C0181E090E1DE
:105410000E94096D64E670E080E090E00E94986E62
:1054200040E855E260E070E081E090E10E94D24AFD
:1054300064E670E080E090E00E94986E6BEC74E0AF
:1054400089EA93E10E94C75D69EA73E1CE010196A2
:105450000E94325F42E350E06FEF7FEFCE01019692
:105460000E94C540CE0101960E94505E60EC74E03F
:1054700089EA93E10E94C75D69EA73E1CE01019672
:105480000E94325F42E350E06FEF7FEFCE01019662
:105490000E948C3FCE0101960E94505E8091230EA7
:1054A0009091240E8D7F2B961FAE2B97A12CB12CA3
:1054B000C12CD12CE12CF12C019709F475C0CE013F
:1054C000809628969FAF8EAF2897DE015E962A962B
:1054D000BFAFAEAF2A970E94D06EDC01CB0184191A
:1054E0009509A609B709883B9B40A105B10508F0BD
:1054F0005BC081E090E10E94FE6A892B09F44DC0F7
:105500008CED95E0A0E0B0E080930510909306103C
:10551000A0930710B09308100E94057997FD06C06C
:1055200082349105C9F780E090E002C08FEF9FEFD1
:10553000892B99F5DE0111961D014D010E94057917
:1055400097FF06C089818D3441F520E030E00BC023
:10555000D4018D934D012896EEADFFAD2897AE177F
:10556000BF0761F7EFCFD1018D911D01280F311DCC
:105570002A96EEADFFAD2A97AE17BF07A1F72E5BB7
:105580003F4F8E8D90E0982F88274F8D840F911D6F
:105590002817390711F40C94FD3762E370E080E0BE
:1055A00090E00E94986E97CF0E94D06EDC01CB01F4
:1055B00084199509A609B709883B9B40A105B10547
:1055C00028F42B962FAD2B972111C7C00E94283F9E
:1055D00069EA73E1CE0180960E94325F42E350E0B7
:1055E00066E070E0CE0180960E94C540CE018096B4
:1055F0000E94505E2B962FAD2B97222311F40C9412
:10560000183882E090E09093240E8093230E4AE0B5
:10561000B501CE0180960E94DF5E4AE0B601CE0160
:105620008E960E94DF5E4AE0B701CE01CA960E94C4
:10563000DF5EBE01665C7F4FCE01C4960E94325F82
:1056400062E179E0CE01C4960E94495DBE01625DCF
:105650007F4F0E94605D62E179E00E94495DBE017A
:10566000605E7F4F0E94605DBC018FEA93E10E9403
:10567000025ECE01C4960E94505ECE01CA960E9480
:10568000505ECE018E960E94505ECE0180960E94A2
:10569000505E6FEA73E1CE0180960E94325F4AE06D
:1056A00050E06FEF7FEFCE0180960E948C3FCE01DD
:1056B00080960E94505E6DE37AE08BEB94E10E944D
:1056C000986063E47AE08FEA93E10E94ED5D4AE03E
:1056D000B501CE0180960E94DF5E4AE0B601CE01A0
:1056E0008E960E94DF5E4AE0B701CE01CA960E9404
:1056F000DF5EBE01665C7F4FCE01C4960E94325FC2
:1057000068E87DE0CE01C4960E94495DBE01625DFD
:105710007F4F0E94605D68E87DE00E94495DBE01A8
:10572000605E7F4F0E94605D6DE37AE00E94495D9C
:10573000BC018FEA93E10E94C15DCE01C4960E9434
:10574000505ECE01CA960E94505ECE018E960E9497
:10575000505ECE0180960E94505E62E370E080E071
:1057600090E00E94986E81E090E10E94096DF6C67B
:10577000E0900002F090010267ED74E089EA93E1A5
:105780000E94C75D0E94283F69EA73E1CE0101963D
:105790000E94325F4AE050E06FEF7FEFCE0101964A
:1057A0000E94C540CE0101960E94505EC7010E9432
:1057B000FA9262966CAF7DAF8EAF9FAF629780908A
:1057C000A5049090A604A090A704B090A804A501F9
:1057D00094016091A1047091A2048091A30490911E
:1057E000A4040E94C1A52B013C0120E030E0A901E6
:1057F0000E9432A4882309F45BC0C090AD04D0900D
:10580000AE04E090AF04F090B00420E030E0A901D5
:10581000C701B6010E9432A418160CF049C080914D
:10582000A9049091AA04A091AB04B091AC042E9667
:105830008CAF9DAFAEAFBFAF2E979C01AD01C7013E
:10584000B6010E9432A4882399F1A70196012E96F1
:105850006CAD7DAD8EAD9FAD2E970E9488A60E9447
:10586000BDA72E966CAF7DAF8EAF9FAF2E97A501D3
:10587000940162966CAD7DAD8EAD9FAD62970E9436
:10588000C1A5A30192010E9488A62E962CAD3DAD24
:105890004EAD5FAD2E970E9497A40E94F5A69B0186
:1058A000AC01C701B6010E9497A46B017C0103C043
:1058B000C12CD12C760169EA73E1CE0101960E94D8
:1058C000325F4AE050E060E070E0CE0101960E9455
:1058D000C540CE0101960E94505E20E030E64AEEBF
:1058E00056E4C701B6010E9477A718163CF463E599
:1058F0007AE08FEA93E10E94ED5D25C021E0B701D7
:10590000A601CE0180960E94845E62E67AE0CE0116
:1059100001960E943A5FBE01605E7F4FCE01019604
:105920000E94605D66E67AE00E94495DBC018FEAF4
:1059300093E10E94025ECE0101960E94505ECE016C
:1059400080960E94505E6FEA73E1CE0101960E943C
:10595000325F4AE050E06FEF7FEFCE0101960E9488
:105960008C3FCE0101960E94505E64E670E080E0BC
:1059700090E00E94986E1ACCE090CE04F090CF0494
:105980000E94283F65E070E080E090E00E94986E01
:10599000C7010E94F17FAB01BC0123E0CE0101965B
:1059A0000E94845E61E77DE0CE0180960E943A5FAE
:1059B000BE016F5F7F4FCE0180960E94605D65ECF7
:1059C00076E00E94495DBC018FEA93E10E94025E8D
:1059D000CE0180960E94505ECE0101960E94505EDC
:1059E0006AE67AE009C89091100E81E089278093D9
:1059F000100E8091DE0D882331F06FEA73E184E6AA
:105A00009FE00E94886068EC70E080E090E0D8CB76
:105A10001092DE0D1092B2120C94D43781E0809374
:105A2000DE0D8093B2128091A912882349F161EAB8
:105A300078E08BEB93E10E94ED5D86EE9FEF909313
:105A4000220E8093210E2091AC123091AD128091E4
:105A5000AE129091AF128217930724F01092AF12FA
:105A60001092AE121092A0121092A1121092A212D5
:105A70001092A3126CE271E080E090E00E94986EB8
:105A80006BEB73E181EC93E10E94025E8091210E49
:105A90009091220E9093E0148093DF140C94D437ED
:105AA0000E946B410C94D43781E090E10E94096D13
:105AB00040E052EC61E070E081E090E10E94D24A67
:105AC0008CED95E0A0E0B0E0809305109093061077
:105AD000A0930710B093081064E670E080E090E0B7
:105AE0000E94986E62E77AE08FEA93E10E94ED5D92
:105AF0006FEA73E1CE0101960E94325FCE010196FA
:105B00000E946B45CE0101960E94505E62E370E0F8
:105B100080E090E00E94986E6FEA73E1CE010196FA
:105B20000E94325F42E350E06FEF7FEFCE010196BB
:105B30000E94C540CE0101960E94505E6EE77AE059
:105B400089EA93E10E94ED5D69EA73E1CE01019675
:105B50000E94325F44E150E06FEF7FEFCE0101968B
:105B60000E948C3FCE0101960E94505E8091230ED0
:105B70009091240E019739F484E090E00E942092E5
:105B80006B017C0103C0C12CD12C76018091230EC6
:105B90009091240E892B31F481E090E00E942092B4
:105BA0006B017C0120E030E040EA51E4C701B6011E
:105BB0000E9477A7181664F521E0B701A601CE016F
:105BC00001960E94845E6BEF77E0CE0180960E9482
:105BD0003A5FBE016F5F7F4FCE0180960E94605D8D
:105BE0006AE87AE00E94495DBC018FEA93E10E9475
:105BF000025ECE0180960E94505ECE0101960E9408
:105C0000505E81E090E09093240E8093230E10C0AC
:105C10006DE87AE08FEA93E10E94ED5D8091230EBA
:105C20009091240E019721F41092240E1092230ECD
:105C30006FEA73E1CE0101960E94325F4AE050E0C4
:105C400060E070E0CE0101960E94C540CE01019651
:105C50000E94505E6FEA73E1CE0101960E94325FAE
:105C600068E87DE0CE0101960E94495D69EA73E132
:105C70000E94605DBC018FEA93E10E94025ECE014A
:105C800001960E94505E81E090E10E94096D8ECAEB
:105C900060E775E0CE0101960E942A5F4AE050E07D
:105CA0006FEF7FEFCE0101960E948C3FCE010196EF
:105CB0000E94505E6091CC047091CD0480912705C4
:105CC000909128050E94537AB4E18B2E912CA12C3F
:105CD000B12CC12CD12CAFEFCA1ADA0AC501B4011C
:105CE0000E94986E6091CC047091CD04809127053C
:105CF000909128050E94537A7C01B3E0CB16D10421
:105D000034F494E1890E911CA11CB11CE4CFEEE1A6
:105D1000CE16D1041CF4892BA1F703C0009709F01B
:105D20000DC180912705909128058B309105C9F40C
:105D30008091191490911A14A0911B14B0911C1405
:105D40008093DB149093DC14A093DD14B093DE14E5
:105D50008091151490911614A0911714B0911814F5
:105D60001DC08631910521F30C9701F58091CE1469
:105D70009091CF14A091D014B091D1148093DB14E2
:105D80009093DC14A093DD14B093DE148091CA14B8
:105D90009091CB14A091CC14B091CD148093D714D2
:105DA0009093D814A093D914B093DA144091DB14D3
:105DB0005091DC146091DD147091DE1421E0CE016D
:105DC00001960E94845E6FE07AE0CE0180960E9488
:105DD0003A5FBE016F5F7F4FCE0180960E94605D8B
:105DE000BC018FEA93E10E94025ECE0180960E9480
:105DF000505ECE0101960E94505E4091D7145091A2
:105E0000D8146091D9147091DA1421E0CE01019672
:105E10000E94845E69E97AE0CE0180960E943A5F32
:105E2000BE016F5F7F4FCE0180960E94605DBC0116
:105E30008FEA93E10E94C15DCE0180960E94505E80
:105E4000CE0101960E94505E62E37AE08FEA93E110
:105E50000E94B35D6FEB7CE0CE0101960E943A5F39
:105E600044E150E060E070E0CE0101960E94C54040
:105E7000CE0101960E94505EC090DB14D090DC14DD
:105E8000E090DD14F090DE1420E030E0A901C701BD
:105E9000B6010E9477A720E030E040E05FE387FD95
:105EA00005C0C701B6010E94C2A504C0C701B60162
:105EB0000E94C1A50E9421A72AE0AB01BC01CE012E
:105EC00001960E94B35EBE016F5F7F4F89EA93E146
:105ED0000E94175ECE0101960E94505E60E087E04E
:105EE0000E941F7669EA73E18BEB94E10E94995F4F
:105EF0006FED8BEB94E10E94925F6FE97AE08BEBA0
:105F000094E10E9498606091D7147091D8148091A8
:105F1000D9149091DA140E9421A74AE050E08BEB4B
:105F200094E10E946F6062E37AE08BEB94E10E945F
:105F3000986064E670E080E090E042C98F3FFFEF38
:105F40009F07ACF062E675E0CE0101960E942A5FE1
:105F50004AE050E060E070E0CE0101960E94C5404A
:105F6000CE0101960E94505E6FE375E046C0029636
:105F700081F161E375E0CE0101960E942A5F4AE05B
:105F800050E060E070E0CE0101960E94C540CE0175
:105F900001960E94505E62E275E08FEA93E10E94F2
:105FA000C75D4AE0B701CE0101960E94DF5EBE01E7
:105FB0006F5F7F4F8FEA93E10E94C15DCE01019632
:105FC0000E94505E6CE075E08FEA93E10E94715D83
:105FD000EBC761E075E0CE0101960E942A5F4AE0BE
:105FE00050E060E070E0CE0101960E94C540CE0115
:105FF00001960E94505E61EE74E08FEA93E10E9488
:10600000C75DD2C780918E04882309F4CDC76FEB9A
:106010007CE0CE0101960E943A5F4AE050E061E0E8
:1060200070E0CE0101960E94C540CE0101960E940B
:10603000505E0E94283F0E944E8C2B013C010E9422
:10604000298E4B015C016091B9047091BA04809172
:10605000BB049091BC040E9438A49B01AC016496DF
:106060006FAF649763963FAF639765964FAF659741
:1060700066965FAF66970E944E8C0E9438A4649625
:106080002FAD649763963FAD639765964FAD659767
:1060900066965FAD66970E9488A621E03EED42E4D9
:1060A0005EE30E9430A89B01AC0160E070E080E8F4
:1060B0009FE30E94C1A520E03AE24DE257E40E942E
:1060C00097A46B017C01C301B2010E9438A420E0B7
:1060D00030E048EC52E40E9488A6AB01BC0122E00B
:1060E000CE0101960E94845EBE016F5F7F4F83EAFE
:1060F00093E10E94175ECE0101960E94505E6BE80C
:1061000077E083EA93E10E94B35D63EA73E189EA91
:1061100093E10E94025E67E877E0CE0101960E945B
:106120003A5F63EA73E1CE0101960E94605DBC01B3
:1061300083EA93E10E94025ECE0101960E94505EC6
:106140006FE07AE08FEA93E10E94ED5D21E0B50116
:10615000A401CE0101960E94845EBE016F5F7F4F55
:106160008FEA93E10E94C15DCE0101960E94505ECC
:1061700062EA7AE08FEA93E10E94B35D21E0B70121
:10618000A601CE0180960E94845EBE01605E7F4FB4
:10619000CE0101960E94325F66E67DE0CE01019657
:1061A0000E94495DBC018FEA93E10E94C15DCE016E
:1061B00001960E94505ECE0180960E94505E63EA76
:1061C00073E1CE0101960E94325F68E87DE0CE0166
:1061D00001960E94495D6FEA73E10E94605DBC0117
:1061E0008FEA93E10E94025ECE0101960E94505E0A
:1061F00069EA73E1CE0101960E94325F4AE050E005
:1062000060E070E0CE0101960E94C540CE0101968B
:106210000E94505E21E0B501A401CE0101960E94CA
:10622000845EBE016F5F7F4F85EB93E10E94175E36
:10623000CE0101960E94505E65EB73E1CE0101969E
:106240000E94325F4AE050E06FEF7FEFCE0101968F
:106250000E948C3FCE0101960E94505E6FE97AE069
:10626000CE0101960E943A5FCE0101960E944C3FFA
:10627000CE0101960E94505E21E0B701A601CE0139
:1062800080960E94845EBE01605E7F4FCE010196C3
:106290000E94325F66E67DE0CE0101960E94495D74
:1062A000BC0185EB93E10E94025ECE0101960E9443
:1062B000505ECE0180960E94505E65EB73E1CE0188
:1062C00001960E94325F4AE050E068EF7FEFCE0116
:1062D00001960E948C3FCE0101960E94505E8091F3
:1062E000DE0D882309F460C668E572E080E090E086
:1062F0000C94E0288091DE0D81110AC08091A412D7
:10630000811106C0AEE18A2E912CA12CB12C05C0C2
:10631000F3E08F2E912CA12CB12C6EE775E08FEA63
:1063200093E10E94C75D6FEA73E1CE0101960E947E
:10633000325F4AE050E06FEF7FEFCE0101960E949E
:106340008C3FCE0101960E94505E412C512C3201AF
:10635000C12CD12C760183E20E94067687E090E082
:106360000E9401760E94A47566E970E080E090E0EA
:106370000E94986E83E20E94067680E290E00E947E
:1063800001760E94A47566E970E080E090E00E94CA
:10639000986E62E070E083E290E00E94277A40E02D
:1063A00050E0BA018091180F90E02091190F821BE4
:1063B0009109181619062CF58BE391E165964FAFFC
:1063C000659766965FAF669763966FAF63976496BF
:1063D0007FAF64970E94EA7065964FAD65976696A9
:1063E0005FAD669763966FAD639764967FAD649774
:1063F000762F652F542F4427480F511D611D711DA5
:10640000D1CFCB01BA010E9438A42AE939E949E980
:106410005FE30E9488A60E9421A7AB01BC01C416BD
:10642000D506E606F70614F46A017B012AE0CE01E0
:1064300080960E94B35EBE01605E7F4FCE010196E2
:106440000E94325F68EA7AE0CE0101960E94495DBF
:10645000BC0189EA93E10E94025ECE0101960E948E
:10646000505ECE0180960E94505E69EA73E1CE01D3
:1064700001960E94325F4EE150E060E070E0CE0194
:1064800001960E940B40CE0101960E94505E8FEF54
:10649000481A580A680A780A84149504A604B704AE
:1064A0000CF059CF2AE0B701A601CE0180960E94D8
:1064B000B35EBE01605E7F4FCE0101960E94325FE7
:1064C00068EA7AE0CE0101960E94495DBC0189EA42
:1064D00093E10E94025ECE0101960E94505ECE01C1
:1064E00080960E94505E69EA73E1CE0101960E9497
:1064F000325F4AE050E060E070E0CE0101960E9419
:10650000C540CE0101960E94505E2AE0B701A60167
:10651000CE0101960E94B35E6CEA7AE0CE018096CD
:106520000E943A5FBE016F5F7F4FCE0180960E944E
:10653000605D6FEA7AE00E94495D6FEA73E10E9454
:10654000605DBC018FEA93E10E94025ECE018096FD
:106550000E94505ECE0101960E94505E62E370E0A0
:1065600080E090E00C94E028E090CA04F090CB0426
:1065700081E08093DC0464E670E080E090E00E94BB
:10658000986E0E94283FC7010E94736A60E074E021
:10659000681B790B4AE0CE0101960E94DF5E64EB36
:1065A0007AE0CE0180960E943A5FBE016F5F7F4F16
:1065B000CE0180960E94605DBC018FEA93E10E944B
:1065C000025ECE0180960E94505ECE0101960E942E
:1065D000505E60E087E00E941F766EE875E0CE01B5
:1065E00001960E942A5F42E350E068E070E0CE012D
:1065F00001960E94C540CE0101960E94505E6FEA4E
:1066000073E1CE0101960E94325F42E350E06FEFEA
:106610007FEFCE0101960E948C3FCE0101960E9431
:10662000505E6BEB7AE0C8C08091C8049091C904B9
:106630000E94736A7C019093ED0D8093EC0D62E3F0
:1066400070E080E090E00E94986E4AE0B701CE01D1
:1066500001960E94DF5EBE016F5F7F4F8FEA93E17C
:106660000E94175ECE0101960E94505E8091131425
:1066700090911414892B09F45EC06FE074E1CE018F
:1066800080960E94325FBE01605E7F4FCE01019610
:106690000E94325F44E150E060E070E0CE0101967C
:1066A0000E94C540CE0101960E94505E65EC7AE0E2
:1066B000CE0101960E943A5F6FEA73E1CE01019626
:1066C0000E94605DBC0189EA93E10E94025ECE01F6
:1066D00001960E94505E69EA73E1CE0101960E9424
:1066E000325F44E150E06FEF7FEFCE0101960E94F0
:1066F0008C3FCE0101960E94505EBE01605E7F4FCE
:10670000CE0101960E94325F68E87DE0CE010196DD
:106710000E94495D69EA73E10E94605DBC018FEAF5
:1067200093E10E94025ECE0101960E94505ECE016E
:1067300080960C94D42860ED7AE089EA93E10E9477
:10674000ED5D69EA73E1CE0101960E94325F44E19A
:1067500050E060E070E0CE0101960E94C540CE019D
:1067600001960E94505E64EB7AE0CE0101960E9491
:106770003A5F6FEA73E1CE0101960E94605DBC0151
:1067800089EA93E10E94025ECE0101960E94505E6A
:1067900069EA73E1CE0101960E94325F44E150E064
:1067A0006FEF7FEFCE0101960E948C3FCE010196E4
:1067B0000E94505E65EC7AE0CE0101960E943A5F3D
:1067C0006FEA73E1CE0101960E94605DBC018FEA21
:1067D00093E10E94025E0C94D22880918E0488235B
:1067E00009F4E2C38091DE0D811104C08091A412EE
:1067F000882329F082E090E00E949745D5C3C0909D
:106800001502D0901602E0901702F090180220E0D6
:1068100030E040E450E4C701B6010E9477A71816A3
:106820006CF420E030E04AE754E4C701B6010E946E
:1068300097A40E9421A76B017C0106C040E3C42EEF
:1068400045E7D42EE12CF12C0E94283F60E080E047
:106850000E941F7664ED7AE08BEB94E10E949860D1
:1068600061E080E00E941F7665EE7AE08BEB94E1B8
:106870000E94986064E670E080E090E00E94986E6C
:106880000E94D06E6093E80D7093E90D8093EA0D3D
:106890009093EB0D0E94D06E8090E80D9090E90DE2
:1068A000A090EA0DB090EB0DDC01CB01881999099D
:1068B000AA09BB098C159D05AE05BF050CF074C374
:1068C00083E090E00E9497450E94D06E64E170E002
:1068D00080E090E00E94986EDDCF0E94219384E6D4
:1068E0009FE00E94926D60C367E975E089EA93E1D9
:1068F0000E94C75D69EA73E1CE0101960E94325F92
:106900004AE050E060E070E0CE0101960E94C54090
:10691000CE0101960E94505E909110022B969FAF7F
:106920002B978091080E81110DC00E94D06E60934C
:10693000040E7093050E8093060E9093070E81E06F
:106940008093080E8091FC0D81110DC00E94D06EC5
:106950006093F80D7093F90D8093FA0D9093FB0DF1
:1069600081E08093FC0D1092F70D1092F60D2090AF
:10697000F60D3090F70DB8E22B1631040CF086C0FE
:106980002B968FAD2B970E944E6EF101EE0FFF1FDD
:10699000E853F14F918380830E944E7720E030E0EE
:1069A00040EA50E40E9497A420E030E040E85AE337
:1069B0000E9497A46B017C016093F20D7093F30D1C
:1069C0008093F40D9093F50D40900C0250900D02C1
:1069D00060900E0270900F02A30192016091080274
:1069E0007091090280910A0290910B020E94C1A548
:1069F0009B01AC0160E070E080EC90E40E94C1A5D6
:106A00004B015C0120E030E0A9010E9432A420E0AB
:106A100030E040E650E4811105C0C701B6010E9494
:106A200097A41EC0C701B6010E9497A4A3019201BA
:106A30000E94C2A520E030E040E850E40E94C1A5D9
:106A4000A50194010E9488A620E030E040EC50E4CB
:106A50000E9497A420E030E040E850E40E94C2A5E4
:106A60006093EE0D7093EF0D8093F00D9093F10D08
:106A700064E170E080E090E00E94986EAFEF2A1A27
:106A80003A0A3092F70D2092F60D71CFC090EE0DBC
:106A9000D090EF0DE090F00DF090F10D20E030E09F
:106AA000A901C701B6010E9477A787FD1EC022E099
:106AB000B701A601CE0101960E94845E6DEE7AE0D8
:106AC000CE0180960E943A5FBE016F5F7F4FCE017C
:106AD00080960E94605DBC018FEA93E10E94025E95
:106AE000CE0180960E94505E4AC261EF7AE08FEA42
:106AF00093E10E94ED5D47C280918E04882309F4E2
:106B000053C28091DE0D81112BC08091A41281119E
:106B100027C0C0901502D0901602E0901702F090A6
:106B2000180220E030E04AE754E4C701B6010E94B1
:106B300097A40E9421A74B015C0120E030E040EACD
:106B400050E4C701B6010E9497A420E030E040EA7B
:106B500050E40E94C2A50E9421A7A501940108C08B
:106B600021E030E040E050E06AE070E080E090E05A
:106B70000E94B99419C2809190129091911200973D
:106B8000F1F581E090E0909391128093901260E093
:106B90007BE0CE0101960E943A5FCE0101960E94F1
:106BA0006B45CE0101960E94505E69E07BE0CE010C
:106BB00001960E943A5F6FEA74E1CE0101960E944D
:106BC000605DBC01CE0180960E94325F48EC50E0CF
:106BD0006FEF7FEFCE0180960E94C540CE01809678
:106BE0000E94505ECE0101960E94505E84E69FE0B6
:106BF0000E94096D40E052EC61E070E078C00297BD
:106C000099F510929112109290126FE07BE0CE01F4
:106C100001960E943A5FCE0101960E946B45CE011B
:106C200001960E94505E6DE17BE0CE0101960E94CC
:106C30003A5F6FEA74E1CE0101960E94605DBC018B
:106C4000CE0180960E94325F48EC50E06FEF7FEFFC
:106C5000CE0180960E94C540CE0180960E94505E73
:106C6000CE0101960E94505E8091901290919112F7
:106C70000197A9F582E090E0909391128093901291
:106C800061E27BE0CE0101960E943A5FCE0101965F
:106C90000E946B45CE0101960E94505E62E37BE04C
:106CA000CE0101960E943A5F6FEA74E1CE0101962F
:106CB0000E94605DBC01CE0180960E94325F48EC6C
:106CC00050E06FEF7FEFCE0180960E94C540CE016D
:106CD00080960E94505ECE0101960E94505E84E62E
:106CE0009FE00E94096D40E855E260E070E084E6B4
:106CF0009FE00E94D24A109206151092051580E07E
:106D000090E00E943F7967E37BE0CE0101960E940C
:106D10003A5F69EA74E1CE0101960E94605DBC01B0
:106D2000CE0180960E94325F40ED57E06FEF7FEF1B
:106D3000CE0180960E948C3FCE0180960E94505ECC
:106D40002FC168E379E087EC93E10E94ED5D6CE38D
:106D50007BE0CE0101960E943A5F44E650E060E09D
:106D600070E0CE0101960E94C540CE0101960E94BE
:106D7000505E0E94780866E47BE0CE0101960E9496
:106D80003A5F44E650E007C18091250E882309F45C
:106D90000BC165E57BE0CE0101960E943A5FCE0112
:106DA00001960E944A7FFCC08091C60E9091C70E4A
:106DB000892BA1F481E090E09093C70E8093C60EDA
:106DC0008EED93E090930615809305150E946979E6
:106DD00068EC70E080E090E00E94986E6DE57BE0EA
:106DE000CE0101960E943A5F44E650E06FEF7FEFDC
:106DF000CE0101960E948C3FCE0101960E94505E0A
:106E0000E0E0F0E01995D0C00E94D45B0E94283FDA
:106E10000E94EB67C9C09091A91281E089278093F5
:106E2000A912882369F161ED75E08FEA93E10E9470
:106E3000C75D0E94D06E6093A0127093A1128093E0
:106E4000A2129093A3128091AC129091AD121816D9
:106E500019065CF42091AE123091AF122817390751
:106E600024F01092AF121092AE129091B012809155
:106E7000AB1298175CF01092B0121092B11206C0CB
:106E800069EC75E08FEA93E10E94C75D8091A912D9
:106E90008093A4126FEA73E1CE0101960E94325FE3
:106EA0004AE050E068E070E0CE0101960E94C540E3
:106EB000CE0101960E94505E6CEB75E0CE0101960A
:106EC0000E942A5F4AE050E06FEF7FEFCE0101960B
:106ED0000E948C3FCE0101960E94505E6EEA75E0E2
:106EE0008FEA93E10E94715D61EC7CE0CE01019636
:106EF0000E943A5F6FEA73E1CE0101960E94605DE5
:106F0000BC018FEA93E10E94025ECE0101960E94CD
:106F1000505E8091DE0D8093B2128CE291E00E946F
:106F20008F798091DE0D882309F43EC061EA78E014
:106F30008BEB93E10E94ED5D86EE9FEF9093220E26
:106F40008093210E31C0D092220EC092210E60EAB1
:106F500075E08FEA93E10E94C75D84E69FE00E949E
:106F6000926D6FEB7CE0CE0101960E943A5F4AE0A1
:106F700050E060E070E0CE0101960E94C540CE0175
:106F800001960E94505E6FEA73E1CE0101960E9465
:106F9000325F4AE050E06FEF7FEFCE010196BCD741
:106FA000CE0101960E94505E8091B3139091B4136C
:106FB0000097A1F0419720F4023011050CF063C056
:106FC0006FEA73E1CE0101960E94325FCE01019615
:106FD0000E944A7FCE0101960E94505E64E670E0F6
:106FE00080E090E00E94986E60C06CE17AE08FEAE9
:106FF00093E10E94B35D0C941D28EC80F12CFE2CD3
:10700000EE248D81E80EF11CCE80D12CDC2CCC241A
:107010008F81C80ED11CA884B12CBA2CAA248985D2
:10702000A80EB11C21E02B962FAF2B970C94CD2AE4
:1070300065EB74E08FEA93E10E94C75D6FEA73E14C
:10704000CE0180960E94325F4AE050E060E070E03E
:10705000CE01809661D7CE0180960E94505E62EA92
:1070600074E08FEA93E10E94C75D8091230E9091B6
:10707000240E029711F00C94AD2B1092240E109256
:10708000230E0C94AD2B6FEA73E1CE0101960E94A2
:10709000325F4AE050E06FEF7FEFCE0101963CD7C0
:1070A000CE0101960E94505E8BCFCB5ADF4F0FB6B8
:1070B000F894DEBF0FBECDBFDF91CF911F910F912E
:1070C000FF90EF90DF90CF90BF90AF909F908F9008
:1070D0007F906F905F904F903F902F9008952F92E8
:1070E0003F924F925F926F927F928F929F92AF9258
:1070F000BF92CF92DF92EF92FF920F931F93CF93A5
:10710000DF93CDB7DEB728970FB6F894DEBF0FBE7A
:10711000CDBFFC018EE491E19387828780914B1172
:1071200090E0958784878091181290E097878687F2
:1071300080914711853009F0B7C38091501190912B
:107140005111885891098D35910588F480914B1122
:10715000843041F480915211909153118097479758
:1071600008F407C280914B11843408F0E8C1809183
:107170004B118A3108F448C080914E1190914F1103
:10718000843F914050F4118610868FEF9FEFDC0111
:1071900084839583A683B78351C0809150119091C9
:1071A000511185974B9780F514E5E12E11E1F12EF1
:1071B00082E090E040E050E0BA018C010F5F1F4F89
:1071C00020914B1130E0021713076CF49701225005
:1071D0003109D9012D913C912750310927303105D2
:1071E00008F40AC2C8010197959587959187808711
:1071F0000C971CF41186108607C044835583668360
:10720000778384E090E01CC180914B118A3108F4AF
:1072100048C080914E1190914F118032934008F4F4
:10722000B2CF8091501190915111C697869708F472
:1072300003C237C044835583668377838BE090E035
:10724000FFC0D7012D913C91255231092B313105D9
:1072500008F004C2440F551F661F771F4160029655
:10726000B4E0EB0EF11C8C010F5F1F4F20914B110E
:1072700030E00217130764F4970122503109D90155
:107280002D913C912C5031092B303105D0F2C801A1
:10729000019795958795918780870C975CF6118665
:1072A000108680914B11823208F44CC080915011AD
:1072B000909151110697079708F044C044E5C42EF9
:1072C00041E1D42E82E090E040E050E0BA018C0130
:1072D0000F5F1F4F20914B1130E0021713070CF581
:1072E000D6011297ED90FC9011979D01BEE1EB1A2B
:1072F000F108A7E1EA16F10408F0BEC1440F551FDA
:10730000661F771F4160D6012D913C91B4E0CB0EF2
:10731000D11C235031092530310510F40296D7CF06
:10732000C8010197959587959187808740971CF4B0
:107330001186108607C044835583668377838CE06B
:1073400090E07EC07F011C821B8281E090E09A83E6
:10735000898380914B118D3008F475C029E733E0A3
:10736000AE014D5F5F4FBE016F5F7F4FCF010E9447
:10737000D18F892B09F067C029E733E0AE014D5F5B
:107380005F4FBE016F5F7F4FC7010E94D18F019792
:1073900009F059C029E733E0AE014D5F5F4FBE01F0
:1073A0006F5F7F4FC7010E94D18F892B09F04BC0BF
:1073B000812C912C540100E010E080914B1190E061
:1073C00029813A81281739077CF529E733E0AE0196
:1073D0004D5F5F4FBE016F5F7F4FC7010E94D18F2E
:1073E0006C0129E733E0AE014D5F5F4FBE016F5F77
:1073F0007F4FC7010E94D18FE1E0CE16D10449F43E
:10740000892B09F5880C991CAA1CBB1C689480F870
:1074100008C0CD28C1F40197B1F4880C991CAA1CAE
:10742000BB1C0F5F1F4FC9CFD70119961C930E933A
:107430001897F70184829582A682B78281E090E056
:107440009183808329C21C821B8281E090E09A8311
:107450008983D7011C968D919C911D97181619064A
:107460000CF061C01A96ED91FC911B9782E090E0C0
:107470009A8389838281938189974E9708F053C0BC
:1074800083E090E09A838983848195810B970A97A2
:1074900008F049C02CEB31E0AE014D5F5F4FBE01FB
:1074A0006F5F7F4FC7010E94D18F892BE1F52CEBD5
:1074B00031E0AE014D5F5F4FBE016F5F7F4FC7018F
:1074C0000E94D18F019779F5412C512C320100E0B7
:1074D00010E029813A81D7011C968D919C911D97CE
:1074E000281739070CF010C12CEB31E0AE014D5FCD
:1074F0005F4FBE016F5F7F4FC7010E94D18F5C015C
:107500000330110509F0C6C02CEB31E0AE014D5F30
:107510005F4FBE016F5F7F4FC7010E94D18FA816DA
:10752000B90609F4B7C0D7011A96ED91FC911B97E3
:1075300082819381C697869708F4F2C03EC18091FC
:10754000521190915311825491098E9708F00FCEE9
:1075500020E030E0C12CD12C7601A9014C5A5E4EBE
:10756000DA014D915C91495051094930510598F02B
:10757000FECD80915411909155110997099708F00B
:10758000F1CD118610868FEF9FEFDC018483958308
:10759000A683B7838CC1B9016A5A7E4EDB014D9137
:1075A0005C914751510942315105C0F4D701C601E0
:1075B000880F991FAA1FBB1F6C017D016894C0F83A
:1075C0002C5F3F4F2038310541F620E230E0318713
:1075D0002087C482D582E682F78269C1DB014D91A2
:1075E0005C91465051094730510508F0C0CDCC0C94
:1075F000DD1CEE1CFF1CE4CFD7012D913C912351E3
:1076000031092F30310550F4440F551F661F771F85
:1076100041600296B4E0EB0EF11CCFCDD7012D9165
:107620003C912A5031092930310508F0EDCD440F45
:10763000551F661F771FEDCF809152119091531106
:10764000C697869708F02DCE86E5E82E81E1F82EC4
:1076500083E090E040E050E0BA0105CED7012D91E3
:107660003C912C5031092A30310508F01ACE440FD4
:10767000551F661F771FF3CDD9012D913C912C50DA
:1076800031092B30310508F05DCE440F551F661FC0
:10769000771F39CE2CEB31E0AE014D5F5F4FBE015D
:1076A0006F5F7F4FC7010E94D18F6C0103301105BE
:1076B00079F42CEB31E0AE014D5F5F4FBE016F5F9F
:1076C0007F4FC7010E94D18FC816D90609F02BCF72
:1076D000A114B10459F4CA94CD2809F024CF440C64
:1076E000551C661C771C689440F80BC0AA94AB2804
:1076F00009F019CFCD2809F016CF440C551C661C93
:10770000771C0F5F1F4FE5CE19961C930E931897A9
:10771000F701448255826682778282E090E090CEC3
:10772000848195814B97459708F047C0DF011696F5
:107730006F0126ECC20ED11C20E030E040E050E0AA
:1077400060E070E080E090E00D911C91119709508D
:1077500011090830110588F512960D911C911397A7
:10776000015111090D301105D8F401E00E9418A94A
:1077700021601496AC15BD0539F7F70124833583D4
:107780004683578300E20E9433A92283338385E036
:1077900090E09183808380E390E0918780877CC034
:1077A00012960D911C911397045011090530110583
:1077B00020F401E00E9418A9DCCF80914B1189339D
:1077C00040F082819381895791098335910508F4AE
:1077D0007CC180914B11823209F46CC0828193810B
:1077E000895791098335910508F4E6C18281938117
:1077F0008C549109C59708F064C080914B11843076
:1078000031F4848195818097479708F434C2809140
:107810004B11843408F455C08481958189549109B1
:10782000C39708F04EC09F012A5F3F4FAF014A57F0
:107830005F4F812C912C5401D9016D917C9169503D
:10784000710969307105E8F5D90112966D917C9145
:107850001397665171096131710508F022C2D50193
:10786000C401880F991FAA1FBB1F4C015D016894BA
:1078700080F82C5F3F4F24173507F1F620E230E007
:10788000F70131872087D70184829582A682B7824B
:1078900087E090E08D939C9381E090E0BFC282E00E
:1078A0008093471110924B1180E090E0B7C283E0C3
:1078B00090E0C6CD828193810A97099708F460C150
:1078C0008DCF80914B11863460F1828193810C972A
:1078D0000B9708F4F6C125C0D90112966D917C91E1
:1078E00013976E5171096731710508F01EC2D501F9
:1078F000C401880F991FAA1FBB1F4C015D0168942A
:1079000080F84E5F5F4F2C5F3F4F4534510509F4BF
:10791000F3C1D9016D917C916C5071096B30710587
:10792000D8F280914B11883578F182819381855806
:1079300091098B35910508F408C226C0BC016F5F20
:107940007F4FD8012D913C912750310927303105C7
:1079500008F00AC2440F551F416002960C5F1F4F8A
:1079600020914B1130E024503109821793070CF01D
:1079700004C2980122503109D9012D913C9129501E
:10798000310928303105D0F280914B118032E1F479
:107990008281938106970697B8F48481958109972F
:1079A000099790F49F012A5F3F4FAF01425C5F4F00
:1079B000812C912C5401D9016D917C9166507109F3
:1079C0006630710508F4F3C1D7011C962D903C90E8
:1079D0001D97B6E02B1631040CF461CF8F010A5FBE
:1079E0001F4F73E0C72ED12CE5EC8E2EEDE99E2EB5
:1079F000ECE1AE2EE1E8BE2EF80160817181349792
:107A00006080718080E090E00E9436A46D837E8368
:107A10008F839887B30180E090E00E9436A42B0109
:107A20003C012DEC3CEC4CE45FE30E9497A49B01ED
:107A3000AC016D817E818F8198850E9432A487FD83
:107A400019C02DEC3CEC4CE45FE36D817E818F81AD
:107A500098850E9497A49B01AC01C301B2010E94CA
:107A600032A4E82F880FFF0BEE27FF0FEE1FFF2732
:107A7000319602C0E0E0F0E0A501940163E971E015
:107A800080E091E00E94DAA84F01FF0FAA08BB082E
:107A900086269726A826B926FFEFCF1ADF0A0E5FA3
:107AA0001F4FC214D30409F0A7CFD70114968D92AB
:107AB0009D92AD92BC92179780E290E019969C93AC
:107AC0008E9318978FEF9FEFE5CE84819581CA97AB
:107AD000899708F07ECE9F012A5F3F4F812C912C21
:107AE000540143E050E0D9016D917C916A507109D5
:107AF0006930710508F06DCED90112966D917C91B7
:107B00001397665171096131710550F5D501C401B2
:107B1000880F991FAA1FBB1F4C015D01689480F854
:107B20004E5F5F4F2C5F3F4F4B335105E1F69F0196
:107B30002A583F4FD9012D913C912A5031092930C3
:107B4000310508F046CE2CE130E0F701318720877F
:107B5000D70184829582A682B7828AE090E09ACE8D
:107B6000D90112966D917C91139766507109673017
:107B7000710508F02ECE880C991CAA1CBB1CD0CF16
:107B800020914B11CF01820F911D820F911DDC01BD
:107B900012978D919C910A97099708F01FCEF701D3
:107BA000118610868FEF9FEFDC0184839583A68377
:107BB000B78386E090E044CC80914B11813208F489
:107BC00015CE84819581CA97899708F00FCE9F01C1
:107BD0002A5F3F4F812C912C540143E050E0D901A2
:107BE0006D917C916A5071096930710508F0FECD84
:107BF000D90112966D917C9113976651710961318B
:107C0000710570F112966D917C9113976650710910
:107C10006730710508F0EACD880C991CAA1CBB1CC2
:107C20004E5F5F4F2C5F3F4F43325105C1F69F01BE
:107C30002A5B3F4FD9012D913C912A5031092930BF
:107C4000310508F0D3CD20E130E0F70131872087FE
:107C5000D70184829582A682B78286E090E01ACE10
:107C6000D501C401880F991FAA1FBB1F4C015D01DC
:107C7000689480F8D5CF868197810997099708F095
:107C8000C6CDD70119961C921E9218978FEF9FEFC1
:107C9000DC01F70184839583A683B78387E090E0B6
:107CA000CFCBD90112966D917C91139766507109D3
:107CB0006730710508F005CE880C991CAA1CBB1C06
:107CC000D8CD848195810997099708F02ACE8681BD
:107CD00097818C974F9708F024CE8085918589975E
:107CE0004D9708F01ECE9F01265F3F4F812C912CAF
:107CF000540145E050E00DCE9F0126573F4FD9017A
:107D00002D913C912C5031092B30310508F009CED2
:107D100020E230E0F70131872087D7018482958205
:107D2000A682B78288E090E0B5CDD90112966D9118
:107D30007C911397695071096930710508F0F1CD94
:107D4000880C991CAA1CBB1CDCCD848195818254B3
:107D500091098E9708F018CE8F01045C1F4F8DE1BA
:107D600090E040E050E0FCCDD8012D913C912851AD
:107D7000310922313105C0F0CB01019795958795E6
:107D8000D70119969C938E9318978A970CF4FCCD83
:107D9000052E000C660B770BF70144835583668331
:107DA000778389E090E04CCB440F551FD6CDD901A5
:107DB00012966D917C911397695171096331710528
:107DC000E8F4D501C401880F991FAA1FBB1F4C01FD
:107DD0005D01689480F82C5F3F4F2417350709F048
:107DE000EACD2EE030E0F70131872087D701848289
:107DF0009582A682B7828FE090E04CCDD901129691
:107E00006D917C911397695071096930710508F083
:107E1000DBCD880C991CAA1CBB1CDDCF28960FB6A5
:107E2000F894DEBF0FBECDBFDF91CF911F910F91B0
:107E3000FF90EF90DF90CF90BF90AF909F908F908A
:107E40007F906F905F904F903F902F90089508958E
:107E5000809113028823F9F0809112028823D9F0CF
:107E600081E00E9410768BE39FE10197F1F760E0DB
:107E700080E00E941F7667EE76E08BEB94E10E9433
:107E8000A75F61E080E00E941F7667ED76E08BEBF4
:107E900094E10C94A75F0895CF93DF932091130290
:107EA0002223A9F020911202222389F0EC016FED28
:107EB0008BEB94E10E94925F8C819D81892B39F03C
:107EC000BE018BEB94E1DF91CF910C94995FDF9130
:107ED000CF91089580911302882379F08091120246
:107EE000882359F06FED8BEB94E10E94925F6DE275
:107EF0007DE08BEB94E10C949860089580911302DF
:107F0000882349F080911202882329F060E08BEBEE
:107F100094E10C94127308958F929F92AF92BF9246
:107F2000EF92FF920F931F93CF93DF937C01EB01AE
:107F30008A0180911302882309F462C080911202A1
:107F4000882309F45DC077FF18C0C095D09561E023
:107F50008C2F0E941F76B7018BEB94E10E94995FF2
:107F600066EC76E08BEB94E10E94A75FF7018481D9
:107F700061E08C0F0E941F7633C00E94D06E80900B
:107F8000011590900215A0900315B090041524E6F9
:107F9000820E911CA11CB11C86169706A806B90674
:107FA00078F561E08C2F0E941F76B7018BEB94E18E
:107FB0000E94995F65EB76E08BEB94E10E94A75FEE
:107FC000F701848161E08C0F0E941F760E94D06EC1
:107FD0006093011570930215809303159093041517
:107FE000B801110F880B990BDF91CF911F910F9161
:107FF000FF90EF90BF90AF909F908F900C94986EF1
:10800000DF91CF911F910F91FF90EF90BF90AF90B4
:108010009F908F900895AF92BF92CF92DF92EF9290
:10802000FF920F931F93CF93DF93CDB7DEB7629785
:108030000FB6F894DEBF0FBECDBF209113022223EE
:1080400009F492C020911202222309F48DC06A0122
:108050007B015C010E94D06E00911D0E10911E0EDE
:1080600020911F0E3091200E0C591F4F2F4F3F4F64
:10807000061717072807390708F076C0F7FE08C06B
:1080800087010095109560E0802F0E941F764BC0FD
:1080900060E080E00E941F760E94D06E28EE33E000
:1080A00040E050E00E9464A5CA01B90120E831E532
:1080B00041E050E00E9464A5AB01BC012AE0CE0182
:1080C00001960E94B35EBE016F5F7F4FCE0107969F
:1080D0000E94325F63ED76E0CE0107960E94495D13
:1080E000BC01CE010D960E94325FCE0107960E9420
:1080F000505ECE0101960E94505EBE01635F7F4FCD
:108100008BEB94E10E94995F09891A89E114F104CB
:1081100031F00E0D1F1D60E0802F0E941F76CE01F2
:108120000D960E94505EB5018BEB94E10E94995F21
:1081300064EA76E08BEB94E10E94A75FF50184810D
:1081400060E0800F0E941F760E94D06E60931D0E2B
:1081500070931E0E80931F0E9093200EB601DD0CBF
:10816000880B990B0E94986E62960FB6F894DEBF4A
:108170000FBECDBFDF91CF911F910F91FF90EF9078
:10818000DF90CF90BF90AF900895BF92CF92DF92D3
:10819000EF92FF920F931F93CF93DF93CDB7DEB78C
:1081A00062970FB6F894DEBF0FBECDBF6C018B0196
:1081B0007A0180911302882309F47DC08091120214
:1081C000882309F478C077FF07C00095109560E018
:1081D000802F0E941F764EC060E080E00E941F76D4
:1081E0000E94D06E28EE33E040E050E00E9464A58B
:1081F000CA01B90120E831E541E050E00E9464A5E0
:10820000AB01BC012AE0CE0101960E94B35EBE0123
:108210006F5F7F4FCE0107960E94325F63ED76E07D
:10822000CE0107960E94495DBC01CE010D960E94C9
:10823000325FCE0107960E94505ECE0101960E94E9
:10824000505EBE01635F7F4F8BEB94E10E94995FAC
:10825000B98860E08B2D0E941F760115110511F47D
:108260000B2D04C060E0802F0E941F76CE010D967A
:108270000E94505EB6018BEB94E10E94995F63E926
:1082800076E08BEB94E10E94A75FF601848160E0C9
:10829000800F0E941F760E94D06E60931D0E709317
:1082A0001E0E80931F0E9093200EB701FF0C880BBB
:1082B000990B0E94986E62960FB6F894DEBF0FBEBF
:1082C000CDBFDF91CF911F910F91FF90EF90DF9085
:1082D000CF90BF9008952F923F924F925F926F92EE
:1082E0007F928F929F92AF92BF92CF92DF92EF9246
:1082F000FF920F931F93CF93DF93CDB7DEB7E49731
:108300000FB6F894DEBF0FBECDBF8091E70D882376
:1083100019F01092E70DC6C381E08093E70D7E014E
:108320008FE1E80EF11C6FEB7CE0C7010E943A5F21
:10833000212C312C82E08BA71E2D0F2D88EE882E4C
:1083400083E0982EA12CB12C90E8492E91E5592E6E
:1083500066246394712CF1013197EE30F10530F40D
:108360008827E856FF4F8F4F0C9410A980919012E8
:1083700090919112892B01F56DE17BE0CE01019680
:108380000E943A5F6FEA74E1CE0101960E94605D3F
:10839000BC01CE0107960E94325F48EC50E06FEFBF
:1083A0007FEFCE010796F1DECE0107960E94505E68
:1083B000CE0101960E94505E809190129091911290
:1083C000019701F569E07BE0CE0101960E943A5FDA
:1083D0006FEA74E1CE0101960E94605DBC01CE019E
:1083E00007960E94325F48EC50E06FEF7FEFCE01BE
:1083F0000796CBDECE0107960E94505ECE01019615
:108400000E94505E8091901290919112029701F516
:1084100062E37BE0CE0101960E943A5F6FEA74E16D
:10842000CE0101960E94605DBC01CE0107960E94BC
:10843000325F48EC50E06FEF7FEFCE010796A5DE8C
:10844000CE0107960E94505ECE0101960E94505EBA
:1084500067E37BE0CE0101960E943A5F69EA74E12E
:10846000CE0101960E94605DBC01CE0107960E947C
:10847000325F40ED57E06FEF7FEFCE0107964CDDA6
:10848000CE0107960E94505ECE0101960E94505E7A
:1084900080919012909191120197E1F5CE01019691
:1084A0000E942B638D819E81009781F1E981FA8181
:1084B0002081222359F1079748F164E878E0CE0142
:1084C00007960E942A5F48EC50E06FEF7FEFCE01E5
:1084D0000796A1DDCE0107960E94505EBE016F5F38
:1084E0007F4FCE0107960E94325F48EC50E06FEF5D
:1084F0007FEFCE01079610DDCE0107960E94505EF9
:1085000060ED77E080E090E00E94986ECE010196E9
:108510000E94505E64E670E080E090E00E94986EF9
:1085200082E08093471110924B11A3C268E778E074
:10853000CE0101960E942A5F48EC50E06FEF7FEF7A
:10854000CE01019668DDCE0101960E94505E0E9428
:10855000D06E6B017C010E94D06EA50194010E9437
:1085600090A5CA01B901A30192010E9490A520E142
:108570003EE040E050E00E9464A52CA73DA74EA736
:108580005FA72CE330E040E050E00E9464A528ABF8
:1085900039AB4AAB5BABAB01BC012AE0CE01019623
:1085A0000E94B35E2AE048A959A96AA97BA9CE0115
:1085B00007960E94B35E2AE04CA55DA56EA57FA537
:1085C000CE010D960E94B35EC701B601A5019401CC
:1085D0000E9490A5CA01B901A30192010E9490A531
:1085E000BA01A9012AE0CE0149960E94B35EBE01FC
:1085F000675E7F4FCE0143960E94325F6AE67BE062
:10860000CE0143960E94495DBE01635F7F4F0E9489
:10861000605D6DE67BE00E94495DBE01695F7F4F52
:108620000E94605D60E77BE00E94495DBE016F5F74
:108630007F4F0E94605D66EE7CE00E94495DBC0158
:10864000CE0185960E94325FCE0143960E94505E15
:10865000CE0149960E94505ECE010D960E94505E5A
:10866000CE0107960E94505ECE0101960E94505E98
:1086700040ED57E06FEF7FEFCE0185964DDCCE01E8
:108680008596F5C18091230E9091240E019719F4DF
:1086900069E678E002C06BE578E0CE0101960E94C1
:1086A0002A5F48EC50E06FEF7FEFCE010196B3DC1C
:1086B000CE0101960E94505E6BE478E0CBC16BE383
:1086C00078E0CE0101960E942A5F48EC50E06FEFFF
:1086D0007FEFCE0101969FDCCE0101960E94505E95
:1086E0006EE278E0B7C161E278E0CE0101960E94C7
:1086F0002A5F48EC50E06FEF7FEFCE0101968BDCF4
:10870000CE0101960E94505E66E178E0A3C16AE066
:1087100078E0CE0101960E942A5F48EC50E06FEFAE
:108720007FEFCE01019677DCCE0101960E94505E6C
:1087300069EF77E08FC18091230E9091240E03970B
:1087400019F46EEE77E002C064EE77E0CE01019698
:108750000E942A5F48EC50E06FEF7FEFCE01019658
:108760005ADCCE0101960E94505E69ED77E072C13D
:108770006CEC77E0CE0101960E942A5F48EC50E055
:108780006FEF7FEFCE01019646DCCE0101960E948D
:10879000505E6DEB77E05EC162EB77E0CE01019653
:1087A0000E942A5F48EC50E06FEF7FEFCE01019608
:1087B00032DCCE0101960E94505E65EA77E04AC144
:1087C0008091230E9091240E029719F464E977E0CA
:1087D00002C064E877E0CE0101960E942A5F48EC6F
:1087E00050E06FEF7FEFCE01019615DCCE010196D0
:1087F0000E94505E67E777E02DC16BE677E0CE011F
:1088000001960E942A5F48EC50E06FEF7FEFCE01A7
:10881000019601DCCE0101960E94505E6BE577E087
:1088200019C160E577E0CE0101960E942A5F48EC0D
:1088300050E06FEF7FEFCE010196EDDBCE010196A8
:108840000E94505E66E477E005C16AE377E0CE01FE
:1088500001960E942A5F48EC50E06FEF7FEFCE0157
:108860000196D9DBCE0101960E94505E6AE277E064
:10887000F1C0209149126FE177E0812F902F2CAB4E
:108880000E94C75D2CA924306CF422300CF045C046
:10889000222381F0213009F061C063E77BE0812F62
:1088A000902F59C0243009F059C069E77BE08FEA66
:1088B00093E151C0C0904A12D0904B12E0904C12FC
:1088C000F0904D1220E030E048E452E4C701B601D8
:1088D0000E9432A487FF02C081E08BA7A701960106
:1088E00060E070E080EA90E40E9488A6AB01BC01E1
:1088F0002BA5CE0107960E94555E6EEA7BE0CE0165
:1089000001960E943A5FBE01695F7F4FCE010196DA
:108910000E94605D6AE776E018C08AE02802B00134
:1089200011244AE0CE0107960E94DF5E67E77BE0F4
:10893000CE0101960E943A5FBE01695F7F4FCE0172
:1089400001960E94605D65E77BE00E94495DBC0185
:10895000812F902F1DC00E94B35D24C060914912E9
:10896000062E000C770B4AE0CE0107960E94DF5ED0
:1089700069E376E0CE0101960E943A5FBE01695F2D
:108980007F4FCE0101960E94605DBC018FEA93E1AA
:108990000E94C15DCE0101960E94505ECE010796F5
:1089A0000E94505E612F702FCE0101960E94325FAF
:1089B00048EC50E06FEF7FEFCE0101962CDBCE014B
:1089C00001960E94505E64E177E0812F902F0E9413
:1089D000C75D60914712709148124AE0CE01079638
:1089E0000E94DF5E67E77BE0CE0101960E943A5F5E
:1089F000BE01695F7F4FCE0101960E94605D6DE40C
:108A000079E00E94495DBC01812F902F0E94C15DD9
:108A1000CE0101960E94505ECE0107960E94505EE4
:108A2000612F702FCE0101960E94325F17C064E063
:108A300077E0CE0101960E942A5F48EC50E06FEF8C
:108A40007FEFCE010196E7DACE0101960E94505EDB
:108A500067EF76E0CE0101960E942A5F40ED57E075
:108A60006FEF7FEFCE01019657DACE0101960E949B
:108A7000505E0E94888E882319F01092E70D0EC078
:108A80000E9489818091E70D882341F08FEF281A99
:108A9000380A8FE02816310409F05DCCCE014F96DC
:108AA0000E94505EE4960FB6F894DEBF0FBECDBFB5
:108AB000DF91CF911F910F91FF90EF90DF90CF90BA
:108AC000BF90AF909F908F907F906F905F904F90EE
:108AD0003F902F9008950F931F93CF93DF9300D073
:108AE00000D0CDB7DEB72091250E2223A9F08C014E
:108AF00061EC7CE0CE0101960E943A5FB801CE01A4
:108B000001960E94605DBC018EE990E10E94886040
:108B1000CE0101960E94505E26960FB6F894DEBFF5
:108B20000FBECDBFDF91CF911F910F9108954F924E
:108B30005F926F927F928F929F92AF92BF92CF92ED
:108B4000DF92EF92FF920F931F93CF93DF93CDB7F6
:108B5000DEB7CA54D1090FB6F894DEBF0FBECDBF41
:108B60008C016FEB7CE0CE018B960E943A5F6FEB3D
:108B70007CE0CE0185960E943A5FBE016F5F7F4F19
:108B800084EE93E10E94DE6B8D889E88AF88B88C5E
:108B9000498C5A8C6B8C7C8C8D8D9E8DAF8DB8A141
:108BA00027968CAF9DAFAEAFBFAF2797C801019797
:108BB000039708F0D4C1A3019201C501B4019058F4
:108BC0000E9435A62BED3FE049EC5FE30E94C2A571
:108BD0002091B5043091B6044091B7045091B80487
:108BE0000E94C2A56B017C0120E030E0A9010E9437
:108BF00032A487FD09C0C092190ED0921A0EE092DD
:108C00001B0EF0921C0E10C02BED3FE049EC50E41F
:108C1000C701B6010E94C2A56093190E70931A0E87
:108C200080931B0E90931C0EC090190ED0901A0EBC
:108C3000E0901B0EF0901C0E2BED3FE049EC50E451
:108C4000C701B6010E9477A7181684F42BED3FE008
:108C500049EC50E4C701B6010E94C1A56093190E0A
:108C600070931A0E80931B0E90931C0E20E030E040
:108C700044E353E46091190E70911A0E80911B0E1B
:108C800090911C0E0E9497A42BED3FE049E450E424
:108C90000E9488A66093150E7093160E8093170E8F
:108CA0009093180E0E9421A74AE0CE01C7960E9419
:108CB000DF5E61E87BE0CE01C1960E943A5FBE01B3
:108CC000695C7F4FCE01C1960E94605D6BE87BE0DE
:108CD0000E94495DBC0185EB93E10E94025ECE01DA
:108CE000C1960E94505ECE01C7960E94505EC09011
:108CF000150ED090160EE090170EF090180E20E092
:108D000030E044EB52E4C701B6010E9432A41816C9
:108D100094F020E030E040E05FE3C701B6010E943C
:108D2000C2A50E9421A74AE0CE01C7960E94DF5E3D
:108D300062E97BE023C020E030E044E353E4C70174
:108D4000B6010E9432A41816A4F1A701960160E0B2
:108D500070E884E393E40E94C1A56093150E7093BC
:108D6000160E8093170E9093180E0E9421A74AE0CA
:108D7000CE01C7960E94DF5E65E97BE0CE01C19619
:108D80000E943A5FBE01695C7F4FCE01C1960E948E
:108D9000605DBC01CE018B960E94025ECE01C19641
:108DA0000E94505ECE01C7960E94505E60E37BE059
:108DB00063C020E030E047E853E4C701B6010E94F9
:108DC00032A4181604F120E030E044E353E4C70174
:108DD000B6010E94C1A520E030E040E05FE30E94C0
:108DE000C2A56093150E7093160E8093170E909384
:108DF000180E0E9421A74AE0CE01C7960E94DF5EAE
:108E000065E97BE01FC0A701960160E070E084EB9C
:108E100093E40E94C1A520E030E040E05FE30E94BF
:108E2000C2A56093150E7093160E8093170E909343
:108E3000180E0E9421A74AE0CE01C7960E94DF5E6D
:108E400062E97BE0CE01C1960E943A5FBE01695C97
:108E50007F4FCE01C1960E94605DBC01CE018B9612
:108E60000E94025ECE01C1960E94505ECE01C7965E
:108E70000E94505E68E97BE0CE0185960E94ED5D20
:108E8000BE01655D7F4FCE01C1960E94325F4AE010
:108E900050E060E070E0CE01C19677D9CE01C19676
:108EA0000E94505E0E94D06E20911D0E30911E0EC9
:108EB00040911F0E5091200E69017A01A4E6CA0E5E
:108EC000D11CE11CF11CC616D706E806F90608F409
:108ED00036C228962FAF289729963FAF29972A9612
:108EE0004FAF2A972B965FAF2B970E94D06E0E94B0
:108EF00036A46B017C0128962FAD289729963FADAB
:108F000029972A964FAD2A972B965FAD2B97CA01CA
:108F1000B9010E9438A420E030E048EC51E40E94FE
:108F2000C2A59B01AC01C701B6010E9432A487FD16
:108F300006C268E87DE0CE01C1960E943A5FBE019C
:108F40006B5D7F4FCE01C1960E94605DBC01CE017A
:108F50008B960E94C15DCE01C1960E94505EC801F1
:108F60000297029708F0C5C120E030E040E251E4EA
:108F7000C501B4010E9497A46B017C0120E030E0A0
:108F800040E251E4C301B2010E9497A44B015C018D
:108F900020E030E040E251E427966CAD7DAD8EAD2F
:108FA0009FAD27970E9497A42B013C010E94D06E91
:108FB0002091E80D3091E90D4091EA0D5091EB0DB3
:108FC000621B730B840B950B0E9436A420E030E0EB
:108FD0004AE754E40E9488A6AB01BC0123E0CE011D
:108FE000C7960E94845E6EEA7BE0CE01C1960E9425
:108FF0003A5FBE01695C7F4FCE01C1960E94605D01
:1090000063ED76E00E94495DBC0183EA93E10E9432
:10901000025ECE01C1960E94505ECE01C7960E94AC
:10902000505E63EA73E1CE01C1960E94325F65EB48
:1090300073E1CE01C1960E94605DBE01655D7F4F08
:109040000E94605DBC01CE018B960E94025ECE0143
:10905000C1960E94505E6AE97BE08FEA93E10E942C
:10906000ED5D21E0B701A601CE01C1960E94845EAC
:10907000BE016F5C7F4F8FEA93E10E94C15DCE011C
:10908000C1960E94505E21E0B301A201CE01CD96AF
:109090000E94845E21E0B501A401CE01C7960E9422
:1090A000845E68E87DE0CE01C1960E943A5FBE0111
:1090B000695C7F4FCE01C1960E94605D68E87DE0EB
:1090C0000E94495DBE01635C7F4F0E94605D65EA5E
:1090D0007BE00E94495DBC018FEA93E10E94C15D83
:1090E000CE01C1960E94505ECE01C7960E94505E8E
:1090F000CE01CD960E94505EA7019601C701B60130
:109100000E9497A46B017C01A5019401C501B401E3
:109110000E9497A49B01AC01C701B6010E94C2A5A1
:109120006B017C01A3019201C301B2010E9497A4CB
:109130009B01AC01C701B6010E94C2A50E9480A894
:109140006B017C016093110E7093120E8093130ECD
:109150009093140E69EA7BE08FEA93E10E94B35D7D
:1091600021E0B701A601CE01C1960E94845EBE0136
:109170006F5C7F4FCE01C7960E94325F6AEB7BE047
:10918000CE01C7960E94495DBC0185EB93E10E9428
:10919000025ECE01C7960E94505ECE01C1960E942B
:1091A000505E65EB73E18FEA93E10E94C15DC09070
:1091B000110ED090120EE090130EF090140E20E0DD
:1091C00030E04AE754E4C701B6010E9477A787FD63
:1091D00029C020E030E04AE754E4C701B6010E940C
:1091E00088A6AB01BC0123E0CE01C1960E94555E6A
:1091F000BE016F5C7F4FCE01C7960E94325F6BEB62
:109200007BE0CE01C7960E94495DBC0185EB93E1EE
:109210000E94025ECE01C7960E94505ECE01C196AA
:109220000E94505E20E030E64AE656E46091110E5E
:109230007091120E8091130E9091140E0E9432A420
:10924000BE01655D7F4F87FF50C0CE01C1960E9471
:10925000325F6DEA7BE0CE01C1960E94495D6FEA04
:1092600073E10E94605DBC018FEA93E10E94025E9F
:10927000CE01C1960E94505E03301105A1F46FEA41
:1092800073E1CE01C1960E94325FCE01C1960E9469
:109290004A7FCE01C1960E94505E6FEB7CE08FEA60
:1092A00093E10E94ED5D60EB7BE0CE01C1960E94F0
:1092B0003A5F65EB73E1CE01C1960E94605DBC012F
:1092C000CE01C7960E94325F4AE050E06FEF7FEF19
:1092D000CE01C7960E948C3FCE01C7960E94505E79
:1092E000CE01C1960E94505E04C08FEA93E10E94B5
:1092F000025E6AE070E080E090E00E94986ECE012D
:1093000085960E94505ECE018B960E94505EC65B91
:10931000DF4F0FB6F894DEBF0FBECDBFDF91CF9108
:109320001F910F91FF90EF90DF90CF90BF90AF9083
:109330009F908F907F906F905F904F9008956FEB0C
:109340007CE0CE01C1960E943A5FCE01C1960E9498
:109350004C3FCE01C1960E94505EBE016B5D7F4FB7
:109360008BEB94E10E94995FE4CD1F93CF93DF9341
:10937000CDB7DEB7A8970FB6F894DEBF0FBECDBF4E
:10938000182F0E9428778EE10E94067662E08BE318
:1093900091E10E94329960E08BE391E10E94329961
:1093A0000E94A4758EE10E94067661E08BE391E154
:1093B0000E94329960E28BE391E10E9432990E940F
:1093C000A47580E290E09093E8138093E71380E027
:1093D00090E8A9E8B4E48093D8049093D904A093CA
:1093E000DA04B093DB0480E090E0A5E7B4E4809376
:1093F000D4049093D504A093D604B093D704BE01AF
:109400006F5F7F4F84EE93E10E94916B112309F40B
:1094100099C08091250E882309F494C068E676E00F
:109420008EE990E10E94A75F8EE990E10E9475604D
:1094300068E576E08EE990E10E94A75FBE016F5F6C
:109440007F4F8EE990E10E94786068E476E08EE9D3
:1094500090E10E94A75F4D855E856F8578892AE03F
:1094600030E08EE990E10E9428608EE990E10E9450
:10947000756068E376E08EE990E10E94A75F498914
:109480005A896B897C892AE030E08EE990E10E945C
:1094900028608EE990E10E94756068E276E08EE9CE
:1094A00090E10E94A75F20E030E040E251E4698D46
:1094B0007A8D8B8D9C8D0E9497A442E00E944A7603
:1094C00069EB7BE08EE990E10E94786068E176E0EC
:1094D0008EE990E10E94A75F20E030E040E251E495
:1094E0006D8D7E8D8F8D98A10E9497A442E00E9481
:1094F0004A7669EB7BE08EE990E10E94786068E053
:1095000076E08EE990E10E94A75F20E030E040E243
:1095100051E469A17AA18BA19CA10E9497A442E089
:109520000E944A7669EB7BE08EE990E10E947860C8
:1095300062EE75E08EE990E10E94A75F8EE990E10E
:109540000E94756064EF71E080E090E00E94986E88
:10955000A8960FB6F894DEBF0FBECDBFDF91CF91B6
:109560001F910895EF92FF920F931F93CF93DF9374
:109570001F92CDB7DEB77C01FC0100811181C801CB
:1095800069830E944EA56981681719F0C8010E947D
:1095900056A5C7010F90DF91CF911F910F91FF90BA
:1095A000EF900895CF92DF92EF92FF920F931F9367
:1095B000CF93DF93EC016A017B01E889F98982E0AE
:1095C00080834115514E61057105B1F060E079E08D
:1095D0008DE390E0A70196010E9490A589019A0170
:1095E00001501109210931093695279517950795DD
:1095F000980101151041A8F0E889F989108260E806
:1096000074E88EE190E0A70196010E9490A5DA012E
:10961000C9010197A109B109B695A79597958795B5
:109620009C01EC85FD853083EE85FF852083188EB7
:10963000EC89FD8986E08083EA89FB8980818061ED
:109640008083EA89FB89808188608083EA89FB893D
:10965000808180688083EA89FB8980818F7D808317
:10966000DF91CF911F910F91FF90EF90DF90CF90FE
:109670000895CF93DF93EC01FB01248135810E9493
:109680004E5FCE01DF91CF9108954F925F926F921E
:109690007F928F929F92AF92BF92DF92EF92FF9252
:1096A0000F931F93CF93DF93CDB7DEB7A9970FB674
:1096B000F894DEBF0FBECDBFD82E882351F0809125
:1096C000250E882331F06FEB7CE08EE990E10E945B
:1096D00078600E94287760E08DE20E946C8860E1EB
:1096E0008DE20E946C8868E08DE20E946C88409058
:1096F00025145090261460902714709028144982E5
:109700005A826B827C828090291490902A14A090B7
:109710002B14B0902C148D829E82AF82B8868091DB
:109720002D1490912E14A0912F14B09130148EA36B
:109730009FA3A8A7B9A789879A87AB87BC87DD2095
:1097400089F18091250E882369F17E019DE0E90E63
:10975000F11C67E67CE0C7010E942A5FC701BBD904
:10976000C7010E94505E8E010F5F1F4FD8016D919F
:109770007D918D919D918D0146E00E944A7668E829
:109780007DE08EE990E10E9498600E151F0571F74B
:109790006FEB7CE0C8010E943A5FC8019CD9C80108
:1097A0000E94505E23E938E144E85FE3C301B2015F
:1097B0000E9497A42B013C016D877E878F87988B31
:1097C00022E430E645E85FE3C501B4010E9497A4B6
:1097D0004B015C01698B7A8B8B8B9C8B25E83BEE74
:1097E00041E95FE36EA17FA188A599A50E9497A496
:1097F0006D8B7E8B8F8B988F409225145092261400
:1098000060922714709228148092291490922A143E
:10981000A0922B14B0922C1460932D1470932E14DC
:1098200080932F1490933014DD2009F4A3C080910D
:10983000250E882309F49EC07E01B9E1EB0EF11CD0
:109840006AE57CE0C7010E942A5FC70144D9C701CD
:109850000E94505E8E01035F1F4FF801619171916C
:10986000819191918F0142E00E944A7668E87DE003
:109870008EE990E10E9498600E151F0571F76FEB5D
:109880007CE0C8010E943A5FC80125D9C8010E9446
:10989000505E41E354E166E070E082E30E9401889B
:1098A00080903214912C982C882480913114882A2D
:1098B000A0903414B12CBA2CAA2480913314A82A75
:1098C000E0903614F12CFE2CEE2480913514E82A19
:1098D0006DE47CE08EE990E10E94A75F4AE050E0F1
:1098E000B4018EE990E10E946F6068E87DE08EE946
:1098F00090E10E9498604AE050E0B5018EE990E165
:109900000E946F6068E87DE08EE990E10E949860B7
:109910004AE050E0B7018EE990E10E946F606FEB82
:109920007CE08EE990E10E947860C8010E94C088C6
:1099300064E47CE08EE990E10E94A75F7E01F5E29D
:10994000EF0EF11CD8016D917D918D919D918D014E
:109950004AE00E944A7668E87DE08EE990E10E9444
:1099600098600E151F0571F76FEB7CE08EE990E1B2
:109970000E94786061E08DE10E946C88DD20B1F08A
:109980008091250E882391F060E37CE08EE990E1E0
:109990000E94A75FAE014B5D5F4F61E070E08DE11B
:1099A0000E9401888DA190E00E943C8862E08EE1D7
:1099B0000E946C8863E08FE10E946C8864E080E222
:1099C0000E946C88DD2009F450C08091250E882308
:1099D00009F44BC064E17CE08EE990E10E94A75F4E
:1099E000AE014B5D5F4F61E070E08EE10E94018847
:1099F000ADA0B12CAE014B5D5F4F61E070E08FE137
:109A00000E940188EDA0F12CAE014B5D5F4F61E03B
:109A100070E080E20E9401880DA110E04AE050E071
:109A2000B5018EE990E10E946F6068E87DE08EE903
:109A300090E10E9498604AE050E0B7018EE990E121
:109A40000E946F6068E87DE08EE990E10E94986076
:109A50004AE050E0B8018EE990E10E946F606FEB40
:109A60007CE08EE990E10E94786065E081E20E94EE
:109A70006C88DD20B1F08091250E882391F061E0A3
:109A80007CE08EE990E10E94A75FAE014B5D5F4FE5
:109A900061E070E081E20E9401888DA190E00E9467
:109AA0003C8866E082E20E946C88DD20B1F0809103
:109AB000250E882391F069EE7BE08EE990E10E940B
:109AC000A75FAE014B5D5F4F61E070E082E20E94F4
:109AD00001888DA190E00E943C8867E083E20E94AB
:109AE0006C88DD20B1F08091250E882391F063ED24
:109AF0007BE08EE990E10E94A75FAE014B5D5F4F76
:109B000061E070E083E20E9401888DA190E00E94F4
:109B10003C8868E084E20E946C88DD20B1F080918E
:109B2000250E882391F06BEB7BE08EE990E10E949B
:109B3000A75FAE014B5D5F4F61E070E084E20E9481
:109B400001888DA190E00E943C8869E085E20E9436
:109B50006C88DD20B1F08091250E882391F061EAB8
:109B60007BE08EE990E10E94A75FAE014B5D5F4F05
:109B700061E070E085E20E9401888DA190E00E9482
:109B80003C886AE086E20E946C88DD20B1F080911A
:109B9000250E882391F06BE87BE08EE990E10E942E
:109BA000A75FAE014B5D5F4F61E070E086E20E940F
:109BB00001888DA190E00E943C886BE088E20E94C1
:109BC0006C88DD20B1F08091250E882391F062E74A
:109BD0007BE08EE990E10E94A75FAE014B5D5F4F95
:109BE00061E070E088E20E9401888DA190E00E940F
:109BF0003C886CE089E20E946C88DD2009F479C021
:109C00008091250E882309F474C06AE57BE08EE913
:109C100090E10E94A75FAE014B5D5F4F61E070E095
:109C200089E20E9401888DA190E00E943C8863E453
:109C30007BE08EE990E10E94A75F66E070E087E23A
:109C40000E94528890E00E943C886CE27BE08EE9A2
:109C500090E10E94A75F65E070E087E20E94528871
:109C600090E00E943C8865E17BE08EE990E10E94F3
:109C7000A75F64E070E087E20E94528890E00E9453
:109C80003C886CEF7AE08EE990E10E94A75F62E089
:109C900070E087E20E94528890E00E943C8863EE68
:109CA0007AE08EE990E10E94A75F61E070E087E2D0
:109CB0000E94528890E00E943C886AEC7AE08EE92B
:109CC00090E10E94A75F60E070E087E20E94528806
:109CD00090E00E943C8869EB7AE08EE990E10E9476
:109CE000A75F63E070E087E20E94528890E00E94E4
:109CF0003C8841E067E070E087E20E94818841E0B3
:109D000063E070E087E20E94818841E063E070E0F8
:109D10008AE20E948188DD2091F08091250E8823BF
:109D200071F060EA7AE08EE990E10E94A75F63E05B
:109D300070E08AE20E94528890E00E943C8840E0F5
:109D400063E070E08AE20E948188DD2091F08091DA
:109D5000250E882371F066E87AE08EE990E10E9492
:109D6000A75F63E070E08AE20E94528890E00E9460
:109D70003C8841E062E070E08AE20E948188DD2058
:109D800091F08091250E882371F06AE67AE08EE9E1
:109D900090E10E94A75F62E070E08AE20E94528830
:109DA00090E00E943C8840E062E070E08AE20E941D
:109DB0008188DD2091F08091250E882371F06DE47B
:109DC0007AE08EE990E10E94A75F62E070E08AE2AB
:109DD0000E94528890E00E943C8841E061E070E07F
:109DE0008AE20E948188DD2091F08091250E8823EF
:109DF00071F061E37AE08EE990E10E94A75F61E093
:109E000070E08AE20E94528890E00E943C8840E024
:109E100061E070E08AE20E948188DD2091F080910B
:109E2000250E882371F064E17AE08EE990E10E94CA
:109E3000A75F61E070E08AE20E94528890E00E9491
:109E40003C8841E060E070E08AE20E948188DD2089
:109E500091F08091250E882371F068EF79E08EE90A
:109E600090E10E94A75F60E070E08AE20E94528861
:109E700090E00E943C8840E060E070E08AE20E944E
:109E80008188DD2091F08091250E882371F06BEDA3
:109E900079E08EE990E10E94A75F60E070E08AE2DD
:109EA0000E94528890E00E943C8841E066E070E0A9
:109EB00087E20E94818841E065E070E087E20E94CD
:109EC000818841E064E070E087E20E94818840E0A0
:109ED00062E070E087E20E94818840E061E070E02B
:109EE00087E20E94818840E060E070E087E20E94A3
:109EF0008188DD2009F475C08091250E882309F43E
:109F000070C063EC79E08EE990E10E94A75F66E0A3
:109F100070E08BE20E94528890E00E943C8865EAE3
:109F200079E08EE990E10E94A75F65E070E08BE246
:109F30000E94528890E00E943C8867E879E08EE9B0
:109F400090E10E94A75F64E070E08BE20E9452887B
:109F500090E00E943C886EE679E08EE990E10E94F4
:109F6000A75F62E070E08BE20E94528890E00E945E
:109F70003C8865E579E08EE990E10E94A75F61E0A9
:109F800070E08BE20E94528890E00E943C886CE373
:109F900079E08EE990E10E94A75F60E070E08BE2DB
:109FA0000E94528890E00E943C8869E279E08EE944
:109FB00090E10E94A75F63E070E08BE20E9452880C
:109FC00090E00E943C8864E179E08EE990E10E9493
:109FD000A75F64E070E08CE20E94528890E00E94EB
:109FE0003C8840E064E070E08CE20E948188AE0131
:109FF0004B5D5F4F61E070E08CE20E9401886DA1D3
:10A00000607F66608CE20E946C88DD2009F465C088
:10A010008091250E882309F460C060E079E08EE924
:10A0200090E10E94A75FAE014B5D5F4F61E070E081
:10A030008CE20E9401886DA16F7070E0665071091A
:10A04000072E000C880B990B0E9438A49B01AC01D1
:10A0500060E070E080E090E40E9430A820E030E012
:10A0600048EC50E40E9497A40E94B18869EE78E021
:10A070008EE990E10E94A75FAE014B5D5F4F61E00A
:10A0800070E080E30E9401884DA150E060E070E044
:10A090002AE08EE990E10E94E05F8EE990E10E9463
:10A0A000756061ED78E08EE990E10E94A75F61E064
:10A0B00070E080E30E94528890E00E943C8868EB48
:10A0C00078E08EE990E10E94A75F61E070E08FE2A6
:10A0D0000E94528890E00E943C8841E061E070E07C
:10A0E0008FE20E948188DD2091F08091250E8823E7
:10A0F00071F060EA78E08EE990E10E94A75F61E08C
:10A1000070E08EE20E94528890E00E943C8841E01C
:10A1100061E070E08EE20E94818840E067E070E0DC
:10A1200081E30E948188DD2009F455C08091250ECD
:10A13000882309F450C06DE878E08EE990E10E9430
:10A14000A75F67E070E081E30E94528890E00E9480
:10A150003C886DEB7BE08EE990E10E949860AE0157
:10A160004B5D5F4F61E070E080E00E9401888DA14F
:10A170000E9427746FEB7CE08EE990E10E9478608A
:10A180000DE110E069EE7BE08EE990E10E949860BD
:10A1900040E150E0B8018EE990E10E946F6061EC0F
:10A1A0007BE08EE990E10E949860AE014B5D5F4FCD
:10A1B00061E070E0802F0E9401888DA10E942774C9
:10A1C0006FEB7CE08EE990E10E9478600F5F1F4F9B
:10A1D0000A331105B9F6A9960FB6F894DEBF0FBE83
:10A1E000CDBFDF91CF911F910F91FF90EF90DF9046
:10A1F000BF90AF909F908F907F906F905F904F90A7
:10A2000008958F929F92AF92BF92CF92DF92EF927A
:10A21000FF920F931F93CF93DF93CDB7DEB7629773
:10A220000FB6F894DEBF0FBECDBF61E089E10E949A
:10A230000F6E61E089E10E94DD6D0E94287764EC79
:10A240007BE08EE990E10E94786077E2C72ED12C06
:10A25000E12CF12C00E010E08C2D0E9406760E948B
:10A26000A475811127C060ED7BE08EE990E10E942A
:10A27000986020E1B701A6018EE990E10E94E05FBD
:10A280008EE990E10E947560C092BF146CEE7BE095
:10A290008EE990E10E94986020E1B701A6018EE965
:10A2A00090E10E94E05F8EE990E10E9475600F5F8F
:10A2B0001F4F13C0843089F466E07CE08EE990E1A2
:10A2C0000E94986020E1B701A6018EE990E10E940A
:10A2D000E05F8EE990E10E9475608FEFC81AD80A9E
:10A2E000E80AF80AE0E4CE16D104E104F10409F02A
:10A2F000B3CF012B19F461E27CE002C067E37CE09C
:10A300008EE990E10E9478600E94D45B80E40E9414
:10A3100010760EEB14E0F80161918F018BEB94E164
:10A320000E941273F4E0063C1F07A9F70E94283F21
:10A330000E94EB678EED93E09093061580930515D0
:10A340000E944EA58093C60E8FED93E00E944EA50D
:10A350008093C70E8091C60E9091C70E18161906ED
:10A3600054F41092BD04019731F41092C70E10926C
:10A37000C60E0E94697965E47DE0CE0101960E94D7
:10A380002A5F4AE050E06FEF7FEFCE0101960E9416
:10A39000C540CE0101960E94505E40E052EC61E063
:10A3A00070E08EE990E1FED88091BD04882331F001
:10A3B00068EE73E080E090E00E94986E8EE990E194
:10A3C0000E94DC6A182F59EAC52E52E1D52E6CE2A4
:10A3D000E62EFF24F394C7010E944EA5F601819357
:10A3E0006F01FFEFEF1AFF0A86E2E81682E0F80637
:10A3F00091F78091AA1218160CF05CC61D36E1F494
:10A4000059C6CE0107960E94505E63E57CE08EE956
:10A4100090E10E9498602AE04AEF50E060E070E02E
:10A420008EE990E10E94E05F8EE990E10E94756004
:10A43000CE010D960E94505E8091B21281118091E2
:10A44000A9128093A4120E94D06E6093A012709300
:10A45000A1128093A2129093A312123709F465C13E
:10A4600010920615109205154AE1C42E42E1D42E31
:10A47000E12CF12CC7010E944EA5F60181936F01DA
:10A48000FFEFEF1AFF0A86E8E816F10499F78091CA
:10A490001A1290911B12A0911C12B0911D128536B8
:10A4A0009105A105B1050CF440C18093B9049093C6
:10A4B000BA04A093BB04B093BC0480911E12909187
:10A4C0001F12A0912012B09121128093B504909395
:10A4D000B604A093B704B093B8048091221290916F
:10A4E0002312A0912412B09125128093B10490936D
:10A4F000B204A093B304B093B40466E372E1CE0156
:10A5000001960E943A5FBE016F5F7F4F85EB94E139
:10A510000E94175ECE0101960E94505E64E972E1CE
:10A52000CE0101960E943A5FBE016F5F7F4F8FEAB6
:10A5300094E10E94175ECE0101960E94505E23E0D6
:10A5400030E040E050E065EB74E1CE0107960E94F8
:10A550004E5F23E030E040E050E06FEA74E1CE016E
:10A5600001960E944E5F2D813E818B859C85281728
:10A57000390729F589819A816F817885009719F0CB
:10A5800061157105B9F46115710559F02115310591
:10A5900041F0FB01208130E088279927821B930B33
:10A5A0000BC0009771F0232B61F0FC019081892F83
:10A5B00090E002C00E9486AB01E0892B19F000E018
:10A5C00001C001E0CE0101960E94505ECE010796C7
:10A5D0000E94505E011106C065EB74E18FEA94E1C0
:10A5E0000E94025E8091261290912712A09128125B
:10A5F000B09129128093AD049093AE04A093AF0460
:10A60000B093B00480912A1290912B12A0912C1239
:10A61000B0912D128093A9049093AA04A093AB0447
:10A62000B093AC0480912E1290912F12A091301211
:10A63000B09131128093A5049093A604A093A7042F
:10A64000B093A8048091321290913312A0913412E9
:10A65000B09135128093A1049093A204A093A30417
:10A66000B093A40460913E1270913F128091401209
:10A67000909141129B01AC010E94C1A8811130C090
:10A680006091421270914312809144129091451250
:10A690009B01AC010E94C1A8811122C00091461209
:10A6A000602F002E000C770B880B990B0E9438A4AA
:10A6B0009B01AC010E94C1A8811112C0A090471259
:10A6C000B0904812B5010B2C000C880B990B0E941E
:10A6D00038A49B01AC010E94C1A8882309F4CCC511
:10A6E0000E946499E12CF12CF701E859FD4E80801D
:10A6F0009180A280B380A5019401C501B4010E949C
:10A70000C1A8811107C0F701EA5DF14F80829182F3
:10A71000A282B382E4E0EE0EF11CF8E2EF16F1043F
:10A7200019F781E090E00E9438690EE8010F0230CD
:10A7300070F080911A1290911B12A0911C12B0918E
:10A740001D1285369105A105B1050CF0EDC0809173
:10A75000B9049091BA04A091BB04B091BC04809359
:10A760001A1290931B12A0931C12B0931D12809189
:10A77000B5049091B604A091B704B091B804809349
:10A780001E1290931F12A0932012B0932112809159
:10A79000B1049091B204A091B304B091B404809339
:10A7A000221290932312A0932412B09325121337F0
:10A7B000B1F086E392E1009739F048E050E0BC0147
:10A7C00085EB94E10E94638B84E992E1009739F074
:10A7D0004CE050E0BC018FEA94E10E94638B8091D1
:10A7E000AD049091AE04A091AF04B091B0048093F9
:10A7F000261290932712A0932812B09329128091C9
:10A80000A9049091AA04A091AB04B091AC048093E8
:10A810002A1290932B12A0932C12B0932D12809198
:10A82000A5049091A604A091A704B091A8048093D8
:10A830002E1290932F12A0933012B0933112809168
:10A84000A1049091A204A091A304B091A4048093C8
:10A85000321290933312A0933412B09335120E94A7
:10A860006499E6E2FEE0A8E6B2E14191519161917E
:10A8700071914D935D936D937D938EE0EE34F80767
:10A88000A1F76FE27DE0CE0101960E942A5FCE0122
:10A8900001960E946B45CE0101960E94505E2FE802
:10A8A000C22E24E0D22E32E5A32E32E1B32EE12CCB
:10A8B000F12C80918F04909190048E159F0554F196
:10A8C000F60180819181F501819391935F018091DF
:10A8D000250E8823C1F061EC7CE08EE990E10E94B6
:10A8E00098604AE050E0B7018EE990E10E946F6005
:10A8F00063E77CE08EE990E10E949860F601808138
:10A9000091810E943C88FFEFEF1AFF0A82E0C80E97
:10A91000D11CCFCF023040F41092061510920515CD
:10A9200080E090E00E943F79809190129091911286
:10A930008D7F892B41F440E855E260E070E084E6C9
:10A940009FE00E94D24A80919012909191120197BB
:10A9500041F440E052EC61E070E084E69FE00E9448
:10A96000D24A64E670E080E090E00E94986E8091A8
:10A97000901290919112892B09F0B7C01E3671F098
:10A9800080911A1290911B12A0911C12B0911D126D
:10A9900085369105A105B1050CF0A7C06FEB7CE0F1
:10A9A000CE0101960E943A5F6CE478E0CE010796F2
:10A9B0000E943A5F6FEA74E1CE0107960E94605DE3
:10A9C000BC01CE0101960E94025ECE0107960E9454
:10A9D000505EBE016F5F7F4F84E69FE00E94995FEB
:10A9E00068EB7BE080E090E00E94986EBE016F5FB4
:10A9F0007F4FCE0107960E94325FCE0107960E94DC
:10AA00006B45CE0107960E94505E6CE271E080E0DB
:10AA100090E00E94986E4091B3145091B41442504B
:10AA200051096FEA74E1CE0107960E94394BBE01CD
:10AA3000695F7F4FCE0101960E94175ECE01079697
:10AA40000E94505EBE016F5F7F4FCE0107960E944D
:10AA5000325FBE016F5F7F4FCE0107960E94605D3F
:10AA6000BC01CE0101960E94025ECE0107960E94B3
:10AA7000505E6FE878E0CE0107960E943A5FBE0113
:10AA80006F5F7F4FCE0107960E94605DBC01CE01D3
:10AA900001960E94025ECE0107960E94505EBE01A2
:10AAA0006F5F7F4F84E69FE00E94995F68EB7BE0D9
:10AAB00080E090E00E94986EBE016F5F7F4FCE01F4
:10AAC00007960E94325FCE0107960E946B45CE0129
:10AAD00007960E94505E6CE271E080E090E00E9478
:10AAE000986ECE0101960E94505E64E670E080E0B0
:10AAF00090E00E94986EF89482E08093B00080937A
:10AB0000B10094E69093B3001092B200809370006D
:10AB100078948093471110924B118091481160E016
:10AB20000E940F6E68E77CE0CE0101960E943A5FBA
:10AB30004AE050E06FEF7FEFCE0101960E94C540E2
:10AB4000CE0101960E94505E8091901290919112D8
:10AB5000892B01F56DE17BE0CE0101960E943A5F01
:10AB60006FEA74E1CE010196ABD7BC01CE01079626
:10AB70000E94325F4AE050E06FEF7FEFCE01079610
:10AB80000E948C3FCE0107960E94505ECE01019636
:10AB90000E94505E8091901290919112019701F560
:10ABA00069E07BE0CE0101960E943A5F6FEA74E1B2
:10ABB000CE01019685D7BC01CE0107960E94325F77
:10ABC0004AE050E06FEF7FEFCE0107960E948C3F86
:10ABD000CE0107960E94505ECE0101960E94505E03
:10ABE0008091901290919112029701F562E37BE0BF
:10ABF000CE0101960E943A5F6FEA74E1CE010196A0
:10AC00005FD7BC01CE0107960E94325F4AE050E058
:10AC10006FEF7FEFCE0107960E948C3FCE01079623
:10AC20000E94505ECE0101960E94505E809190126B
:10AC300090919112019709F05BC0CE0101960E949C
:10AC40002B638D819E81009709F449C0E981FA81C7
:10AC50002081222309F443C0079708F440C068E824
:10AC60007CE0CE0107960E943A5FBE016F5F7F4F86
:10AC7000CE01079625D7BC01CE010D960E94325F0A
:10AC8000CE010D960E944A7FCE010D960E94505E25
:10AC9000CE0107960E94505E66E27DE0CE010796E7
:10ACA0000E942A5F48EC50E06FEF7FEFCE010796DD
:10ACB0000E940B40CE010796F3D7BE016F5F7F4F16
:10ACC000CE0107960E94325F48EC50E06FEF7FEFB5
:10ACD000CE0107960E948C3FCE010796E1D768EE21
:10ACE00073E080E090E00E94986ECE010196D8D784
:10ACF00061EC7CE0CE0101960E943A5F6FEA74E15C
:10AD0000CE010196DDD66BE97CE0C3D6BC01CE0155
:10AD100007960E94325FCE0107960E944A7FCE01BD
:10AD20000796BED7CE010196BBD764E670E080E0FF
:10AD300090E00E94986E0E94287764E670E080E0C0
:10AD400090E00E94986E83E20E94067681E090E097
:10AD50000E9401760E94A47583E090E09093240EF7
:10AD60008093230E8CE40E9437896B017C0162E39F
:10AD700070E080E090E00E94986EA7019601C70104
:10AD8000B6010E94C1A8882309F479C086E60E9412
:10AD900037896B017C0162E370E080E090E00E9403
:10ADA000986EA7019601C701B6010E94C1A8882329
:10ADB00009F465C081E090E09093240E8093230E07
:10ADC00040E052EC61E070E081E090E10E94D24A04
:10ADD00064E670E080E090E00E94986E81E090E18F
:10ADE0000E94096D40E052EC61E070E081E090E18A
:10ADF0000E94D24A8CED95E0A0E0B0E0809305106F
:10AE000090930610A0930710B093081064E670E0CA
:10AE100080E090E00E94986E92E0C92ED12C00E074
:10AE200065E070E080E090E00E94986EE12CF12CEB
:10AE3000812C912C5401011191C281E090E10E947A
:10AE4000FE6A892B39F4E5E18E169104A104B10460
:10AE50000CF084C2F3E0EF16F1040CF4C3C27EC21E
:10AE6000002309F489C26DE07DE0CE010196F2D79E
:10AE7000CE0101960E946B45CE01019611D78091BB
:10AE8000230E9091240E039761F46EED7CE0CE01C9
:10AE90000196E0D7CE0101960E946B45CE01019646
:10AEA000FFD683E08093CD130E94287780ED0E9427
:10AEB000307A853509F0C2C28AEA0E94058C9093E7
:10AEC000CF138093CE138CEA0E94058C9093D113FC
:10AED0008093D0138EEA0E94058C9093D3138093B5
:10AEE000D21380EB0E94058C9093DF138093DE13C6
:10AEF00082EB0E94058C9093E1138093E01384EB26
:10AF00000E94058C9093E3138093E21386EB0E94DA
:10AF1000058C9093D5138093D41388EB0E94058CF5
:10AF20009093D7138093D6138AEB0E94058C90934D
:10AF3000D9138093D8138CEB0E94058C9093DB136C
:10AF40008093DA138EEB0E94058C9093DD1380932F
:10AF5000DC1365EA7CE08FEA93E119D60E944E8CFF
:10AF60000E9438A40E9421A70E9438A420E030E06B
:10AF700048EC52E40E9488A6AB01BC0122E0CE015D
:10AF80000196C2D6BE016F5F7F4FCE0107966AD78A
:10AF90006BE877E0CE0107967CD5BC018FEA93E1A0
:10AFA000F0D5CE0107967CD6CE01019679D66FEA10
:10AFB00073E1CE01019656D7CE0101960E946B45F2
:10AFC000CE0101966DD66FE87CE08FEA93E1DFD584
:10AFD0006091B9047091BA048091BB049091BC0453
:10AFE0000E9438A420E030E048EC52E40E9488A699
:10AFF000AB01BC0122E0CE01019686D6BE016F5F97
:10B000007F4FCE0107962ED76BE877E0CE010796EB
:10B0100040D5BC018FEA93E1B4D5CE01079640D666
:10B02000CE0101963DD66FEA73E1CE0101961AD7A3
:10B03000CE0101960E946B45CE01019631D61136A4
:10B0400029F481E00E94454B81E011C08EE990E136
:10B050000E94DC6A182F64E670E080E090E00E94B5
:10B06000986E113671F380E00E94454B80E00E949B
:10B07000B54964E670E080E090E00E94986E10911F
:10B08000BD04112331F068EE73E080E090E00E948F
:10B09000986E65E577E08BEB93E19FD582E090E0D9
:10B0A0009093220E8093210E112309F4D6C10E94A1
:10B0B000897CD3C16FEB7CE0CE010D96DBD610927C
:10B0C000A91288E18093AA1284E08093AB121092B7
:10B0D000B0121092B11268E577E0CE010D967DD5E1
:10B0E00083EB92E1892B41F044E050E063EB72E1A5
:10B0F000CE010D960E94638B81E08093B71283E0AE
:10B100008093B81282E090E09093BA128093B912C3
:10B1100085E090E09093BC128093BB1265E577E0E8
:10B12000CE010D965AD58DEB92E1009739F044E0AF
:10B1300050E0BC01CE010D960E94638B82E08093AB
:10B14000C11283E08093C21282E090E09093C41217
:10B150008093C31285E090E09093C6128093C5124D
:10B1600062E577E0CE010D9638D587EC92E1009745
:10B1700039F044E050E0BC01CE010D960E94638B93
:10B1800083E08093CB128093CC1282E090E0909386
:10B19000CE128093CD1285E090E09093D0128093F0
:10B1A000CF126EE37CE0CE010D9617D581ED92E1D2
:10B1B000009739F044E050E0BC01CE010D960E94AA
:10B1C000638B85EF8093D51283E08093D61282E063
:10B1D00090E09093D8128093D71285E090E09093FE
:10B1E000DA128093D9128CE291E00E94B979CE01F3
:10B1F00001960E941462BE016F5F7F4F8EE990E15D
:10B2000087D7CE0101964CD561E47CE08EE990E1D0
:10B210008FD72AE04AE050E060E070E08EE990E1EC
:10B22000CFD68EE990E161D765E77CE0CE01079645
:10B2300011D6BE01695F7F4F8EE990E169D7E12C9D
:10B24000F12C8091AB12082E000C990BE816F90630
:10B250000CF0D7C8B701CE0101960E944D86BE0101
:10B260006F5F7F4F8EE990E153D7CE01019618D5DD
:10B27000EFEFEE1AFE0AE5CF90904912692D092CE6
:10B28000000C770B880B990B0E9438A49B01AC0132
:10B290000E94C1A8811124CAC0904A12D0904B12BA
:10B2A000E0904C12F0904D12A7019601C701B60133
:10B2B0000E94C1A8811114CA60914E1270914F1260
:10B2C00080915012909151129B01AC010E94C1A833
:10B2D000811106CA609164127091651280916612A4
:10B2E000909167129B01AC010E94C1A88111F8C91D
:10B2F0006091901270919112072E000C880B990B9F
:10B300000E9438A49B01AC010E94C1A88111E8C928
:10B310006091921270919312072E000C880B990B7A
:10B320000E9438A49B01AC010E94C1A88111D8C918
:10B3300003300CF0D5C9F2E0F9150CF4D1C98BEF4C
:10B34000A816B1040CF0CCC920E030E0A901C70177
:10B35000B6010E9432A487FFC5C9C2C964E670E085
:10B3600080E090E00E94986ECA94CD2809F478CDD0
:10B37000CC24C394D12C54CD1092240E1092230EC1
:10B3800081E090E10E94096D64E670E080E090E069
:10B390000E94986E40E855E260E070E081E090E144
:10B3A0000E94D24A81E090E10E94FE6A892B09F452
:10B3B00066CD63EF7CE0CE0101964CD5CE010196BF
:10B3C0000E946B45CE0101966BD482E090E0909391
:10B3D000240E8093230E64E670E080E090E00E94EB
:10B3E000986E4DCD81E090E10E94FE6A892B71F04C
:10B3F00081E090E10E94DC6AE1E0F0E0EC0FFD1FEB
:10B40000EE0DFF1D8083EFEFEE1AFE0A65E070E09F
:10B4100080E090E00E94986EF2E0EF16F10444F0B4
:10B4200089818B3B29F401E08A818A3A09F000E0A6
:10B430008FEF881A980AA80AB80AFDCC68EB7CE05E
:10B44000CE01019607D5CE0101960E944A7FCE011A
:10B45000019626D410928E040CCE62960FB6F89404
:10B46000DEBF0FBECDBFDF91CF911F910F91FF9037
:10B47000EF90DF90CF90BF90AF909F908F90089506
:10B480000895CF92DF92EF92FF920F931F93CF9385
:10B49000DF936C017A018B01C0E0D0E0CE15DF05AF
:10B4A00089F0D8016D918D01D601ED91FC9101904B
:10B4B000F081E02DC6011995892B11F47E0102C09F
:10B4C0002196ECCFC701DF91CF911F910F91FF9093
:10B4D000EF90DF90CF90089584E69FE00E94FE6A8F
:10B4E00021E0892B09F420E0822F089581E090E18A
:10B4F0000E94FE6A21E0892B09F420E0822F089542
:10B500008EE990E10E94FE6A21E0892B09F420E097
:10B51000822F08950E9460ABCF93DF93EC01888166
:10B520009981009711F00E94E4A9198218821D8266
:10B530001C821B821A82DF91CF9108950F931F9373
:10B54000CF93DF93EC0188819981009729F02A81BC
:10B550003B812617370788F48B016F5F7F4F0E946E
:10B560007CAA009761F0998388831B830A832C81CE
:10B570003D81232B11F4FC01108281E001C080E0A9
:10B58000DF91CF911F910F910895EF92FF920F934A
:10B590001F93CF93DF93FC012481358161157105E1
:10B5A00011F480E018C041155105A1F07B01EC01B8
:10B5B0008A01020F131FB801C1DF882391F328818C
:10B5C00039818C819D81B701820F931F0E948FABBF
:10B5D0001D830C8381E0DF91CF911F910F91FF902C
:10B5E000EF900895EF92FF920F931F93CF93DF9305
:10B5F000EC017B018A01BA01A1DF811103C0CE01F8
:10B600008BDF07C01D830C83B701888199810E945D
:10B610008FABCE01DF91CF911F910F91FF90EF90F3
:10B620000895FF920F931F93CF93DF93CDB7DEB7AB
:10B630002B970FB6F894DEBF0FBECDBF81E090E12F
:10B640000E94096D40E855E260E070E081E090E121
:10B650000E94D24A64E670E080E090E00E94986E1A
:10B660008CED95E0A0E0B0E080930510909306107B
:10B67000A0930710B093081064E670E080E090E0BB
:10B680000E94986E8FEF898381E08A8386E88B839E
:10B690001C821D821E821F82188689E7898781E0AD
:10B6A00090E10E94926D62E370E080E090E00E9481
:10B6B000986E81E090E10E94CD6A089744F049E0DD
:10B6C00050E0BE016F5F7F4F81E090E1DADE62E320
:10B6D00070E080E090E00E94986E81E090E10E942E
:10B6E000FE6A892B01F181E090E10E94CD6A089702
:10B6F0008CF465E070E080E090E00E94986E00E0DD
:10B7000010E0F12C81E090E10E94FE6A0230110508
:10B71000A4F50BC049E050E0BE016F5F7F4F81E0B0
:10B7200090E1AFDEE6CFF12C28C081E090E10E94ED
:10B73000FE6A892BA1F465E070E080E090E00E9451
:10B74000986E02301105F1F69A8589819813DACF47
:10B750009B858B819813D6CFFF24F394D3CF81E0C0
:10B7600090E10E94DC6AEAE0F0E0EC0FFD1FE00FE0
:10B77000F11F80830F5F1F4FDECF62E370E080E038
:10B7800090E00E94986E81E090E10E94096D8F2DFB
:10B790002B960FB6F894DEBF0FBECDBFDF91CF91D1
:10B7A0001F910F91FF900895CF93DF930E94287708
:10B7B0001092C0148091C414823018F098E09093D5
:10B7C000C0149091C514992339F0813029F48091E7
:10B7D000C01484608093C01462E370E080E090E065
:10B7E0000E94986E6091C6148BEB94E10E94E47203
:10B7F00068EE73E080E090E00E94986E60E38BEB6F
:10B8000094E10E94FC72CBE4D6E4CE010197F1F7FB
:10B8100060E38BEB94E10E94FC722197F1F760E307
:10B820008BEB94E10E94FC7283E592E00197F1F7C3
:10B8300060E28BEB94E10E94FC728091C014806204
:10B840000E94107684E08093C1148CE00E941076F0
:10B8500081E00E941076CBE3DFE1CE010197F1F7A2
:10B8600082E08093C21486E00E94107682E00E94FB
:10B8700010762197F1F7DF91CF910895FC01808137
:10B880009181009711F00C945E9F60E070E0CB0115
:10B890000895FC0180819181009711F00C947E9FA6
:10B8A00060E070E0CB010895AF92BF92CF92DF923B
:10B8B000EF92FF920F931F93CF93DF93DC01CD9014
:10B8C000DC901197C114D10409F442C01496CD91B3
:10B8D000DC9115972097E1F18C0156017501BFEFBE
:10B8E000AB1ABB0AF7018081082E000C990B0E944D
:10B8F00002A4892B99F72197CC0DDD1D8881082E94
:10B90000000C990B0E9402A4892B91F4AE014F5FA9
:10B910005F4F4E195F09D80115965C934E931497AB
:10B92000CE14DF0450F4B701C6010E947DAB05C000
:10B93000CE15DF0558F32197E1CFD801ED91FC91A9
:10B94000119714968D919C911597E80FF91F10820D
:10B95000DF91CF911F910F91FF90EF90DF90CF90EB
:10B96000BF90AF900895AF92BF92CF92DF92EF92C7
:10B97000FF920F931F93CF93DF93FC0124813581B6
:10B98000FB01448155818901041B150B41155105AB
:10B9900051F12115310539F12417350720F102172E
:10B9A000130718F08901015011097B01FC01A080E7
:10B9B000B180C501DFEFCFEF6501C00ED11EC81603
:10B9C000D906A0F0F701608171810E94B3AB0097A6
:10B9D00069F09C012A193B090217130710F0D22FB6
:10B9E000C32F0196ECCF8FEF9FEF02C08D2F9C2FBE
:10B9F000DF91CF911F910F91FF90EF90DF90CF904B
:10BA0000BF90AF900895CF93DF93FC0124813581DF
:10BA1000232B71F0FB01DC01CD91DC916081718100
:10BA2000CE010E94B3AB009719F08C1B9D0B02C096
:10BA30008FEF9FEFDF91CF910895FC012481358135
:10BA40006217730748F480819181009729F0FC0107
:10BA5000E60FF71F8081089580E00895FB0144817F
:10BA60005581FC01248135812417350778F08081C8
:10BA70009181009759F0FB01608171816115710519
:10BA800029F00E9496AB21E0892B09F020E0822F5B
:10BA90000895CF93DF93EC016115710559F0FB0117
:10BAA00001900020E9F73197AF01461B570B6DDD80
:10BAB000811102C0CE0130DDCE01DF91CF9108951A
:10BAC000CF93DF93EC01FB0144815581608171814B
:10BAD0005CDD811102C0CE011FDDCE01DF91CF916F
:10BAE0000895EF92FF920F931F93CF93DF93611509
:10BAF000710511F480E01DC08B01EC01CB010E94A7
:10BB0000AB9F0097A9F02C813D817C01E20EF31ED2
:10BB1000B701CE0113DD882369F3288139818C8137
:10BB20009D81B801820F931F0E94A49FFD82EC8229
:10BB300081E0DF91CF911F910F91FF90EF900895D9
:10BB4000CF93DF931F921F92CDB7DEB769831A821E
:10BB500041E050E0BE016F5F7F4F17DD0F900F9007
:10BB6000DF91CF9108956115710549F0FB010190B6
:10BB70000020E9F73197AF01461B570B06CD80E057
:10BB80000895FB014481558160817181FECCEF9263
:10BB9000FF920F931F93CF93DF93EC018B016115FD
:10BBA000710549F0CB010E94AB9F7C01BC01CE0125
:10BBB000C5DC811103C0CE01AFDC07C0FD82EC8281
:10BBC000B801888199810E94A49FCE01DF91CF9115
:10BBD0001F910F91FF90EF900895CF93DF93EC01A9
:10BBE0006115710551F0FB0101900020E9F73197D3
:10BBF000AF01461B570BF6DC01C08EDCCE01DF9196
:10BC0000CF910895CF93DF93EC01FB01861797073F
:10BC100051F0608171816115710521F04481558178
:10BC2000E1DC01C079DCCE01DF91CF9108950F9363
:10BC30001F93CF93DF938C01EB01FC0180819181F5
:10BC40000097B1F0688179816115710579F04281C1
:10BC500053812C813D814217530740F00E948FABE6
:10BC60008C819D81F8019583848313C00E94E4A98F
:10BC700088819981F801918380838A819B81938354
:10BC800082838C819D8195838483198218821B8293
:10BC90001A821D821C82DF91CF911F910F9108950E
:10BCA000FC01808191810C94E4A9EF92FF920F93A3
:10BCB0001F93CF93DF93CDB7DEB7A1970FB6F8945C
:10BCC000DEBF0FBECDBF7C01CB01BA01F7011182EF
:10BCD0001082138212821582148242E0420F8E017A
:10BCE0000F5F1F4F0E943F9FBC01C70176DFA196E7
:10BCF0000FB6F894DEBF0FBECDBFDF91CF911F917D
:10BD00000F91FF90EF900895EF92FF920F931F9382
:10BD1000CF93DF93CDB7DEB7A1970FB6F894DEBF10
:10BD20000FBECDBF7C01CB01BA01F7011182108299
:10BD3000138212821582148242E0420F8E010F5F3D
:10BD40001F4F0E943F9FBC01C70147DFA1960FB65E
:10BD5000F894DEBF0FBECDBFDF91CF911F910F9141
:10BD6000FF90EF9008950F931F93CF93DF93CDB77C
:10BD7000DEB7A2970FB6F894DEBF0FBECDBF8C0121
:10BD8000CB01BA01F801118210821382128215824E
:10BD9000148230E0AE014F5F5F4F0E94C89FBE012A
:10BDA0006F5F7F4FC80119DFA2960FB6F894DEBF10
:10BDB0000FBECDBFDF91CF911F910F9108950F93CB
:10BDC0001F93CF93DF93CDB7DEB762970FB6F8948A
:10BDD000DEBF0FBECDBF8C01CB01F80111821082F6
:10BDE000138212821582148250E0BE016F5F7F4F72
:10BDF0000E94B49FBE016F5F7F4FC801EEDE629666
:10BE00000FB6F894DEBF0FBECDBFDF91CF911F916B
:10BE10000F910895CF93DF931F921F92CDB7DEB796
:10BE2000FC011182108213821282158214826983AE
:10BE30001A82BE016F5F7F4FD0DE0F900F90DF91AF
:10BE4000CF910895FC011182108213821282158213
:10BE50001482EDCEFC0111821082138212821582AF
:10BE6000148295CEFC0111821082138212821582F7
:10BE70001482C8CEFC0111821082138212821582B4
:10BE800014826115710549F0FB0101900020E9F76A
:10BE90003197AF01461B570BA5CB0895BF92CF92A8
:10BEA000DF92EF92FF920F931F93CF93DF937C016A
:10BEB0006B018A01E9012417350720F4812F8901DC
:10BEC000C42FD82F6FEB7CE0C701D4DFD6011496C6
:10BED0008D919C91159708171907C8F48C179D0729
:10BEE00008F4EC01D601ED91FC911197EC0FFD1FC8
:10BEF000B08010824D915C91BA01600F711FC70133
:10BF00006CDED601ED91FC91EC0FFD1FB082C701F4
:10BF1000DF91CF911F910F91FF90EF90DF90CF9025
:10BF2000BF900895DC01ED91FC910190F081E02D2E
:10BF30001994DC01ED91FC91DB0114964D915C911B
:10BF400015976D917C910280F381E02D1994EF9209
:10BF5000FF920F931F93CF93DF938C017B01C0E07F
:10BF6000D0E0F701EC0FFD1F6491662361F0D8016A
:10BF7000ED91FC910190F081E02DC8011995892B7C
:10BF800011F02196EECFCE01DF91CF911F910F914D
:10BF9000FF90EF9008956115710579F0FB01019014
:10BFA0000020E9F73197AF01461B570BDC01ED91FB
:10BFB000FC910280F381E02D199480E090E00895D7
:10BFC0004F925F926F927F92EF92FF920F931F9327
:10BFD000CF93DF93CDB7DEB7A1970FB6F894DEBF4E
:10BFE0000FBECDBF7C01FA01CB0119A2223008F4AB
:10BFF0002AE08E010F5D1F4F422E512C612C712CB7
:10C00000BF01A30192010E9490A5F901CA0101504C
:10C0100011096A3014F4605D01C0695CD8016C9349
:10C02000232B242B252B61F7B801C701B4DFA19680
:10C030000FB6F894DEBF0FBECDBFDF91CF911F9139
:10C040000F91FF90EF907F906F905F904F900895C9
:10C05000CF92DF92EF92FF920F931F93CF93DF93D4
:10C06000EC016A017B012115310579F4E881F98140
:10C070000190F081E02D642FDF91CF911F910F91FE
:10C08000FF90EF90DF90CF9019942A303105D9F4CA
:10C0900077FF18C06DE246DF8C0144275527BA01AF
:10C0A0004C195D096E097F092AE0CE0189DF800FF6
:10C0B000911FDF91CF911F910F91FF90EF90DF9033
:10C0C000CF9008952AE0B701A601CE01DF91CF916C
:10C0D0001F910F91FF90EF90DF90CF9071CF9A0159
:10C0E000AB01770F660B770BB3CF6DEB7CE053CFD3
:10C0F0000F931F93CF93DF93EC014DDF8C01CE01A3
:10C10000F4DF800F911FDF91CF911F910F91089560
:10C110000F931F93CF93DF93EC010BDF8C01CE01C4
:10C12000E4DF800F911FDF91CF911F910F91089550
:10C1300032CF1F920F920FB60F9211240BB60F92AF
:10C140002F933F934F935F936F937F938F939F931F
:10C15000AF93BF93EF93FF9384E69FE00E942B6D14
:10C16000FF91EF91BF91AF919F918F917F916F91CF
:10C170005F914F913F912F910F900BBE0F900FBE8B
:10C180000F901F9018951F920F920FB60F921124C7
:10C190000BB60F922F933F934F935F936F937F93C1
:10C1A0008F939F93AF93BF93EF93FF9384E69FE0AA
:10C1B0000E94C76CFF91EF91BF91AF919F918F91BA
:10C1C0007F916F915F914F913F912F910F900BBE97
:10C1D0000F900FBE0F901F9018951F920F920FB6E1
:10C1E0000F9211240BB60F922F933F934F935F93AF
:10C1F0006F937F938F939F93AF93BF93EF93FF932F
:10C2000081E090E10E942B6DFF91EF91BF91AF9182
:10C210009F918F917F916F915F914F913F912F915E
:10C220000F900BBE0F900FBE0F901F9018951F928E
:10C230000F920FB60F9211240BB60F922F933F93CC
:10C240004F935F936F937F938F939F93AF93BF931E
:10C25000EF93FF9381E090E10E94C76CFF91EF9113
:10C26000BF91AF919F918F917F916F915F914F910E
:10C270003F912F910F900BBE0F900FBE0F901F900C
:10C2800018951F920F920FB60F9211240BB60F92B2
:10C290002F933F934F935F936F937F938F939F93CE
:10C2A000AF93BF93EF93FF938EE990E10E942B6DC4
:10C2B000FF91EF91BF91AF919F918F917F916F917E
:10C2C0005F914F913F912F910F900BBE0F900FBE3A
:10C2D0000F901F9018950F931F93CF93C091D20486
:10C2E00060E08C2F0E94DD6D83E090E00197F1F714
:10C2F00061E08C2F0E94DD6D83E290E00197F1F701
:10C3000060E08C2F0E94DD6D8091D0049091D1046B
:10C310009927FC01E157F14F6491FC01E75BF14F74
:10C32000E491F0E0EE0FFF1FE15DF14F85919491F4
:10C3300000E412E42FE030E0462F0E94B79B611525
:10C3400071058105910549F0DC01CB010196A11D24
:10C35000B11DBC01CD019F7003C060E070E0CB0156
:10C360000E9436A420E030E048EC52E40E9488A607
:10C370002091520E3091530E4091540E5091550E13
:10C380000E9497A420E030E44CE156E40E9488A685
:10C3900020E030E040E05FE30E9497A4CF911F913E
:10C3A0000F910895CF92DF92EF92FF9294DF6B018D
:10C3B0007C0120E030E040E050E40E9477A71816AE
:10C3C0001CF489DF6B017C0120E030E040E050E4A8
:10C3D000C701B6010E9477A718161CF47CDF6B0119
:10C3E0007C0120E030E040E050E4C701B6010E944B
:10C3F00077A718161CF46FDF6B017C0120E030E09A
:10C4000040E050E4C701B6010E9477A718162CF44B
:10C41000FF90EF90DF90CF905ECFC701B601FF9005
:10C42000EF90DF90CF900895EF92FF920F931F93BC
:10C43000CF93DF93CDB7DEB768970FB6F894DEBF22
:10C440000FBECDBF8C0168E87DE0CE01079612DDFE
:10C4500060EC7CE0CE0101960DDD67ED7DE0C8016A
:10C46000F9DCBE016F5F7F4FC8018BDB6EEC7DE0B6
:10C47000C80137DB89EAE82E82E1F82EF7016081F6
:10C4800070E04AE0CE010D969ADCBE01635F7F4FFB
:10C49000CE014396E7DCBE01695F7F4FCE01439634
:10C4A0000FDBBC01C8016DDBCE014396F9DBCE0189
:10C4B0000D96F6DB61EC7DE0C80113DBF7016181CD
:10C4C000062E000C770B4AE0CE010D9678DCBE01FB
:10C4D000635F7F4FCE014396C5DCBE01695F7F4F2E
:10C4E000CE014396EDDABC01C8014BDBCE01439689
:10C4F000D7DBCE010D96D4DB67EB7DE0C801F1DA26
:10C50000F7016281062E000C770B4AE0CE010D96F2
:10C5100056DCBE01635F7F4FCE014396A3DCBE01B4
:10C52000695F7F4FCE014396CBDABC01C80129DB9E
:10C53000CE014396B5DBCE010D96B2DB6FEA7DE00E
:10C54000C801CFDAF701638174814AE0CE010D960C
:10C5500036DCBE01635F7F4FCE01439683DCBE01B4
:10C560006F5F7F4FCE014396ABDABC01C80109DB98
:10C57000CE01439695DBCE010D9692DB68E97DE016
:10C58000C801AFDAF701658176814AE0CE010D96E8
:10C5900016DCBE01635F7F4FCE01439663DCBE01B4
:10C5A000695F7F4FCE0143968BDABC01C801E9DA9F
:10C5B000CE01439675DBCE010D9672DB6FE87DE010
:10C5C000C8018FDAF7016781062E000C770B6F5FC9
:10C5D0007F4F4AE0CE010D96F2DBBE01635F7F4FD5
:10C5E000CE0143963FDCBE01695F7F4FCE0143968B
:10C5F00067DABC01C801C5DACE01439651DBCE0132
:10C600000D964EDB64E87DE0C8016BDAF7016085CA
:10C61000062E000C770B4AE0CE010D96D0DBBE0152
:10C62000635F7F4FC801ADDACE010D9639DBCE01D5
:10C63000019636DBCE01079633DBC80168960FB64C
:10C64000F894DEBF0FBECDBFDF91CF911F910F9148
:10C65000FF90EF9008958F929F92AF92BF92CF92EA
:10C66000DF92EF92FF920F931F93CF93DF93CDB79B
:10C67000DEB768970FB6F894DEBF0FBECDBF6C0172
:10C680008091901290919112019729F06FEB7CE0CC
:10C69000C601F0DB1DC163EC7CE0CE010D96EADB48
:10C6A000BE01635F7F4F84E69FE043DC6CE271E094
:10C6B00080E090E00E94986ECE0107960E94B799A4
:10C6C00064E670E080E090E00E94986E00E010E088
:10C6D00085E0A82EB12C9AE0892E912C6EEC7CE09E
:10C6E000CE010196C7DBBE016F5F7F4FCE0107967B
:10C6F0008AD97C01CE010196D3DAA7014F5F5F4F43
:10C70000BE01695F7F4FCE0101960E94394BBE0189
:10C710006F5F7F4FCE010D968ADACE010196C0DAA7
:10C7200089899A89892B61F060E070E0CE010D96CD
:10C7300084D9082E000C990BC0970A9708F4B3C04F
:10C74000F12C64E77DE0CE01019684DB44E150E00A
:10C750006FEF7FEFCE0101960E940B40CE01019654
:10C760009FDA0F5F1F4F62E370E080E090E00E946D
:10C77000986EC801B5010E94FDA8019759F5CE0138
:10C7800001960E9429808D819E81892B59F0BE01DE
:10C790006F5F7F4F87EC93E135DA0E947808FF24C2
:10C7A000F39415C00431110594F0C801B4010E943E
:10C7B000FDA8892B61F4BE01635F7F4F84E69FE093
:10C7C000B8DB68EC70E080E090E00E94986ECE01EB
:10C7D000019666DACE0101960E94B799BE016F5F9D
:10C7E0007F4FCE01079623DACE01019659DA62E334
:10C7F00070E080E090E00E94986E0436110519F018
:10C80000FF2009F46BCF8091250E8823C9F061ECDD
:10C810007CE0CE0101962EDBBE01635F7F4FCE012F
:10C8200001964ED9BC01CE0143961CDBCE01439646
:10C830000E944A7FCE01439633DACE01019630DA68
:10C8400089899A89892B69F060E070E0CE010D96A4
:10C85000F4D8282F880F330B205331092A303105A3
:10C8600028F060ED7CE0C60105DB16C06CED7CE0D5
:10C87000CE010196FFDABE016F5F7F4FCE010D96AC
:10C88000EDD8182FCE0101960BDA1111EACFBE01B7
:10C89000635F7F4FC601D6DACE01079601DACE017B
:10C8A0000D96FED915C06CED7CE0CE010196E2DA62
:10C8B000BE016F5F7F4FCE010D96D0D8E82ECE011E
:10C8C0000196EED9FF24F394EE2009F43ACF38CF45
:10C8D000C60168960FB6F894DEBF0FBECDBFDF91DC
:10C8E000CF911F910F91FF90EF90DF90CF90BF906D
:10C8F000AF909F908F9008954F925F926F927F922A
:10C900008F929F92AF92BF92CF92DF92EF92FF925F
:10C91000CF93DF93CDB7DEB760970FB6F894DEBF45
:10C920000FBECDBF61E08091D2040E940F6E60E027
:10C930008091D0040E940F6E0E94298E60934E0E4B
:10C9400070934F0E8093500E9093510E23E333E972
:10C9500048E853E40E9488A620E030E040E85FE326
:10C960000E94C2A50E9480A826E636EA45EA53E462
:10C970000E9497A46093520E7093530E8093540EAE
:10C980009093550E0FDDAB01BC0123E0CE01019663
:10C99000BBD9BE016F5F7F4FCE01079663DA66E6B3
:10C9A0007DE0CE01079675D8BC0189EA93E12AD9CA
:10C9B000CE01079675D9CE01019672D967E07DE068
:10C9C000CE01019657DA69EA73E1CE01019678D873
:10C9D000BC018FEA93E116D9CE01019661D9E2DC60
:10C9E0009B01AC016D873E874F87588B0E94736E09
:10C9F0002B013C016EE170E080E090E00E94986EB7
:10CA0000D1DC6B017C010E94736E4B015C018418C8
:10CA10009508A608B7082D853E854F85588981ED74
:10CA2000881687E09806A104B1040CF43FC0C70142
:10CA3000B6010E94C1A56B017C0120E030E0A90194
:10CA40000E9477A718165CF426EA3BE944EC5BE306
:10CA5000C701B6010E9432A487FF0BC027C026EA97
:10CA60003BE944EC5BEBC701B6010E9477A71816BF
:10CA7000ECF0C501B40128EE33E040E050E00E9444
:10CA800064A5CA01B9010E9438A44B015C0120E0F1
:10CA900030E04AE754E4C701B6010E9497A4A5011B
:10CAA00094010E9488A6AB01BC0103C040E050E0A5
:10CAB000BA0122E0CE01019627D9BE016F5F7F4FF8
:10CAC000CE010796CFD964EE7CE0CE0107960E9496
:10CAD000495DBC0183EA93E195D8CE010796E0D881
:10CAE000CE010196DDD868EE7CE0CE010196C2D978
:10CAF00063EA73E1CE0101960E94605DBC018FEA9A
:10CB000093E13FD8CE010196CBD868E87DE0CE0115
:10CB10000196B0D963EA73E1CE0101960E94605D8F
:10CB2000BC0189EA93E12DD8CE010196B9D86CEE0B
:10CB30007CE0CE0101969ED94AE050E060E070E0D2
:10CB4000CE0101960E94C540CE010196A9D869EA9E
:10CB500073E1CE01019686D945E050E06FEF7FEF9B
:10CB6000CE0101960E948C3FCE01019699D863EFC9
:10CB70007CE08FEA93E10E94B35D60E08091D20493
:10CB80000E940F6E60960FB6F894DEBF0FBECDBF49
:10CB9000DF91CF91FF90EF90DF90CF90BF90AF905B
:10CBA0009F908F907F906F905F904F9008954F92DD
:10CBB0005F926F927F928F929F92AF92BF92CF922D
:10CBC000DF92EF92FF92CF93DF93CDB7DEB76897F6
:10CBD0000FB6F894DEBF0FBECDBF6B017C010E9483
:10CBE000D06E698B7A8B8B8B9C8B61E08091D204A9
:10CBF0000E940F6E60E08091D0040E940F6E0E9430
:10CC0000298E60934E0E70934F0E8093500E90932A
:10CC1000510E23E333E948E853E40E9488A620E05C
:10CC200030E040E85FE30E94C2A50E9480A826E6AB
:10CC300036EA45EA53E40E9497A46093520E70933B
:10CC4000530E8093540E9093550EACDB6D877E8708
:10CC50008F87988B0E94736E4B015C016AE070E0D5
:10CC600080E090E00E94986E66E57DE08FEA93E1B7
:10CC70000E94C75D20E030E04AE754E4C701B601F6
:10CC80000E9497A46D8B7E8B8F8B988F412C512C9B
:10CC90003201C12CD12C7601C701B6010E9438A403
:10CCA0002D893E894F89588D0E9432A487FF7AC111
:10CCB0000E94D06E29893A894B895C89621B730B6B
:10CCC000840B950B0E9436A420E030E04AE754E440
:10CCD0000E9488A6AB01BC0123E0CE01019614D8C6
:10CCE000BE016F5F7F4F89EA93E10E94175ECE011C
:10CCF00001960E94505E56DB6B017C01F4D79B01CC
:10CD0000AC01281939094A095B0949015A0131ED79
:10CD1000831637E09306A104B1040CF441C020E06F
:10CD200030E0A901C701B6010E9477A718165CF48C
:10CD300026EA3BE944EC5BE3C701B6010E9432A45A
:10CD400087FF0BC02DC026EA3BE944EC5BEBC70133
:10CD5000B6010E9477A718161CF1C501B40128EE90
:10CD600033E040E050E00E9464A5CA01B9010E948E
:10CD700038A44B015C012D853E854F855889C7013C
:10CD8000B6010E94C1A520E030E04AE754E40E94C9
:10CD900097A4A50194010E9488A64B015C0103C0E1
:10CDA000812C912C540169EA73E1CE0101965AD885
:10CDB00066EE7CE0CE0101960E94495DBC0189EAE5
:10CDC00093E10E94025ECE0101960E94505E23E034
:10CDD000B701A601CE0101960E94845EBE016F5F7D
:10CDE0007F4FCE0107963ED860E77BE0CE010796E5
:10CDF0000E94495DBC0183EA93E10E94025ECE017C
:10CE000007960E94505ECE0101960E94505E22E07D
:10CE1000B501A401CE0107960E94845E6EEA7BE014
:10CE2000CE01019627D869EA73E1CE0101960E94EE
:10CE3000605D66E07DE00E94495D63EA73E10E9407
:10CE4000605D69EE7CE00E94495DBE01695F7F4FD5
:10CE50000E94605D64EE7CE00E94495DBC018FEA47
:10CE600093E10E94C15DCE0101960E94505ECE0109
:10CE700007960E94505E20E030E0A901C501B40190
:10CE80000E9477A787FD06C068E87DE083EA93E10A
:10CE90000E94B35D22E0B501A401CE0101960E947B
:10CEA000845EBE016F5F7F4FCE0107960E94325FA6
:10CEB00064EE7CE0CE0107960E94495DBC0183EAE6
:10CEC00093E10E94C15DCE0107960E94505ECE01A3
:10CED00001960E94505E6FEA73E1CE0101960E94B6
:10CEE000325FCE0101960E944A7FCE0101960E94D8
:10CEF000505EC301B20125E030E040E050E00E9406
:10CF000064A5672B682B692B21F56CEE7CE0CE01C4
:10CF100001960E943A5F45E050E060E070E0CE018B
:10CF200001960E94C540CE0101960E94505E63EAC0
:10CF300073E1CE0101960E94325F45E050E06FEF51
:10CF40007FEFCE0101960E948C3FCE0101960E9498
:10CF5000505E6FEB7CE08FEA93E10E94ED5D65E04F
:10CF600070E080E090E0E4D61BD76B017C0129895A
:10CF70003A894B895C89C21AD30AE40AF50A12DAA3
:10CF80006D877E878F87988BAED64B015C016AE0F8
:10CF900070E080E090E0CCD63FEF431A530A630A7A
:10CFA000730A7ACE60E08091D20439D668960FB6C3
:10CFB000F894DEBF0FBECDBFDF91CF91FF90EF9011
:10CFC000DF90CF90BF90AF909F908F907F906F90A9
:10CFD0005F904F90089581E0809312028091130238
:10CFE000882341F088E08093C61460E08BEB94E1E5
:10CFF0000C94E47208958091130281110FC081E0B6
:10D0000080931302809312028091C114982F946030
:10D010009093C1148C600E94107618C08091120207
:10D020008823A1F01092C61460E08BEB94E10E947B
:10D03000E472109212028091C1148B7F8093C1140C
:10D0400088600E941076109213020895C4CF2F9228
:10D050003F924F925F926F927F928F929F92AF9288
:10D06000BF92CF92DF92EF92FF920F931F93CF93D5
:10D07000DF93CDB7DEB764970FB6F894DEBF0FBE6F
:10D08000CDBF7C0181E090E1C4D440E855E260E08E
:10D0900070E081E090E10E94D24A64E670E080E0B6
:10D0A00090E046D68CED95E0A0E0B0E080930510CE
:10D0B00090930610A0930710B093081064E670E0F8
:10D0C00080E090E035D68FEF898381E08A8386E81F
:10D0D0008B831C821D821E821F82188689E78987A6
:10D0E000C701880F991F9C8B8B8B212C312CC12C55
:10D0F000D12C812C912C5401CE14DF0444F081E01A
:10D1000090E187D4C114D10489F176012FC08B89B5
:10D110009C89281639069CF781E090E13ED2089759
:10D120004CF049E050E0BE016F5F7F4F81E090E13D
:10D130000E94415A65E070E080E090E0F9D500E09F
:10D1400010E0412C512C320181E090E157D2892B23
:10D1500031F484E048165104610471041CF4023077
:10D1600011057CF19FEF291A390AC6CFC501B40118
:10D170000E9438A44B015C01B701FF0C880B990B8E
:10D180000E9438A49B01AC01C501B4010E9488A68D
:10D1900064960FB6F894DEBF0FBECDBFDF91CF917E
:10D1A0001F910F91FF90EF90DF90CF90BF90AF90C5
:10D1B0009F908F907F906F905F904F903F902F90B7
:10D1C000089581E090E11AD2892B61F081E090E12D
:10D1D000F3D1EAE0F0E0EC0FFD1FE00FF11F8083D8
:10D1E0000F5F1F4F65E070E080E090E0A1D5023056
:10D1F0001105C1F59A858981981334C09B858B816F
:10D20000981330C081E090E1F9D1892B31F494E09A
:10D21000491651046104710484F40930110581F048
:10D2200081E090E1C9D1EAE0F0E0EC0FFD1FE00FF2
:10D23000F11F80830F5F1F4FE5CF043011057CF095
:10D240002D858C8590E0982F8827820F911D092EBF
:10D25000000CAA0BBB0B880E991EAA1EBB1E8FEFDB
:10D26000C81AD80A9FEF491A590A690A790A6CCF75
:10D270002F923F924F925F927F928F929F92AF92A6
:10D28000BF92CF92DF92EF92FF920F931F93CF93B3
:10D29000DF9300D01F92CDB7DEB76C0187E395E036
:10D2A0009C838B83E1E9F4E0FA83E98304E512E1EE
:10D2B000EE24E394F12C9DE3292E312C2EE3422E13
:10D2C000512C30E1A32EB12C41E1842E912C59E157
:10D2D000752E80918F04909190048E159F050CF40B
:10D2E000ECC0F1E0CF16D10431F4F80180819181D6
:10D2F000E981FA8109C0F2E0CF16D10439F4E9815D
:10D30000FA8180819181F80191838083E981FA819A
:10D3100080819181009749F4EB81FC818281938126
:10D320009093CF048093CE0428C08130910549F4B6
:10D33000EB81FC81828193819093CD048093CC0416
:10D340001CC08230910549F4EB81FC81828193817C
:10D350009093CB048093CA0410C0039771F4EB81BF
:10D36000FC81828193819093C9048093C8046FEB00
:10D370007CE08FE094E10E94ED5DE981FA8181918A
:10D380009191FA83E9838430910549F4EB81FC8122
:10D3900022813381309311022093100230C08530F6
:10D3A000910549F4EB81FC812281338130930102A4
:10D3B0002093000224C08630910549F4EB81FC8162
:10D3C0002281338130930E0520930D0524C08730D0
:10D3D000910549F4EB81FC8122813381309307026E
:10D3E0002093060224C08A30910549F4EB81FC8128
:10D3F000228133813093C7042093C6043AC085311B
:10D40000910549F4EB81FC8122813381309305023F
:10D41000209304022EC08631910549F4EB81FC81F2
:10D4200022813381309303022093020222C087318C
:10D430009105F9F4EB81FC8122813381A9014750E8
:10D4400051094230510540F4B092D304A092D20465
:10D450009092D1048092D0042550310922303105B8
:10D4600040F43092D3042092D2045092D1044092DE
:10D47000D0049C012B5031092A30310598F4EB81FE
:10D48000FC81228133813093C9042093C804789EA3
:10D49000B001799E700D1124635E7D4F8FE094E1A1
:10D4A0000E94ED5DFFEFEF1AFF0A8B819C810296CF
:10D4B0009C838B830E5F1F4F0CCF0F900F900F90AC
:10D4C0000F90DF91CF911F910F91FF90EF90DF9020
:10D4D000CF90BF90AF909F908F907F905F904F9034
:10D4E0003F902F9008957F928F929F92AF92BF921C
:10D4F000CF92DF92EF92FF920F931F93CF93DF9320
:10D50000782E8AE0882E912CCC24CA9493E0D92ED0
:10D51000EE24EA9423E0F22EA12CB12C00E010E0DE
:10D52000C0E0D0E0872DBAD30817190728F0A81655
:10D53000B90618F45C0101C08C018E159F0528F016
:10D540008C159D0518F46C0101C07C01C80FD91F12
:10D5500065E070E080E090E0EBD381E0881A91080C
:10D5600009F70A0D1B1DCE01801B910B8C199D091B
:10D570008E199F0966E070E00E94E9A8CB01DF9157
:10D58000CF911F910F91FF90EF90DF90CF90BF90C0
:10D59000AF909F908F907F900895FC01538D448DA4
:10D5A000252F30E0842F90E0821B930B541710F04E
:10D5B000CF96089501970895FC01918D828D98175B
:10D5C00061F0828DDF01A80FB11D5D968C91928D67
:10D5D0009F5F9F73928F90E008958FEF9FEF089564
:10D5E000FC01918D828D981731F0828DE80FF11D2D
:10D5F000858D90E008958FEF9FEF0895FC01918D48
:10D60000228D892F90E0805C9F4F821B91098F7340
:10D610009927089580E090E0892B21F00E94805A9C
:10D6200081111DC080E090E0892B41F080E090E006
:10D63000892B21F00E940000811114C080E090E04D
:10D64000892B21F00E94765A81110FC080E090E072
:10D65000892B81F00E946C5A81110AC008950E94A2
:10D660000000E0CF0E940000E9CF0E940000EECF52
:10D670000C940000089590E0FC013197E231F1052F
:10D6800008F04EC08827EA55FF4F8F4F0C9410A921
:10D69000809180008F7703C0809180008F7D809380
:10D6A0008000089580918000877FF9CF84B58F77BF
:10D6B00002C084B58F7D84BD08958091B0008F77BE
:10D6C00003C08091B0008F7D8093B0000895809159
:10D6D00090008F7707C0809190008F7D03C080916C
:10D6E0009000877F8093900008958091A0008F77AD
:10D6F00007C08091A0008F7D03C08091A000877F2C
:10D700008093A0000895809120018F7707C08091B9
:10D7100020018F7D03C080912001877F80932001AD
:10D7200008950F931F93CF93DF938C01EB0188E251
:10D73000FB0111928A95E9F74BE050E06AE07DE049
:10D74000CE010E94A4AB1B8681E090E0A0E0B0E097
:10D750008C879D87AE87BF87F80185899689A789C1
:10D76000B08D888B998BAA8BBB8B82E090E0A0E078
:10D77000B0E08C8B9D8BAE8BBF8B1CA21DA21EA21A
:10D780001FA280E090E0A8E4B4E4888F998FAA8F6C
:10D79000BB8F80E090E0A8E4B4EC8C8F9D8FAE8FBF
:10D7A000BF8F8DEC9CECACE4BEE388A399A3AAA345
:10D7B000BBA3DF91CF911F910F9108954F925F927C
:10D7C0006F927F928F929F92AF92BF92CF92DF9291
:10D7D000EF92FF920F931F93CF93DF938C01EB0196
:10D7E00084E2FB0111928A95E9F78EE10E940676A8
:10D7F00083E090E00E9401760E94A47566E08EE1CD
:10D800000E94E3791092190F8093180F90E08630F0
:10D810009105ECF38BE391E1DDD4882E8BE391E16C
:10D82000D9D4982E8BE391E1D5D4682E8BE391E186
:10D83000D1D4782E8BE391E1CDD4482E8BE391E1C6
:10D84000C9D4582EB82CA12CB5016929072E000C7B
:10D85000880B990B0E9438A44B015C01F801658389
:10D86000768387839087D42CC12CB6016529072E37
:10D87000000C880B990B0E9438A4F801618772870D
:10D8800083879487F62CE12CB7016729072E000CBB
:10D89000880B990B0E9438A4F801658776878787E3
:10D8A000908B118A128A138A148A84E290E0A0E095
:10D8B000B0E088839983AA83BB8385899689A789E9
:10D8C000B08D8C839D83AE83BF8382E090E0A0E027
:10D8D000B0E088879987AA87BB87188A198A1A8A2D
:10D8E0001B8AC090D804D090D904E090DA04F0905C
:10D8F000DB04A7019601C501B4010E9488A620E0BF
:10D9000030E048EC52E40E9497A46C8B7D8B8E8BA8
:10D910009F8BA7019601F8016185728583859485A7
:10D920000E9488A620E030E048EC52E40E9497A4D0
:10D93000688F798F8A8F9B8F2091D4043091D50482
:10D940004091D6045091D704F80165857685878586
:10D9500090890E9488A620E030E048EC52E40E94C2
:10D9600097A46C8F7D8F8E8F9F8F81E0DF91CF91F9
:10D970001F910F91FF90EF90DF90CF90BF90AF90ED
:10D980009F908F907F906F905F904F900895FC01D3
:10D99000A089B1898C91A689B78982FD0FC09C911D
:10D9A000818D8F5F8F73228D821749F0218DDF016A
:10D9B000A20FB11D5D969C93818F08958C9108955F
:10D9C0001F920F920FB60F9211240BB60F922F9346
:10D9D0003F934F935F936F937F938F939F93AF93F7
:10D9E000BF93EF93FF938EE990E1D1DFFF91EF9129
:10D9F000BF91AF919F918F917F916F915F914F9167
:10DA00003F912F910F900BBE0F900FBE0F901F9064
:10DA10001895CF93DF93EC01E881F9810680F781B7
:10DA2000E02D1995EA89FB8980818F7E8083EA89C0
:10DA3000FB898081877F8083EA89FB8980818F775A
:10DA40008083EA89FB8980818F7D80838A8D898F9D
:10DA5000DF91CF910895FC01848DDF01A80FB11DE6
:10DA6000A35ABF4F2C91848D90E001968F73992714
:10DA7000848FA689B7892C93A089B1898C91806401
:10DA80008C93938D848D981306C00288F389E02DC2
:10DA900080818F7D80830895EF92FF920F931F9373
:10DAA000CF93DF93EC0181E0888F9B8D8C8D981351
:10DAB00005C0E889F989808185FD23C0F62E0B8D8C
:10DAC00010E00F5F1F4F0F731127E02E8C8DE812AF
:10DAD0000BC00FB607FCFACFE889F989808185FF72
:10DAE000F5CFCE01B8DFF2CF8B8DFE01E80FF11D2F
:10DAF000E35AFF4FF0820B8FEA89FB8980818062B5
:10DB000007C0EE89FF896083E889F9898081806494
:10DB1000808381E090E0DF91CF911F910F91FF9082
:10DB2000EF900895CF93DF93EC01888D8823C1F0A7
:10DB3000EA89FB89808185FD05C0A889B9898C9116
:10DB400086FD0EC00FB607FCF5CF808185FFF2CFB2
:10DB5000A889B9898C9185FFEDCFCE017CDFE8CF14
:10DB6000DF91CF910895CF93DF93282F30E0F90113
:10DB7000EB52F14F8491F901E157F14FD491F90142
:10DB8000E75BF14FC491CC2389F0811174DDEC2F58
:10DB9000F0E0EE0FFF1FE15DF14FA591B491EC9124
:10DBA000ED2381E090E021F480E002C080E090E08D
:10DBB000DF91CF910895862FD6CF1F93CF93DF9318
:10DBC000282F30E0F901EB52F14F8491F901E15730
:10DBD000F14FD491F901E75BF14FC491CC23C1F02F
:10DBE000162F811148DDEC2FF0E0EE0FFF1FEB5EEA
:10DBF000F14FA591B4918FB7F894111105C09C9184
:10DC0000ED2FE095E92302C0EC91ED2BEC938FBF53
:10DC1000DF91CF911F910895862F642FCECFCF93A0
:10DC2000DF9390E0FC01E157F14F2491FC01E75BA9
:10DC3000F14F8491882361F190E0880F991FFC01D6
:10DC4000E550F24FC591D491FC01EB5EF14FA591E7
:10DC5000B491611109C09FB7F894888120958223FF
:10DC60008883EC912E230BC0623061F49FB7F89447
:10DC70003881822F809583238883EC912E2B2C93DF
:10DC80009FBF06C08FB7F894E8812E2B28838FBFE3
:10DC9000DF91CF910895862F642FC1CF863308F08E
:10DCA000865390917B00282F2870977F922B90931A
:10DCB0007B0087702091DC0490E4299F900111245F
:10DCC000822B80937C0080917A00806480937A001C
:10DCD00080917A0086FDFCCF8091780020917900B8
:10DCE00090E0922B08953FB7F89480915B0E90914D
:10DCF0005C0EA0915D0EB0915E0E26B5A89B05C08E
:10DD00002F3F19F00196A11DB11D3FBFBA2FA92FBA
:10DD1000982F8827820F911DA11DB11DBC01CD0137
:10DD200042E0660F771F881F991F4A95D1F7089523
:10DD30008F929F92AF92BF92CF92DF92EF92FF921B
:10DD40006B017C01D0DF4B015C01C114D104E10403
:10DD5000F104E9F0C8DFDC01CB0188199909AA09AF
:10DD6000BB09883E9340A105B10578F321E0C21AB2
:10DD7000D108E108F10888EE880E83E0981EA11C06
:10DD8000B11CC114D104E104F10421F7DECFFF90EE
:10DD9000EF90DF90CF90BF90AF909F908F900895BD
:10DDA0002FB7F8946091570E7091580E8091590ECC
:10DDB00090915A0E2FBF08951F920F920FB60F9297
:10DDC00011242F933F938F939F93AF93BF93809191
:10DDD000570E9091580EA091590EB0915A0E309155
:10DDE000560E23E0230F2D3720F40196A11DB11DFF
:10DDF00005C026E8230F0296A11DB11D2093560EE3
:10DE00008093570E9093580EA093590EB0935A0ECC
:10DE100080915B0E90915C0EA0915D0EB0915E0EB4
:10DE20000196A11DB11D80935B0E90935C0EA09393
:10DE30005D0EB0935E0EBF91AF919F918F913F9118
:10DE40002F910F900FBE0F901F9018958F929F9259
:10DE5000AF92BF92CF92DF92EF92FF920F931F93F8
:10DE6000CF93DF93EC018E819F81A6D240E06CECD2
:10DE70008E819F8135D2488164E48E819F8130D22A
:10DE80008A81882309F43EC0E981E950E33040F4F7
:10DE9000F0E0EE0FFF1FE75BFA4F0081118102C037
:10DEA0000EEE12E08B818823E1F08881811119C088
:10DEB00077DF4B015C016801110FEE08FF088E81CE
:10DEC0009F81BBD18130F1F06BDFDC01CB018C197C
:10DED0009D09AE09BF0988159905AA05BB0578F308
:10DEE00011C0B801110F880B990BDF91CF911F91D1
:10DEF0000F91FF90EF90DF90CF90BF90AF909F90E9
:10DF00008F9016CFDF91CF911F910F91FF90EF90DF
:10DF1000DF90CF90BF90AF909F908F9008954F92D9
:10DF20005F926F927F928F929F92AF92BF92CF92A9
:10DF3000DF92EF92FF920F931F93CF93DF931F9285
:10DF40001F92CDB7DEB72C018A01FC018681978133
:10DF500069837A8331D269817A818823A1F1F201C0
:10DF600086819781FED140E06EEBF2018681978138
:10DF7000B7D178014801F9E08F0E911CF20166805B
:10DF8000778088E0A82EB12CCC24C394D12CC30177
:10DF900054D18111DC28CC0CF1E0AF1AB108B9F7EB
:10DFA000F701D1927F01E815F90541F7F201868169
:10DFB000978102D2813039F468E0C80127D191E01D
:10DFC000F8012085821390E0892F0F900F90DF9148
:10DFD000CF911F910F91FF90EF90DF90CF90BF9066
:10DFE000AF909F908F907F906F905F904F9008952B
:10DFF000CF93DF93CDB7DEB729970FB6F894DEBF86
:10E000000FBECDBFAE014F5F5F4F89DF882389F020
:10E010008D818F3361F020F48F3159F489E00CC089
:10E020008F3519F08F3739F004C08BE005C08AE0D6
:10E0300003C080E001C08CE029960FB6F894DEBFE3
:10E040000FBECDBFDF91CF910895DF92EF92FF9287
:10E050000F931F93CF93DF937C018B01D42EDC01B0
:10E060001696ED91FC911797138615861486DF019D
:10E070001B9633961E92AE17BF07E1F7C0E0B801BA
:10E08000D70116968D919C9117970E94F789D82FEA
:10E09000811102C0D0E00DC0CD1107C067E0C801FA
:10E0A000B5D0F8019781891721F0CF5FDC1690F386
:10E0B000E6CF8D2FDF91CF911F910F91FF90EF90C1
:10E0C000DF9008950F931F93CF93DF93CDB7DEB703
:10E0D00061970FB6F894DEBF0FBECDBF8C01462FFF
:10E0E000BE01665F7F4FB1DF811105C060E070E067
:10E0F0008EEF92EC4AC0AE014F5F5F4FBE01665F8C
:10E100007F4FC8010CDF882359F1698148E0649F83
:10E11000B00111248A81282F30E0322F2227330FBB
:10E12000330F330F262B372B8A858031E1F4688536
:10E1300070E08F81AB01481B5109CA019695982F59
:10E140008827979587950E94FDA860517109207FC7
:10E1500053E0220F331F5A95E1F7620F731F04C07B
:10E1600060E874EE01C0B901613854EE75070CF433
:10E17000BDCF072E000C880B990B0E9438A420E01D
:10E1800030E040E05CE30E9497A461960FB6F894FB
:10E19000DEBF0FBECDBFDF91CF911F910F910895CC
:10E1A00085ED8093BC008091BC0084FDFCCF109273
:10E1B000400F08950895E091190F8091180FE81706
:10E1C00030F4F0E0EA55F14F808190E008958FEF50
:10E1D0009FEF08959091190F8091180F981750F4A0
:10E1E000E92FF0E0EA55F14F208130E09F5F9093F6
:10E1F000190F02C02FEF3FEFC90108958091180F4A
:10E2000090E02091190F821B91090895DC0180E0B4
:10E21000615090F09D919827E92FEF70F0E0E55E56
:10E22000F04F249192959F70E92FF0E0E55DF04F5B
:10E23000E4918E2F8227ECCF0895FC01908101801C
:10E24000F281E02DF8948181892B81832281892FAD
:10E25000809528232283A7E0B0E01197F1F7218170
:10E2600082238183A3E2B0E01197F1F78081789453
:10E27000EFECF0E03197F1F7982381E009F480E0CA
:10E280000895FC0190810180F281E02D892F809515
:10E2900060FF12C0F8942281822382838181892BBE
:10E2A0008183A3E2B0E01197F1F78281982B9283EA
:10E2B000789487ED90E011C0F894228182238283C4
:10E2C0008181892B8183AFEFB0E01197F1F78281D3
:10E2D000982B928378948FE090E00197F1F708955E
:10E2E000CF92DF92EF92FF920F931F93CF93DF9322
:10E2F0001F92CDB7DEB76C01E62E08E010E0FF24D8
:10E30000F39461E08F2D8E2109F460E0C60149830A
:10E31000B8DFFF0C0150110949810115110589F77A
:10E32000411115C0F894D6011196ED91FC91129708
:10E3300091818C918095892381831196ED91FC9137
:10E34000129792818C9180958923828378940F9083
:10E35000DF91CF911F910F91FF90EF90DF90CF90C1
:10E360000895CF92DF92EF92FF920F931F93CF9376
:10E37000DF931F92CDB7DEB78C01F62E40E065E546
:10E380007983AEDFCF2C7981D72E760188E0E80E35
:10E39000F11CF60161916F0140E0C801A1DFCE14CC
:10E3A000DF04B9F70F90DF91CF911F910F91FF908C
:10E3B000EF90DF90CF900895FC0190810180F28171
:10E3C000E02DF8948181292F2095822381837894F0
:10E3D0008DE743E050E0815021F1DA011197F1F728
:10E3E00030813923C1F3F894828182238283818131
:10E3F000892B81837894ABE7B7E01197F1F7F89414
:10E40000818128232183A3E1B1E01197F1F7808175
:10E41000982381E009F080E07894E3E6F6E0319714
:10E42000F1F70895EF92FF920F931F93CF93DF932D
:10E43000CDB7DEB728970FB6F894DEBF0FBECDBFBD
:10E440008C01DC011696ED91FC91179713861586C9
:10E450001486DF011B9633961E92AE17BF07E1F7B5
:10E46000F80114821582EE24E394BE016F5F7F4FA2
:10E47000F801868197810E94F789882309F469C091
:10E4800067E0CE010196C2DE98858913EECFD801F0
:10E490008C91811121C016968D919C9117978CDFDC
:10E4A000BE016F5F7F4FF801868197815ADF40E0A0
:10E4B00064EBD80116968D919C91179711DFF801A6
:10E4C00086819781BADEF82ED80116968D919C919F
:10E4D000179772DFFF20B1F1F801F1808981803157
:10E4E000A1F1BE016F5F7F4FC80182DD8F1520F45F
:10E4F000D80111968C910AC08981803111F48CE089
:10E5000005C0BE016F5F7F4FC80172DDF8018183D6
:10E5100084818F5F84838981883261F030F4803117
:10E5200049F0823209F0A1CF05C08B3319F0823453
:10E5300009F09BCFD80115968C9115978F5F159692
:10E540008C9393CFD801EC92C7CFBCE0BF1580F27B
:10E55000D6CF28960FB6F894DEBF0FBECDBFDF91A1
:10E56000CF911F910F91FF90EF9008950F931F93FC
:10E57000CF93DF93EC01162F60E0812F50DB612FEA
:10E5800070E0FB01E157F14FE491E883FB01E75BA9
:10E59000F14FE491F0E0EE0FFF1FE15DF14F859147
:10E5A00094919A8389831B861D861C86FE013B9667
:10E5B0008E010D5F1F4F1292E017F107E1F7DF9117
:10E5C000CF911F910F9108950F931F93CF93DF93D6
:10E5D0001F92CDB7DEB78C01FC018481698316D30D
:10E5E000F80183856981862B90E00BD30F90DF9132
:10E5F000CF911F910F91A8C20F931F93CF938C01BE
:10E60000C62FE2DF6C2F6460C801DEDF6C2F6B7FEA
:10E61000C801DADF83EC90E00197F1F7CF911F9109
:10E620000F9108950F931F93CF938C01C62F607F96
:10E630006160E2DF80E1C89FB00111246160C80120
:10E64000DBDF81E090E0CF911F910F9108951F9241
:10E650000F920FB60F9211240BB60F922F933F9388
:10E660004F935F936F937F938F939F93AF93BF93DA
:10E67000EF93FF938091481176DA20914C113091FD
:10E680004D112F5F3F4F30934D1120934C119091BE
:10E690004B11953618F096E09093471190914711E1
:10E6A0009430C9F128F4923069F09330D1F05EC013
:10E6B000953009F451C0963009F058C091E090931C
:10E6C000181251C0811152C020914C1130914D113E
:10E6D0002436310508F442C01092181210924B11E2
:10E6E0001CC0813009F042C0E0914B1191E09E0FB7
:10E6F00090934B11F0E020914C1130914D11EE0FA1
:10E70000FF1FE95BFE4E3087278310924D11109258
:10E710004C1194E029C0811117C0E0914B1191E098
:10E720009E0F90934B11F0E020914C1130914D11C0
:10E73000EE0FFF1FE95BFE4E3087278310924D11CD
:10E7400010924C1193E010C020914C1130914D115A
:10E750002536310558F007C0811108C010924D11BF
:10E7600010924C1103C095E09093471190914A117B
:10E770009923B1F081110AC080914911882321F0B9
:10E780008091491161E009C02F9A0AC08091491116
:10E79000882329F08091491160E00FDA01C02F9899
:10E7A000FF91EF91BF91AF919F918F917F916F9169
:10E7B0005F914F913F912F910F900BBE0F900FBE25
:10E7C0000F901F901895CF92DF92EF92FF92CF9308
:10E7D000DF93EC01072E000C880B990B0E9438A4E4
:10E7E0006B017C0120E030E040E45FE30E9497A4ED
:10E7F00020E030E048E452E40E9488A60E9421A76D
:10E80000C617D707D4F020E030E040EA5FE3C70145
:10E81000B6010E9497A420E030E048E452E40E9450
:10E8200088A620E030E040E85FE30E94C2A50E9495
:10E8300021A721E06C177D070CF420E0822F90E0E7
:10E84000DF91CF91FF90EF90DF90CF9008950F93DD
:10E850001F93CF93DF93082F6BE87AE08EE990E166
:10E860000E949860C7E0D0E010E0B8010C2E02C012
:10E87000759567950A94E2F76170772742E050E05A
:10E880008EE990E10E946F60219778F7DF91CF9138
:10E890001F910F9108951F920F920FB60F9211249E
:10E8A0000BB60F922F933F934F935F936F937F938A
:10E8B0008F939F93AF93BF93EF93FF938091B90092
:10E8C000887F803609F49CC068F5883209F45BC003
:10E8D00090F4803109F454C038F4882309F4F6C068
:10E8E000883009F44DC0F5C0883109F44CC080323D
:10E8F00009F45DC0EEC0803409F468C048F4803388
:10E9000009F455C0883309F0E4C080933E0FD8C0A5
:10E91000803509F44FC0883509F45DC0883409F0AA
:10E92000D8C0D6C0883909F4C7C0A8F4883709F41C
:10E9300067C038F4883609F463C0803709F460C0D2
:10E94000C8C0883809F4B8C0803909F45FC080387D
:10E9500009F0BFC05BC0803B09F486C038F4803A40
:10E9600009F466C0883A09F47FC0B3C0803C09F45A
:10E97000A7C0883C09F4A4C0883B09F48AC0A9C098
:10E9800080911B0F10C090913D0F80913C0F981704
:10E9900070F5E0913D0F81E08E0F80933D0FF0E028
:10E9A000E45EF04F80818093BB0085EC86C080934D
:10E9B0003E0F8EC0E0913D0F81E08E0F80933D0FA2
:10E9C0008091BB00F0E0E45EF04F808390913D0FBA
:10E9D00080913C0F6EC0E0913D0F81E08E0F8093DF
:10E9E0003D0F8091BB00F0E0E45EF04F80838091AA
:10E9F0003F0F81116DC081E080931A0F84EA61C0DE
:10EA000083E08093400F1092A50ECFCF8091A50E8A
:10EA1000803208F051C0E091A50E81E08E0F809306
:10EA2000A50E8091BB00F0E0EB57F14F8083BDCF86
:10EA300085EC8093BC001092400F8091A50E80322F
:10EA400030F4E091A50EF0E0EB57F14F10826091A9
:10EA5000A50E70E0E091830EF091840E85E89EE0B3
:10EA600019951092A50E35C084E08093400F109246
:10EA7000820E1092810EE0917F0EF091800E19951A
:10EA80008091810E811105C081E08093810E1092EA
:10EA90005F0EE091820E81E08E0F8093820EF0E097
:10EAA000E15AF14F80818093BB009091820E80915A
:10EAB000810E981708F479CF85E88093BC0009C0CF
:10EAC00085EC8093BC001092400F03C010923E0F63
:10EAD00067DBFF91EF91BF91AF919F918F917F91F4
:10EAE0006F915F914F913F912F910F900BBE0F90BF
:10EAF0000FBE0F901F9018954091810E262F30E089
:10EB0000240F311D21323105DCF42091400F2430D7
:10EB1000C9F4FC0180E090E0861758F43091810E32
:10EB20002191DC01A15AB14FA30FB11D2C93019685
:10EB3000F3CF8091810E680F6093810E80E008957D
:10EB400081E0089582E008952091630F9091C714A9
:10EB5000213208F04AC08091400F8111FCCF32E091
:10EB60003093400F31E030933F0F3FEF30933E0F33
:10EB700010923D0F20933C0FA3E4BFE04CE15FE017
:10EB8000FA013E2F341B321718F43D913193F9CF1F
:10EB900010921B0F20911B0F990F922B90931B0F1C
:10EBA00090911A0F913061F410921A0F90911B0FEF
:10EBB0009093BB009091BC0093FDF8CF95EC01C001
:10EBC00095EE9093BC009091400F9230E1F39091BC
:10EBD0003E0F9F3F79F080913E0F803241F080914F
:10EBE0003E0F803331F084E005C081E003C082E055
:10EBF00001C083E01092420F1092630F1092410FF8
:10EC00000895682F8BE391E10C94329991E09093F1
:10EC1000410F8093C7141092420F1092630F089512
:10EC2000CF93C82F682F607F8BEB94E1E5DC80E108
:10EC3000C89FB00111248BEB94E1CF91DDCCCF9331
:10EC4000DF93CDB7DEB728970FB6F894DEBF0FBEBF
:10EC5000CDBF98E0EFE4F5E0DE01119601900D9252
:10EC60009A95E1F79091C414961710F46FEF690F1D
:10EC7000FE013196E60FF11DE60FF11D9081890F1F
:10EC8000806828960FB6F894DEBF0FBECDBFDF9127
:10EC9000CF91C6CF4F925F926F927F928F929F9249
:10ECA000AF92BF92CF92DF92EF92FF926B017C0105
:10ECB000B42E9B01AC010E94C1A8882319F060E228
:10ECC0007DE027C026013701E89477F82FEF3FEF6A
:10ECD0004FE75FE7C301B2010E94C1A881110DC0D7
:10ECE0002FEF3FEF4FE75FE7C301B2010E9432A46D
:10ECF00018161CF464E27DE00CC02FEF3FEF4FE7E5
:10ED00005FE4C701B6010E9477A7181694F468E281
:10ED10007DE08EE990E1FF90EF90DF90CF90BF9083
:10ED2000AF909F908F907F906F905F904F900C94DA
:10ED3000CB5F2FEF3FEF4FE75FECC701B6010E94BB
:10ED400032A487FDE4CF20E030E0A901C701B6017D
:10ED50000E9432A487FF0BC06DE28EE990E10E9411
:10ED6000925F4C01F7FAF094F7F8F09402C0812C0E
:10ED7000912CA12C60E070E080E09FE3AB1441F0A7
:10ED800020E030E040E251E40E9488A6A394F6CF50
:10ED90009B01AC01C701B6010E94C2A52B013C0139
:10EDA0000E9426A76B017C010E9436A49B01AC0146
:10EDB000C301B2010E94C1A52B013C012AE0B701A9
:10EDC000A6018EE990E10E94E05F7C01E80CF91C4D
:10EDD000BB2039F06EE28EE990E10E94925FE80E6E
:10EDE000F91EDB2CDD2031F120E030E040E251E47F
:10EDF000C301B2010E9497A42B013C010E9426A7E7
:10EE00004B01A12CB12C2AE0B501A4018EE990E1BF
:10EE10000E94E05FE80EF91EC501B4010E9436A40D
:10EE20009B01AC01C301B2010E94C1A52B013C01B1
:10EE3000DA94D8CFC701FF90EF90DF90CF90BF90CA
:10EE4000AF909F908F907F906F905F904F900895BC
:10EE50001092190F1092180F1092420F1092630F18
:10EE60001092400F81E080933F0F10921A0F61E0E3
:10EE700084E10E94DD6D61E085E10E94DD6DE9EBDA
:10EE8000F0E080818E7F808380818D7F808388E425
:10EE90008093B80085E48093BC0008952F923F9240
:10EEA0004F925F926F927F928F929F92AF92BF929A
:10EEB000CF92DF92EF92FF920F931F93CF93DF9346
:10EEC000CDB7DEB728970FB6F894DEBF0FBECDBF23
:10EED0004091C80E5091C90EC090CA0ED090CB0E72
:10EEE0004C155D052CF03C2D2D2D6A01432F522F22
:10EEF000ECECFEE060E070E0CB01019111910417B1
:10EF0000150754F44A01550FAA08BB08680D791D6E
:10EF10008A1D9B1DA80115C0C016D10654F40D2CE6
:10EF2000000CEE08FF086C0D7D1D8E1D9F1D6801F5
:10EF300008C0012E000C220B330B600F711F821FC3
:10EF4000931F2FE0E831F207C1F60E9438A420E0B9
:10EF500030E048E152E40E9488A66B017C0108EC95
:10EF60001EE0812C912C5401D8016D917D918D0171
:10EF7000072E000C880B990B0E9438A4A70196015C
:10EF80000E94C1A59B01AC010E9497A49B01AC010A
:10EF9000C501B4010E94C2A54B015C01BFE008316C
:10EFA0001B0711F720E030E04CE152E40E9488A6F4
:10EFB0000E9480A84B015C0120E030E040E85FE364
:10EFC0000E9477A718160CF06EC008EC1EE0212CEA
:10EFD000312C19821A821B821C82F8018191919135
:10EFE0008F019C01990F440B550B2D833E834F835A
:10EFF0005887CA01B9010E9438A4A70196010E944E
:10F00000C1A52B013C0120E030E0A9010E9477A7B7
:10F01000181624F077FA709477F87094A50194018B
:10F02000C301B2010E9432A487FF13C089819A8173
:10F03000AB81BC812D813E814F815885820F931F0A
:10F04000A41FB51F89839A83AB83BC833FEF231A28
:10F05000330A4FE00831140709F0BFCF20E030E059
:10F0600040EC5FE3C501B4010E9497A44B015C0131
:10F0700055E0251631040CF4A8CF69817A818B8183
:10F080009C810E9438A46B017C01B101330C880B78
:10F09000990B0E9438A49B01AC01C701B6010E94E4
:10F0A00088A66B017C01C701B60128960FB6F894BB
:10F0B000DEBF0FBECDBFDF91CF911F910F91FF90AB
:10F0C000EF90DF90CF90BF90AF909F908F907F9008
:10F0D0006F905F904F903F902F9008954F925F9266
:10F0E0006F927F928F929F92AF92BF92CF92DF9258
:10F0F000EF92FF920F931F93CF93DF9300D01F9255
:10F10000CDB7DEB76B017C0111E0A12EB12C45011A
:10F11000880C991C880C991CF401EB50FB4F408023
:10F12000518062807380A3019201C701B6010E94E1
:10F1300077A7181614F41F5FE8CFA3019201C70147
:10F14000B6010E9432A4840103521B4F811106C0F4
:10F15000D8016D917D918D919C9142C0C5018150E6
:10F16000904C880F991F880F991FFC01EB50FB4FA3
:10F17000208131814281538129833A834B835C838F
:10F18000FC01E352FB4F80809180A280B380C701D5
:10F19000B6010E94C1A56B017C01A5019401D801B3
:10F1A0006D917D918D919C910E94C1A59B01AC01B7
:10F1B000C701B6010E9497A46B017C0129813A81A5
:10F1C0004B815C81C301B2010E94C1A59B01AC01CE
:10F1D000C701B6010E9488A6A50194010E94C2A59C
:10F1E0000F900F900F900F90DF91CF911F910F9183
:10F1F000FF90EF90DF90CF90BF90AF909F908F9057
:10F200007F906F905F904F9008950F931F930E948F
:10F21000D06E6093091070930A1080930B10909336
:10F220000C10E0910110F09102100284F385E02DA2
:10F2300081E090E1199597FF1FC00E94D06E009168
:10F24000091010910A1020910B1030910C10DC0164
:10F25000CB01801B910BA20BB30B009105101091F9
:10F260000610209107103091081080179107A2070F
:10F27000B307B8F28FEF9FEF1F910F910895EF92B0
:10F28000FF920F931F93CF93DF931F921F92CDB7DF
:10F29000DEB70AE112E18A5192417C019701200F09
:10F2A000311FF80161918F013A832983CE010196C4
:10F2B0000E94B24AF2E1003A1F0781F78AE192E127
:10F2C0000F900F90DF91CF911F910F91FF90EF90D2
:10F2D00008950F931F93CF93DF931F921F92CDB783
:10F2E000DEB706EC1EE0F80160818EED93E09A83B4
:10F2F0008983CE0101960E94B24AF80161818FEDA7
:10F3000093E09A838983CE0101960E94B24AC80194
:10F310000F900F90DF91CF911F910F910895EF9271
:10F32000FF920F931F93CF93DF931F921F92CDB73E
:10F33000DEB709EA12E1895A92417C019701200F58
:10F34000311FF80161918F013A832983CE01019623
:10F350000E94B24AF2E1033B1F0781F789EA92E17A
:10F360000F900F90DF91CF911F910F91FF90EF9031
:10F370000895EF92FF920F931F93CF93DF931F9205
:10F380001F92CDB7DEB709EA12E1895A92417C019A
:10F390009701200F311FF80161918F013A83298372
:10F3A000CE0101960E94B24AF3E1033A1F0781F7AA
:10F3B00089EA92E10F900F90DF91CF911F910F9109
:10F3C000FF90EF9008959091400F9111FCCF91E044
:10F3D0009093400F90933F0F2FEF20933E0F10928A
:10F3E0003D0F260F20933C0F90931B0F90911B0F06
:10F3F000880F892B80931B0F80911A0F813061F445
:10F4000010921A0F80911B0F8093BB008091BC005B
:10F4100083FDF8CF85EC01C085EE8093BC00809120
:10F42000400F8130E1F380913D0F861710F4609119
:10F430003D0FACE1BFE026EA3EE0F9018E2F821BD2
:10F44000861718F48D918193F9CF862F0895613234
:10F4500008F060E2B8DF1092190F8093180F08953A
:10F460001F93CF93DF931F92CDB7DEB7682F87E747
:10F470006983CCDB69818BE391E10E94329964DB83
:10F4800087E7C4DB61E070E087E790E0E0DF8BE3D3
:10F4900091E10E94EA70182F57DB812F0F90DF91C6
:10F4A000CF911F9108958F929F92AF92BF92CF926A
:10F4B000DF92EF92FF920F931F93CF93DF937C0124
:10F4C000862F9BE0E916F10409F070C09091221498
:10F4D000992309F0F89462E10E946D87EC01809114
:10F4E0002214882309F07894209709F074C0D090F2
:10F4F0001D14C0901E146D2D70E080E090E00E94FD
:10F5000038A44B015C016C2D70E080E090E00E941B
:10F5100038A42DEC3CEC4CEC5DE30E9497A49B01DD
:10F52000AC01C501B4010E94C2A56093151470938B
:10F530001614809317149093181410911F140091AF
:10F540002014612F6F7770E080E090E00E9438A473
:10F550004B015C01602F70E080E090E00E9438A4D5
:10F560002DEC3CEC4CEC5DE30E9497A49B01AC01BC
:10F57000C501B4010E94C2A517FD09C0609319140A
:10F5800070931A1480931B1490931C140BC0DC010D
:10F59000CB01B0588093191490931A14A0931B14A4
:10F5A000B0931C14DC0C1D0D100F6FC096E1E91612
:10F5B000F10409F071C090912214992309F0F89494
:10F5C00061E00E946D87EC0180912214882309F08C
:10F5D00078942097A9F080E090ECA9E7B4EC8093B0
:10F5E000151490931614A0931714B09318148093C5
:10F5F000191490931A14A0931B14B0931C144FC0A9
:10F6000000911E14D0901D14602F70E07D2980E0C1
:10F6100090E00E9436A42DEC3CEC4CEC5DE30E94A3
:10F6200097A46093151470931614809317149093F5
:10F630001814C090201410911F14812F8F776C2DF7
:10F6400070E0782B80E090E00E9436A42DEC3CEC3A
:10F650004CEC5DE30E9497A417FD09C06093191458
:10F6600070931A1480931B1490931C140BC0DC012C
:10F67000CB01B0588093191490931A14A0931B14C3
:10F68000B0931C140D0DC00E1C0D80912114811718
:10F6900031F0CFEFDFEF03C0CFEFDFEF48C0CF3F58
:10F6A0009FEFD90709F410C1209709F01CC1809081
:10F6B000151490901614A0901714B090181420E010
:10F6C00030E048EC52E4C501B4010E9477A7181657
:10F6D0000CF006C1CBEFDFEF20E030E0A901C5015F
:10F6E000B4010E9432A487FF02C0CAEFDFEF80900E
:10F6F000191490901A14A0901B14B0901C1420E0C0
:10F7000030E048EC52ECC501B4010E9432A487FFFE
:10F7100002C0C9EFDFEF20E030E040EF52E4C50166
:10F72000B4010E9477A7181614F4C8EFDFEF8CE03D
:10F73000E816F10409F0DFC08CE568DA80E090E0BB
:10F7400060DA02DA65E08CE53EDE1092190F8093F4
:10F75000180FC82FD0E02097B1F0C530D10584F044
:10F7600000E010E08BE391E10E94EA70F801E653BB
:10F77000FB4E80870F5F1F4F0C171D079CF306C0C1
:10F78000CDEFDFEFB8C0CEEFDFEFB5C0C091D21440
:10F790000091D3146C2F70E080E090E00E9438A4B8
:10F7A0006B017C01602F70E080E090E00E9438A443
:10F7B0002DEC3CEC4CEC5DE30E9497A49B01AC016A
:10F7C000C701B6010E94C2A56093CA147093CB14FE
:10F7D0008093CC149093CD14D091D4141091D5145F
:10F7E0006D2F6F7770E080E090E00E9438A46B018D
:10F7F0007C01612F70E080E090E00E9438A42DEC45
:10F800003CEC4CEC5DE30E9497A49B01AC01C7016A
:10F81000B6010E94C2A5D7FF5AC0DC01CB01B05887
:10F820008093CE149093CF14A093D014B093D1149E
:10F83000802F8C0FC82FCD0FC10F8091D6148C1341
:10F8400043C0C090CA14D090CB14E090CC14F09078
:10F85000CD1420E030E048EC52E4C701B6010E942C
:10F8600077A718161CF4CBEFDFEF02C0C0E0D0E0A2
:10F8700020E030E0A901C701B6010E9432A487FF51
:10F8800002C0CAEFDFEFC090CE14D090CF14E0904A
:10F89000D014F090D11420E030E048EC52ECC701D5
:10F8A000B6010E9432A487FF02C0C9EFDFEF20E05B
:10F8B00030E040EF52E4C701B6010E9477A7181666
:10F8C000D4F4C8EFDFEF17C0CFEFDFEF14C06093C1
:10F8D000CE147093CF148093D0149093D114A8CFEA
:10F8E000C0E0D0E0F9CE229619F0CCEFDFEF1FCFC9
:10F8F000CEEFDFEF1CCFCE01DF91CF911F910F91A3
:10F90000FF90EF90DF90CF90BF90AF909F908F903F
:10F9100008958F929F92AF92BF92CF92DF92EF9213
:10F92000FF92CF93DF93CDB7DEB72C970FB6F89445
:10F93000DEBF0FBECDBF60EF7FE0CE0101960E941B
:10F940002A5F4CE251E06FEF7FEFCE0101960E94FB
:10F950008C3FCE0101960E94505E6091CC04709164
:10F96000CD0480912705909128059DDD84E1882EA6
:10F97000912CA12CB12CE12CF12C8FEFE81AF80A74
:10F98000C501B4010E94986E6091CC047091CD04C1
:10F99000809127059091280586DD23E0E216F10489
:10F9A00034F424E1820E911CA11CB11CE6CF2FE09F
:10F9B000E216F1041CF4892BA1F703C0892B09F08E
:10F9C0008BC180912705909128058B309105C9F452
:10F9D0008091191490911A14A0911B14B0911C14C9
:10F9E0008093DB149093DC14A093DD14B093DE14A9
:10F9F0008091151490911614A0911714B0911814B9
:10FA00001DC08631910521F30C9701F58091CE142C
:10FA10009091CF14A091D014B091D1148093DB14A5
:10FA20009093DC14A093DD14B093DE148091CA147B
:10FA30009091CB14A091CC14B091CD148093D71495
:10FA40009093D814A093D914B093DA144091DB1496
:10FA50005091DC146091DD147091DE1421E0CE0130
:10FA600007960E94845E6FE07AE0CE0101960E94C4
:10FA70003A5FBE01695F7F4FCE0101960E94605DD3
:10FA8000BC018FEA93E10E94025ECE0101960E94C2
:10FA9000505ECE0107960E94505E4091D71450915F
:10FAA000D8146091D9147091DA1421E0CE01079630
:10FAB0000E94845E69E97AE0CE0101960E943A5F75
:10FAC000BE01695F7F4FCE0101960E94605DBC015F
:10FAD0008FEA93E10E94C15DCE0101960E94505EC3
:10FAE000CE0107960E94505E62E37AE08FEA93E1CE
:10FAF0000E94B35D6FEB7CE0CE0101960E943A5FFD
:10FB000044E150E060E070E0CE0101960E94C54003
:10FB1000CE0101960E94505EC090DB14D090DC14A0
:10FB2000E090DD14F090DE1420E030E0A901C70180
:10FB3000B6010E9477A720E030E040E05FE387FD58
:10FB400005C0C701B6010E94C2A504C0C701B60125
:10FB50000E94C1A50E9421A72AE0AB01BC01CE01F1
:10FB600001960E94B35EBE016F5F7F4F89EA93E109
:10FB70000E94175ECE0101960E94505E60E087E011
:10FB80005ED869EA73E18BEB94E10E94995F6FEDB7
:10FB90008BEB94E10E94925F6FE97AE08BEB94E14A
:10FBA0000E9498606091D7147091D8148091D914F4
:10FBB0009091DA140E9421A74AE050E08BEB94E187
:10FBC0000E946F6062E37AE08BEB94E10E949860A0
:10FBD00064E670E080E090E00E94986EC090DB14D4
:10FBE000D090DC14E090DD14F090DE1420E030E0E2
:10FBF00040EF51E4C701B6010E9477A787FD03C01B
:10FC000061EE7FE054C020E030E040ED51E4C701F8
:10FC1000B6010E9477A787FD1FC061ED7FE0CE018E
:10FC200001960E942A5F4AE050E06FEF7FEFCE011D
:10FC300001960E948C3FCE0101960E94505E8091F9
:10FC4000BD04882331F06CED75E080E090E00E9407
:10FC5000986E61EC7FE02BC020E030E040EB51E497
:10FC6000C701B6010E9477A787FD03C063EB7FE061
:10FC70001EC064EA7FE0CE0101960E942A5F4AE03E
:10FC800050E06FEF7FEFCE0101960E948C3FCE01D6
:10FC900001960E94505E8091BD04882331F06CED86
:10FCA00075E080E090E00E94986E66E97FE0CE010A
:10FCB00001960E942A5F4AE050E06FEF7FEFCE018D
:10FCC00001960E948C3FCE0101960E94505E62E335
:10FCD00070E080E090E0CBC00E94283F6EE170E0D1
:10FCE00080E090E00E94986E0E94298E6B017C015A
:10FCF00064E670E080E090E00E94986E6FE07AE049
:10FD00008FEA93E10E94ED5D21E0B701A601CE01EB
:10FD100001960E94845EBE016F5F7F4F8FEA93E180
:10FD20000E94C15DCE0101960E94505E6FEA73E1B0
:10FD3000CE0101960E94325F4AE050E060E070E040
:10FD4000CE0101960E94C540CE0101960E94505EF0
:10FD50000E946A3F6CE27DE08FEA93E10E94B35D0E
:10FD6000C092DB14D092DC14E092DD14F092DE1429
:10FD700020E030E040EF51E4C701B6010E9477A7D0
:10FD800087FD03C066E87FE054C020E030E040ED2E
:10FD900051E4C701B6010E9477A787FD1FC066E73F
:10FDA0007FE0CE0101960E942A5F4AE050E06FEFAB
:10FDB0007FEFCE0101960E948C3FCE0101960E94FA
:10FDC000505E8091BD04882331F06CED75E080E0D9
:10FDD00090E00E94986E66E67FE02BC020E030E065
:10FDE00040EB51E4C701B6010E9477A787FD03C02D
:10FDF00068E57FE01EC069E47FE0CE0101960E94C5
:10FE00002A5F4AE050E06FEF7FEFCE0101960E943B
:10FE10008C3FCE0101960E94505E8091BD048823E4
:10FE200031F06CED75E080E090E00E94986E6BE33D
:10FE30007FE0CE0101960E942A5F4AE050E06FEF1A
:10FE40007FEFCE0101960E948C3FCE0101960E9469
:10FE5000505E6CE271E080E090E00E94986E8091CC
:10FE6000BD04882331F068EE73E080E090E00E94EA
:10FE7000986E2C960FB6F894DEBF0FBECDBFDF9103
:10FE8000CF91FF90EF90DF90CF90BF90AF909F9079
:10FE90008F900895CF93DF93FC0124813581232B2C
:10FEA00069F0EC01BC018EE990E10E948860BE011E
:10FEB00084E69FE0DF91CF910C948860DF91CF9131
:10FEC0000895CF92DF92EF92FF92CF93C0914912A3
:10FED000C43014F5C1300CF04DC0C11179C00E947E
:10FEE000736ABC01990F880B990B0E9438A420E01B
:10FEF00030E040EA50E40E9497A420E030EC4FE765
:10FF000054E40E9488A620914A1230914B124091ED
:10FF10004C1250914D1259C0C43009F059C00E9482
:10FF2000736ABC01990F880B990B0E9438A420E0DA
:10FF300030E040EA50E40E9497A420E030EC4FE724
:10FF400054E40E9488A620E030E040EA50E40E9499
:10FF500088A620E030E040E851E40E9497A420E029
:10FF600030E040E850E40E94C2A520E030E04AE7DB
:10FF700054E42BC00E94736ABC01990F880B990B43
:10FF80000E9438A42AE137E64CE950E40E9497A485
:10FF900020914A1230914B1240914C1250914D12C7
:10FFA0000E94C1A56B017C01EC2FEE0FFF0BE55306
:10FFB000FA4F80819181BC01990F880B990B0E94A7
:10FFC00038A49B01AC01C701B6010E9488A603C0FA
:10FFD00060E070E0CB01CF91FF90EF90DF90CF9089
:10FFE0000895CF92DF92EF92FF927C0180914612AA
:10FFF000082E000C990B0E94619F039714F5C7010E
:020000021000EC
:100000000E94736ABC01990F880B990B0E9438A457
:100010006B017C018091471290914812BC01990FAD
:10002000880B990B0E9438A49B01AC01C701B60153
:100030000E9497A420E030EC4FE754E40E9488A689
:1000400003C060E070E0CB01FF90EF90DF90CF90B5
:100050000895DF92EF92FF920F931F93CF93DF9358
:10006000CDB7DEB762970FB6F894DEBF0FBECDBF37
:100070008C011092C9146FEB7CE0CE0101960E94B6
:100080003A5FFF24F3948EE990E10E94FE6A20918A
:10009000C91418161906ECF521113BC08EE990E140
:1000A0000E94DC6A682F8093C8148A3039F06D3062
:1000B00029F0CE0101960E94A05D24C08D819E8111
:1000C000892B01F1F092C9146FE27DE0CE01079611
:1000D0000E943A5FBE016F5F7F4FCE0107960E947C
:1000E000605DBC01CE010D960E94325FCE010D967F
:1000F0000E946B45CE010D960E94505ECE01079680
:100100000E94505E6AE070E080E090E00E94986E8D
:10011000BACF222351F02091C9148D819E812111E3
:1001200093C0009709F090C066C0E12CF12CDD244B
:10013000D39484E69FE00E94FE6A1816190624F5FF
:1001400084E69FE00E94DC6A682F8093C8148A309E
:1001500071F08D3061F08091C914811108C0CE0119
:1001600001960E94A05D8FEFE81AF80A06C08D8103
:100170009E81892B11F0D092C91465E070E080E077
:1001800090E00E94986ED5CF64E170E080E090E04E
:100190000E94986EEF2809F4BECF8D819E81892B35
:1001A00009F4B9CF68E37DE0CE0107960E943A5F7B
:1001B000BE016F5F7F4FCE0107960E94605DBC015C
:1001C000CE010D960E94325FCE010D960E946B45C6
:1001D000CE010D960E94505ECE0107960E94505EA1
:1001E00084E69FE00E94926D64E170E080E090E020
:1001F0000E94986E90CF64E670E080E090E00E94EC
:10020000986E0E94D06ECB0168EE73E00E94FDA84C
:10021000CB0164E670E00E94FDA88236910574F07F
:100220008091DE0D81110AC08BEB93E10E94495C45
:10023000613071058105910509F456C06FEB7CE0D2
:10024000C8010E943A5F52C0019709F046C066EEAD
:100250007CE0CE010D960E943A5FBE01635F7F4F46
:10026000CE0101960E942E5D811116C068EF77E0E5
:10027000CE0107960E943A5FBE01695F7F4FCE01B3
:1002800001960E942E5DFF24F3948111F12CCE0182
:1002900007960E94505E01C0F12CCE010D960E947F
:1002A000505EFF20A1F040E050E0BE016F5F7F4F45
:1002B000CE0107960E94394BBE01695F7F4F8BEBE1
:1002C00093E10E94175ECE0107960E94505E64E1A2
:1002D00070E080E090E00E94986EBE016F5F7F4FFB
:1002E000C8010E94225F02C014DBA8CFCE01019694
:1002F0000E94505EC80162960FB6F894DEBF0FBE32
:10030000CDBFDF91CF911F910F91FF90EF90DF90C4
:1003100008954F925F926F927F92AF92BF92CF9269
:10032000DF92EF92FF920F931F93CF93DF93CDB79E
:10033000DEB762970FB6F894DEBF0FBECDBF81E087
:1003400080931402CE01019684DEBE016F5F7F4F61
:1003500087EC93E10E94175ECE0101960E94505EE9
:100360000091CB131091CC130115110509F0BEC0FB
:100370000E94888EF82E811107C06FEB7CE0CE01C1
:1003800001960E943A5FA7C08091250E882351F103
:100390006EE37DE0CE0101960E943A5FBE016F5F81
:1003A0007F4F8EE990E10E94995FBE016F5F7F4FA2
:1003B00084E69FE00E94995FCE0101960E94505E04
:1003C0006F2D8EE990E10E94925F8EE990E10E948C
:1003D00075606F2D84E69FE00E94925F84E69FE047
:1003E0000E9475602AE2F2121092E70D0E94D06E10
:1003F0006093E30D7093E40D8093E50D9093E60D0B
:100400006F2DCE0107960E940A5F8F2D0F2C000CD6
:10041000990BC0970A97D8F5CE0107960E94495CC0
:10042000633071058105910534F562E370E080E089
:1004300090E00E94986E0E94888E81110AC00F5F22
:100440001F4F05311105B9F06EE170E080E090E0DA
:10045000F0CF8B3084F0682FCE0101960E940A5FA6
:10046000BE016F5F7F4FCE0107960E94C15DCE0136
:1004700001960E94505EBE01695F7F4FCE010196DA
:100480000E94225FCE0107960E94505E24C06F2D0D
:10049000CE0101960E940A5FBE016F5F7F4FCE01C1
:1004A00007960E94175ECE0101960E94505E62E39D
:1004B00070E080E090E00E94986E0E94888E81112A
:1004C000CACF0F5F1F4F0F311105A9F26EE170E027
:1004D00080E090E0F0CFBE016F5F7F4F87EC93E14B
:1004E0000E94175ECE0101960E94505E8091CB1350
:1004F0009091CC13892B09F060C181EF94E10E94A7
:100500006F38892B39F46FEB7CE0CE0101960E94A5
:100510003A5F48C14091F5145091F6146091F71478
:100520007091F814CE010D960E944E9A8091250E7E
:10053000882309F44EC064E47DE0CE0101960E9458
:100540003A5FBE01635F7F4FCE0101960E94605DFE
:1005500062E179E00E94495DBC01CE0107960E94EC
:10056000325FBE01695F7F4F8EE990E10E94995F23
:10057000BE01695F7F4F84E69FE00E94995FCE01D4
:1005800007960E94505ECE0101960E94505E4091F7
:10059000F5145091F6146091F7147091F81420E15D
:1005A0008EE990E10E94E05F8EE990E10E94756023
:1005B0004091F5145091F6146091F7147091F8146D
:1005C00020E184E69FE00E94E05F84E69FE00E94D5
:1005D000756060E070E0CE010D960E941D5D182FE1
:1005E0008A3211F01092E70D0E94D06E6093E30DF5
:1005F0007093E40D8093E50D9093E60D6FEB7CE036
:10060000CE0107960E943A5F812F110F990BC09778
:100610000A9708F05FC0CE010D960E94495C6330D6
:100620007105810591050CF0A3C06CE271E080E0DA
:1006300090E00E94986E82E08093471110924B11D7
:10064000C12CD12C760181EE94E10E946F38892B68
:1006500091F48EE1C816D104E104F10449F16EE190
:1006600070E080E090E00E94986E2FEFC21AD20AEC
:10067000E20AF20AE8CF2EE1C216D104E104F10445
:10068000B9F04091E5145091E6146091E71470912F
:10069000E814CE0101960E944E9ABE016F5F7F4F13
:1006A000CE0107960E94175ECE0101960E94505E11
:1006B0008B859C85892B39F0BE01695F7F4FCE0108
:1006C0000D960E94C15D6FEB7CE0CE0107960E9403
:1006D000ED5D4EC06CE271E080E090E00E94986EAB
:1006E00082E08093471110924B11C12CD12C7601DE
:1006F00081EE94E10E946F38892B91F42EE1C216AD
:10070000D104E104F10449F16EE170E080E090E091
:100710000E94986E8FEFC81AD80AE80AF80AE8CF44
:100720008EE1C816D104E104F104B9F04091E5145A
:100730005091E6146091E7147091E814CE0101968F
:100740000E944E9ABE016F5F7F4FCE0107960E94B6
:10075000175ECE0101960E94505E8B859C85892B89
:1007600039F0BE01695F7F4FCE010D960E94C15DD9
:1007700064E670E080E090E00E94986E82E08093F2
:10078000471110924B11BE01635F7F4FCE0101965E
:100790000E94225FCE0107960E94505ECE010D9608
:1007A0000E94505EBE016F5F7F4F87EC93E10E9415
:1007B000175ECE0101960E94505E8091CB139091FE
:1007C000CC13892B09F441C08091250E8823A1F117
:1007D00061EC7CE0CE0101960E943A5FBE016F5F42
:1007E0007F4F87EC93E10E942E5D182FCE0101967A
:1007F0000E94505E111120C069E47DE0CE01019697
:100800000E943A5F67EC73E1CE0101960E94605D41
:1008100062E57DE00E94495DBC01CE0107960E9421
:10082000325FCE01079636DBCE0107960E94505EFE
:10083000CE0101960E94505E6AE070E080E090E098
:100840000E94986E0E947808E9C18091A4128823C2
:1008500009F49BC18091AE129091AF1297FF04C032
:100860001092AF121092AE128091AC129091AD1214
:10087000181619069CF42091AE123091AF12281769
:10088000390764F01092A4121092A9128CE291E040
:100890000E948F791092AF121092AE12E091B012B6
:1008A0008091AB12E817D4F18091DE0D811107C061
:1008B0008091AC129091AD121816190634F50E9471
:1008C000D06E28EE33E040E050E00E9490A5CA01CF
:1008D000B9010E9436A42091DF0D3091E00D4091C6
:1008E000E10D5091E20D0E94C1A5209119023091B5
:1008F0001A0240911B0250911C020E9477A7181601
:100900000CF08CC11092B01289C11092A9121092F1
:10091000A4128CE291E00E948F7980C10E2F0E2EDE
:10092000000C110B8AE0E802F0011124E755FD4E9E
:10093000E7840E2C000CFF088091B112A82E880FBE
:10094000BB080E94D06E4090A0125090A1126090FF
:10095000A2127090A312641975098609970928EEEE
:1009600033E040E050E00E9490A5CA01B9010E9426
:1009700036A42B013C016701F7FE04C0CC24DD2422
:10098000CE18DF08C501B7FE02C080E090E08C15EC
:100990009D050CF099C08AE0809FF001819FF00DC9
:1009A0001124E755FD4E60897189072E000C880BD4
:1009B000990B0E9438A49B01AC01C301B2010E94B3
:1009C00077A718160CF02AC1F7FE09C08091AE1265
:1009D0009091AF12B6010E94FDA8892B71F48AE0B4
:1009E000809FF001819FF00D1124E755FD4E868513
:1009F000082E000C990B0E9442240E94D06E609336
:100A0000A0127093A1128093A2129093A3128091CE
:100A1000B1128F5F8093B112082E000C990B8C15C8
:100A20009D050CF4FBC08091AB12082E000C990BB5
:100A30000197081719070CF4F1C08091AE1290913C
:100A4000AF1201969093AF128093AE128091DE0D9B
:100A5000811108C08091AC129091AD121816190640
:100A60000CF0DCC08CE291E00E948F7962E170E1D1
:100A70008FEA93E10E94C75D6091AE127091AF1250
:100A80004AE0CE0101960E94DF5EBE016F5F7F4F9C
:100A90008FEA93E10E94C15DCE0101960E94505EF3
:100AA0006CED75E080E090E00E94986E6FEA73E173
:100AB000CE0101960E94325FCE010196EBD9CE01A4
:100AC00001960E94505EAAC03AE0F32EF09EF0011B
:100AD000F19EF00D1124E755FD4E62897389072EB2
:100AE000000C880B990B0E9438A49B01AC01C30138
:100AF000B2010E9477A718160CF090C01092B112A4
:100B00008091B0128F5F8093B012082E000C990B69
:100B10002091AB12022E000C330B8217930704F5C1
:100B2000F89EF001F99EF00D1124E755FD4E8785E2
:100B300087FD06C08685082E000C990B0E94422472
:100B40000E94D06E6093A0127093A1128093A212A3
:100B50009093A3128091B1128F5F8093B1125EC007
:100B60000E94D06E28EE33E040E050E00E9490A555
:100B7000CA01B9010E9436A46093DF0D7093E00DA5
:100B80008093E10D9093E20D49C08091DE0D8823A2
:100B900009F44FC00E94D06E28EEC22E23E0D22E60
:100BA000E12CF12CA70196010E9490A5CA01B90180
:100BB0000E9436A42091DF0D3091E00D4091E10DAF
:100BC0005091E20D0E94C1A52091190230911A02A4
:100BD00040911B0250911C020E9477A718164CF5F9
:100BE0000E94D06EA70196010E9490A5CA01B9018A
:100BF0000E9436A46093DF0D7093E00D8093E10DA9
:100C00009093E20D8091DF149091E0140E944224B1
:100C100064E170E080E090E00E94986E8091DE0DCB
:100C2000882331F164E670E080E090E00E94986EE5
:100C30001FC00E94D06E0091E30D1091E40D209131
:100C4000E50D3091E60DDC01CB01801B910BA20B71
:100C5000B30B88349E4EA105B10500F31092C61463
:100C600060E08BEB94E10E94E47210921202D6CF06
:100C700062960FB6F894DEBF0FBECDBFDF91CF9165
:100C80001F910F91FF90EF90DF90CF90BF90AF90AA
:100C90007F906F905F904F900895BF92CF92DF92B8
:100CA000EF92FF920F931F93CF93DF93CDB7DEB7F1
:100CB00062970FB6F894DEBF0FBECDBF8C016B01FB
:100CC00068E87DE0CE0101960E943A5F60E170E144
:100CD000C8010E942A5F76012FEFE21AF20A4AE069
:100CE000B701CE0107960E94DF5EBE01695F7F4FAC
:100CF000CE010D960E94325F62E179E0CE010D9641
:100D00000E94495DBC01C8010E94C15DCE010D96E3
:100D10000E94505ECE0107960E94505E8AE0B82E77
:100D2000BE9CC001BF9C900D1124FC01E755FD4EF7
:100D30007F018081082E000C990B0E9477AB892BD4
:100D400009F4B6C0B701CE0107960E943A5FBE0112
:100D5000695F7F4FCE010D960E94325F63EA7BE0B0
:100D6000CE010D960E94495DBC01C8010E94C15D83
:100D7000CE010D960E94505ECE0107960E94505EF5
:100D8000BC9CC001BD9C900D11249C0127553D4E7B
:100D90007901F9016685062E000C770B4AE0CE0139
:100DA00007960E94DF5EBE01695F7F4FCE010D9600
:100DB0000E94325F64E57DE0CE010D960E94495DA0
:100DC000BE016F5F7F4F0E94605DBC01C8010E9441
:100DD000C15DCE010D960E94505ECE0107960E9425
:100DE000505E69E070E1C8010E94715DF70167859E
:100DF000062E000C770B4AE0CE0107960E94DF5EBC
:100E0000BE01695F7F4FCE010D960E94325FBE0129
:100E10006F5F7F4FCE010D960E94605DBC01C801DF
:100E20000E94C15DCE010D960E94505ECE010796D4
:100E30000E94505E63E070E1C8010E94715DF7019D
:100E4000608971894AE0CE0107960E94DF5EBE018B
:100E5000695F7F4FCE010D960E94325FBE016F5FCA
:100E60007F4FCE010D960E94605DBC01C8010E94BB
:100E7000C15DCE010D960E94505ECE0107960E9484
:100E8000505E6EEF7FE0C8010E94715DF7016289DC
:100E900073894AE0CE0107960E94DF5EBE01695F5A
:100EA0007F4FC8010E94C15DCE0107960E94505E2F
:100EB000CE0101960E94505EC80162960FB6F8946A
:100EC000DEBF0FBECDBFDF91CF911F910F91FF907D
:100ED000EF90DF90CF90BF9008958F929F92AF9246
:100EE000BF92EF92FF920F931F93CF93DF93D82F70
:100EF000C62F10921D1410921E1410921F141092DF
:100F000020141092211461E00E940F6E60E08D2F7A
:100F10000E94DD6D6C2F70E080E090E00E94986E82
:100F200060E08D2F0E940F6E8BE990E00197F1F742
:100F300000E911E08D2F0E94B36D892B31F401502F
:100F40001109C1F78EEF9FEF51C000E911E08D2F1D
:100F50000E94B36D019721F401501109C1F7F2CF3E
:100F600018E2C0E800E020E9E22EFF24F3948D2F80
:100F70000E94B36D892B29F481E0E81AF108B9F7D2
:100F8000E1CF0E94736E4B015C0190E9E92EFF24D2
:100F9000F3948D2F0E94B36D019729F481E0E81A34
:100FA000F108B9F7CFCF0E94736EDC01CB0188192D
:100FB0009909AA09BB098997A105B10538F0E02F65
:100FC000F0E0EB5EFB4E80858C2B80872C2F30E091
:100FD000359527952115310511F0C22F02C00F5FFD
:100FE000C0E8115009F0BFCF80E090E0DF91CF91D1
:100FF0001F910F91FF90EF90BF90AF909F908F90B7
:101000000895EF92FF920F931F93CF93DF93C82F12
:101010008B017A0183E50E9406766C2F8BE391E1C8
:101020000E9432990E94A47583E50E940676B80159
:1010300083E590E00E94277AE701CE018E199F098F
:101040003091180F2091190F321731F08BE391E195
:101050000E94EA708993F1CF8017910729F01092CE
:10106000231481E080932414DF91CF911F910F917D
:10107000FF90EF900C94A475CF93DF93AC01990F80
:10108000660B770B2AE030E08EE990E10E94286041
:10109000EC018EE990E10E9475608C0F9D1FDF913D
:1010A000CF9108951F93CF93DF931F92CDB7DEB7F3
:1010B000162FAE014F5F5F4F61E070E0A2DF8981C4
:1010C00090E002C0959587951A95E2F781700F9090
:1010D000DF91CF911F910895CF93DF93D82FC62F23
:1010E00083E50E9406766D2F8BE391E10E94329991
:1010F0006C2F8BE391E10E943299DF91CF910C9498
:10110000A475FF920F931F93CF93DF931F92CDB7D8
:10111000DEB7182F062FF42EAE014F5F5F4F61E050
:1011200070E06FDF8981FF2049F041E050E001C0AD
:10113000440F0A95EAF7482B498309C021E030E0C3
:1011400001C0220F0A95EAF7209528232983698197
:10115000812FC2DF0F90DF91CF911F910F91FF90F0
:101160000895CF93DF9342E00E944A76EC018EE926
:1011700090E10E9475608C0F9D1FDF91CF910895C3
:10118000AF92BF92CF92DF92EF92FF921F93CF93D5
:10119000DF93CDB7DEB72A970FB6F894DEBF0FBE48
:1011A000CDBF182F41E354E166E070E082E39F83F6
:1011B00028DF2091321430E0322F22278091311421
:1011C000282B3A8329832091341430E0322F2227B0
:1011D00080913314282B3C832B832091361430E0EC
:1011E000322F222780913514282B3E832D839E0198
:1011F0002F5F3F4F590155E2C52E54E1D52EE12E08
:101200009F81F92EF501619171915F01F6012191A4
:101210003191419151916F01072E000C880B990B70
:101220002F83388749875A870E9438A42F813885B1
:1012300049855A850E9497A4F70161937193819320
:1012400091937F01F1E3CF16F4E1DF06D9F62A96F8
:101250000FB6F894DEBF0FBECDBFDF91CF911F91C7
:10126000FF90EF90DF90CF90BF90AF9008953F92A6
:101270004F925F926F927F928F929F92AF92BF92A6
:10128000CF92DF92EF92FF920F931F93CF93DF9352
:1012900000D01F921F92CDB7DEB7982E0E94D06E5D
:1012A0002B013C0120ED420E27E0521E611C711CF7
:1012B00060E08091A6140E94DD6D35E0832ECE01A2
:1012C00001966C01AA24A394B12C55E0352E380E5A
:1012D000F601282D11922A95E9F7860127E0E22EE2
:1012E000F12C8091A7140E94B36D019739F40E94EC
:1012F000D06E641575058605970598F38091A7143F
:101300000E94B36D892B39F40E94D06E6415750567
:101310008605970598F38091A8140E94B36D892BD8
:1013200051F0F8012081C5010E2C01C0880F0A94EC
:10133000EAF7822B8083F1E0EF1AF10890F60F5F55
:101340001F4F3012CBCF0E94D06E641575058605F5
:10135000970550F061E08091A6140E94DD6D60E079
:1013600070E080EC9FE72CC089818911B1CF9B810F
:101370008A81980F990D8C818913AACF8D818D3028
:1013800009F0A6CF61E08091A6140E94DD6D6A810C
:101390008B8170E0762F6627680F711D072E000C79
:1013A000880B990B0E9438A420E030E040E85DE310
:1013B0000E9497A423E333E948E853E40E94C1A5BF
:1013C0000F900F900F900F900F90DF91CF911F9182
:1013D0000F91FF90EF90DF90CF90BF90AF909F90D4
:1013E0008F907F906F905F904F903F900895AF9255
:1013F000BF92CF92DF92EF92FF920F931F93CF9302
:10140000DF931F92CDB7DEB75C01D62EE72EFC012D
:101410008585811105C0C5010E94DC71811106C05E
:10142000F50113861586148680E065C040E060EF04
:10143000C5010E94707101E0F12CC12C11E0C501C1
:101440000E941D71682FC50169830E941D71698109
:10145000613019F48130B9F433C04F2D50E0681376
:101460001BC0F5018385181730F4E40FF51F838145
:10147000802349F402C0181731F060E0193058F4A5
:10148000F501148708C0F501EF0DF11D8381802B54
:10149000838361E009C0C12EF501E40FF51F93813C
:1014A000802F809589238383C5010E9441711F5F2E
:1014B000000F11F4F39401E0F7E0FF1508F0BFCF3F
:1014C000113408F4ADCFF501C386C11002C081E02C
:1014D0008587F5018381882309F4A2CFD50113966E
:1014E000ED2DFE2D9501255F3F4F8D918193A21724
:1014F000B307D9F781E00F90DF91CF911F910F9142
:10150000FF90EF90DF90CF90BF90AF9008959F92A3
:10151000AF92BF92CF92DF92EF92FF920F931F9301
:10152000CF93DF93CDB7DEB761970FB6F894DEBFE8
:101530000FBECDBF8C018CE0F8018183C12CD12C72
:101540002FE5E22E3FE7B32E4FE1A42E5FE3952E69
:10155000F801848190E0C816D9060CF0A2C04C2D89
:10156000BE01665F7F4FC8010E942570F80181812E
:10157000893038F0F82EFCE0F81728F49CE0F92EBA
:1015800002C089E0F82E8A85803139F0BE01665F9D
:101590007F4FC8010E94F86F01C08CE08F1509F4DD
:1015A0007CC0AE014F5F5F4FBE01665F7F4FC801D9
:1015B0000E948F6F882309F470C08A85803109F4F6
:1015C0006CC08BE0F81651F0ECE0FE1629F0FAE062
:1015D000FF1206C09D8205C0BD8203C0ED8201C01E
:1015E000AD82F801868197810E94DC71BE01665F41
:1015F0007F4FF801868197810E94B17140E06EE4CF
:10160000F801868197810E94707140E06B81F8013A
:10161000868197810E94707140E06C81F80186811B
:1016200097810E9470718A85803139F040E06D8128
:10163000F801868197810E947071F80186819781F7
:101640000E94DC71BE01665F7F4FF8018681978141
:101650000E94B171F801408168E4868197810E94FF
:10166000707164E170E080E090E00E94986EF80193
:101670008081882331F06AE070E080E090E00E9491
:10168000986EF801868197810E94DC71F801818152
:10169000F81608F4F82EF801F182FFEFCF1ADF0AEE
:1016A00057CF61960FB6F894DEBF0FBECDBFDF9166
:1016B000CF911F910F91FF90EF90DF90CF90BF904F
:1016C000AF909F9008950F931F93CF93DF93FC01EA
:1016D000248135812115310519F4FB01108211C0D7
:1016E000EA0121972C173D0708F4E9018B01FC0161
:1016F00060817181AE01C8010E94A4ABC00FD11FEF
:101700001882DF91CF911F910F91089596E0899FE4
:10171000D0011124A95CBB4E90967C936E935F9789
:1017200091E091969C9391979091A314E091A414C9
:10173000F091A514992339F0309751F0811108C028
:101740008091531404C0309719F05C968C911994D1
:1017500008950F931F93CF93DF93C82FD62F86E062
:10176000C89FF0011124E95CFB4E11A2878D90A166
:1017700081309105E9F01CF4892B49F041C0823099
:101780009105A1F10397E1F560E070E033C06623B5
:10179000B9F161E070E08C2FB9DF0E94D06E6093E8
:1017A0008F1470939014809391149093921428C086
:1017B0000E94D06E00918F1410919014209191147A
:1017C00030919214AB01BC01401B510B620B730BA7
:1017D0008091A1149091A214A0E0B0E08417950725
:1017E000A607B70718F462E070E004C0D11108C082
:1017F00063E070E08C2FDF91CF911F910F9186CF26
:10180000DF91CF911F910F9108950F931F93CF9365
:10181000DF931F92CDB7DEB7682F87E769830E94F9
:10182000067669818BE391E10E9432990E94A4754A
:1018300087E70E94067662E070E087E790E00E940A
:10184000277A8BE391E10E94EA7000E010E0182F04
:101850008BE391E10E94EA70082B192B0E94A4757A
:10186000C8010F90DF91CF911F910F91089587E7E5
:101870000E94067664EF8BE391E10E9432996EE25A
:101880008BE391E10E9432990E94A47565E070E0BB
:1018900080E090E00E94986E86EFB7CF3F924F9223
:1018A0005F926F927F928F929F92AF92BF92CF92F0
:1018B000DF92EF92FF920F931F93CF93DF93CDB7F9
:1018C000DEB728970FB6F894DEBF0FBECDBFCFDFCF
:1018D0006C01E12CF12C1091CD131295110F110F09
:1018E000107C1C5C87E70E94067664EF8BE391E135
:1018F0000E943299612F8BE391E10E9432990E94FC
:10190000A4758091CD13811105C065E070E080E081
:1019100090E012C0813029F468E070E080E090E04F
:101920000BC0823029F46EE070E080E090E004C0EB
:101930006AE170E080E090E00E94986E86EF65DFDB
:101940004C01A12CB12CBA2CA92C982C882488EFFE
:101950000E94307A882A3090CD138091E2139091C2
:10196000E313A7019601281B390B41095109A091E6
:10197000E013B091E1130E9480A56B017C01AFE000
:10198000F594E794D794C794AA95D1F76091DA13A8
:101990007091DB13CB01770FAA0BBB0BBC01CD0100
:1019A000BBE0660F771F881F991FBA95D1F720916A
:1019B000DC133091DD138901330F220B330BA901A6
:1019C00098012C0D3D1D4E1D5F1D0E9464A5C20E89
:1019D000D31EE41EF51E20EAC21A2FE0D20AE10847
:1019E000F108A7019601C701B6010E94DAA89B0180
:1019F000AC011CE055954795379527951A95D1F779
:101A000029833A834B835C830091CE131091CF13CB
:101A1000A091D213B091D313A70196010E948AA579
:101A20002B013C018DE075946794579447948A95F7
:101A3000D1F7A091D413B091D51329813A814B816C
:101A40005C810E948AA5BB2797FDB095AB2F840DC2
:101A5000951DA61DB71D0296A11DB11D32E0B595BD
:101A6000A795979587953A95D1F79C01AD01305888
:101A70004F4F5F4FA091DE13B091DF130E9480A5FE
:101A80002B013C014FE076946794579447944A9514
:101A9000D1F788E090E083199109A501940104C071
:101AA00056954795379527958A95D2F72D833E838E
:101AB0004F8358874801110FAA08BB0852E0880CD1
:101AC000991CAA1CBB1C5A95D1F7A091D613B091B2
:101AD000D71329813A814B815C810E948AA59B01A1
:101AE000AC016BE055954795379527956A95D1F7E9
:101AF00029833A834B835C83A091D013B091D11397
:101B0000A70196010E948AA5DC01CB017BE0B59577
:101B1000A795979587957A95D1F729813A814B8139
:101B20005C81820F931FA41FB51F880D991DAA1DEC
:101B3000BB1D032C04C0880F991FAA1FBB1F0A944A
:101B4000D2F7BC01CD016E5F7F4F8F4F9F4F24E0D6
:101B500030E040E050E00E9464A58D819E81AF811D
:101B6000B885821B930BA40BB50B9C01AD0180E5DE
:101B700093ECA0E0B0E0BC01CD0104C09695879540
:101B8000779567953A94D2F70E94DAA897FD0BC033
:101B9000660F771F881F991FA30192010E9490A5CD
:101BA00069017A010AC0A30192010E9490A569010E
:101BB0007A01CC0CDD1CEE1CFF1C9927F7FC9A95D2
:101BC0008F2D7E2D6D2D9B01AC010E94DAA89B010B
:101BD000AC01AEEDBBE00E9480A54C01BB2497FC9C
:101BE000B094AB2CA3E4B3EEA70196010E948CA5A0
:101BF000BB2797FDB095AB2F880D991DAA1DBB1D66
:101C00008153914FAF4FBF4F44E0B595A79597953E
